:100000000C94AA060C94F9060C94F9060C94F906C3
:100010000C94F9060C94F9060C94F9060C94F90664
:100020000C94F9060C948F150C94F9060C94F906AF
:100030000C942D300C94F9060C94F9060C94F906E6
:100040000C94F9060C94F9060C9424140C94F906FB
:100050000C94B10B0C94F9060C947B0B0C94F906E0
:100060000C94861A0C94F9060C94E82E0C94F9065C
:100070000C9448700C94F9060C94446B0C94F9069B
:100080000C94F9060C94F9060C94F906B11AB61AF8
:10009000BB1AC41ADB1AF21A021B121B2F1B891D72
:1000A000F21A4B1C5C1C8B1CA91CC61C201D7B1D42
:1000B000591FD21F8E2005216E2111221C2483245A
:1000C000FD2447259225DF252C268626F3268D271D
:1000D00087280B2F3D2F4C2F772FA92FB92FF92FC2
:1000E000F92FE62FD12FD32FED2FDB2FE62FD62F91
:1000F000D82FED2FDB2FE62FE82FEA2FED2FF12F52
:100100000A0D426174743A0020332043656C6C73AD
:1001100020200020342043656C6C73202000204C8C
:100120006F77207761726E696E67206C6576656C9B
:100130003A2025642E2564000A0D466F756E6420F2
:10014000424C2D4374726C3A2000256420000A0D45
:100150000A0D2121204D495353494E4720424C2D31
:100160004354524C3A202564202121000A0D3D3D84
:100170003D3D3D3D3D3D3D3D3D3D3D3D3D3D3D3DAF
:100180003D3D3D3D3D3D3D3D3D3D3D3D3D3D3D3D9F
:100190003D000A0D43616C6962726174696E67208B
:1001A00070726573737572652073656E736F722EEE
:1001B0002E004F4B0A0D000A0D466C696768742DBE
:1001C00074696D65202575206D696E2020546F74EB
:1001D000616C3A2575206D696E000A0D436F6E746F
:1001E000726F6C3A200048656164696E67486F6C95
:1001F00064004E6F726D616C20284143432D4D6F3A
:10020000646529000A0D3D3D3D3D3D3D3D3D3D3D83
:100210003D3D3D3D3D3D3D3D3D3D3D3D3D3D3D3D0E
:100220003D3D3D3D3D3D3D3D3D0A0D00416E676C10
:10023000654E69636B20202020202020416E676C72
:1002400065526F6C6C202020202020204163634E7B
:1002500069636B20202020202020202041636352EE
:100260006F6C6C20202020202020202059617747AF
:1002700079726F2020202020202020204865696787
:1002800068742056616C7565202020204163635A94
:1002900020202020202020202020202047617320A3
:1002A000202020202020202020202020436F6D703F
:1002B0006173732056616C7565202020566F6C74D5
:1002C000616765205B302E31565D20205265636585
:1002D00069766572204C6576656C20204779726F6F
:1002E00020436F6D70617373202020204D6F746FF9
:1002F0007220312020202020202020204D6F746F7C
:100300007220322020202020202020204D6F746F6A
:100310007220332020202020202020204D6F746F59
:100320007220342020202020202020202020202067
:1003300020202020202020202020202020202020BD
:10034000202020202020202020202020566172699B
:100350006F4D657465722020202020204D4B334D59
:1003600061672043616C53746174652053657276D4
:100370006F2020202020202020202020486F76651C
:100380007267617320202020202020204375727224
:10039000656E74205B302E31415D202043617061B9
:1003A00063697479205B6D41685D202020202020E6
:1003B000202020202020202020202020202020203D
:1003C000202020202020202020202020202020202D
:1003D000202020202020202020202020202020201D
:1003E0002020202020202020202020204932432DA2
:1003F0004572726F72202020202020202020202093
:100400002020202020202020202020204750535F23
:100410004E69636B20202020202020204750535F0E
:10042000526F6C6C202020202020202021212120B0
:10043000494E434F4D50415449424C4520212121C2
:10044000002E000A0D20444143206F7220493243A0
:10045000204552524F522120436865636B20493238
:10046000432C2033567265662C2044414320616E34
:100470006420424C2D4374726C005B25695D005B07
:1004800025695D002B204D696B726F4B6F70746531
:1004900072202B0048573A5625642E256420535766
:1004A0003A25642E256425630053657474696E676C
:1004B0003A256420257300493243204552524F5259
:1004C000212121004D697373696E6720424C2D43D1
:1004D00074726C3A25642121004865696768743A32
:1004E000202025356900536574706F696E743A2554
:1004F00035690050726573737572653A2535690008
:100500004F66667365743A20202535690048656931
:1005100067687420636F6E74726F6C004449534156
:10052000424C45440048656967687420636F6E7487
:10053000726F6C0044495341424C454400616374FE
:100540002E2062656172696E67004E69636B3A20A6
:10055000202020202025356900526F6C6C3A202025
:100560002020202025356900436F6D706173733A38
:10057000202020253569004B313A25346920204B55
:10058000323A25346920004B333A25346920204B18
:10059000343A25346920004B353A25346920204B04
:1005A000363A25346920004B373A25346920204BF0
:1005B000383A25346920004E693A253469202052A2
:1005C0006F3A253469200047733A25346920204763
:1005D000693A253469200050313A25346920205089
:1005E000323A253469200050333A253469202050AE
:1005F000343A25346920004779726F202D205365E5
:100600006E736F72004E69636B2534692028253341
:10061000692E25692900526F6C6C253469202825C4
:1006200033692E25692900476965722534692028B8
:1006300025336929004E69636B20253469202825FC
:1006400033692E25782900526F6C6C20253469207F
:10065000282533692E2578290059617720202534F3
:1006600069202825336929004E69636B2025346988
:10067000202825336929282533692900526F6C6C9D
:100680002025346920282533692928253369290044
:1006900059617720202534692028253369292825A8
:1006A00033692900414343202D2053656E736F72D7
:1006B000004E69636B2025346920282533692900A1
:1006C000526F6C6C20253469202825336929005A23
:1006D0002020202025346920282533692900566FE1
:1006E0006C746167653A2020202533692E253169B5
:1006F000560043757272656E743A20202025336966
:100700002E2531694100506F7765723A20202020F4
:100710002025346957004469736368617267653ADC
:10072000202535696D41680052656365697665729B
:100730000052432D525353493A202020202534693A
:100740000052432D5175616C6974793A20253469E2
:100750000052432D4368616E6E656C733A253469AF
:1007600000436F6D706173730048656164696E6703
:100770003A20202535690056616C75653A202020A5
:10078000202535690053746172743A202020202599
:10079000356900506F7469313A2020253369005063
:1007A0006F7469323A202025336900506F746933C1
:1007B0003A202025336900506F7469343A2020258F
:1007C000336900506F7469353A2020253369005031
:1007D0006F7469363A202025336900506F74693789
:1007E0003A202025336900506F7469383A2020255B
:1007F000336900536572766F202000536574706F03
:10080000696E74202025336900506F736974696FB5
:100810006E3A202533690052616E67653A25336967
:100820002D2533690045787465726E436F6E74725E
:100830006F6C2020004E693A2534692020526F3AAF
:10084000253469200047733A253469202047693AE6
:10085000253469200048693A253469202043663AE6
:100860002534692000424C2D4374726C204572720D
:100870006F72732000253364202533642025336490
:10088000202533642000253364202533642025335C
:10089000642025336420002533642025336420251B
:1008A0003364202533642000424C2D4374726C2045
:1008B000666F756E6420002025632020202563204C
:1008C0002020256320202025632000202563202070
:1008D0002025632020202563202020256320002060
:1008E00025632020202D2020202D2020202D2000B9
:1008F000313000313100313200466C696768742D47
:1009000054696D65202000546F74616C3A2535750B
:100910006D696E004163743A20202535756D696EEE
:100920000028726573657429000A0D47656E65724B
:100930006174696E672064656661756C74205061CE
:1009400072616D6574657220536574202564000AB8
:100950000D5573696E6720506172616D65746572C3
:1009600020536574202564000A0D47656E65726129
:1009700074696E672064656661756C74204D697872
:100980006572205461626C65000A0D4D697865726C
:100990002D436F6E6669673A202725732720282527
:1009A00075204D6F746F727329000A0D3D3D3D3DFA
:1009B0003D3D3D3D3D3D3D3D3D3D3D3D3D3D3D3D67
:1009C0003D3D3D3D3D3D3D3D3D3D000A0D414343E7
:1009D000206E6F742063616C69627261746564215A
:1009E0000D0A000A0D506C6561736520636F6E6EB1
:1009F000656374205370656B7472756D20726563E6
:100A0000656976657220666F722062696E64696ED0
:100A100067204E4F572E2E2E006F6B2E0A0D00545E
:100A2000696D656F75742E0A0D0000008F001E0140
:100A3000AD013B02CA025803E603740402058F05A8
:100A40001B06A7063307BE074808D2085B09E3095F
:100A50006B0AF20A780BFD0B810C040D860D070E54
:100A6000870E060F840F00107B10F5106E11E51134
:100A70005B12CF124213B31323149214FE146A159F
:100A8000D3153B16A11605176717C8172718831823
:100A9000DE1837198E19E319361A871AD61A231B4E
:100AA0006E1BB61BFD1B411C831CC31C001D3C1D83
:100AB000751DAB1DE01D121E421E6F1E9A1EC31E29
:100AC000E91E0D1F2E1F4D1F691F841F9B1FB01F86
:100AD000C31FD31FE11FEC1FF51FFB1FFF1F0020CB
:100AE00003010000606500020101256601030202A6
:100AF000946602000303F1662532692E253169569A
:100B000000253033646D2025303364256300537431
:100B10006174757300253469202532693A253032B5
:100B200069002534696D2563004E69636B20526F3F
:100B30006C6C2020596177002534692025346920A8
:100B4000253469002532692E253169562020253348
:100B5000692E253169410025346957202536696D94
:100B60004168005361743A25303264004E6F466923
:100B700078003244466978003344466978003F3F44
:100B8000466978002F4447505300486F6D653A25F9
:100B90003033646D20253033642563004E6F204E62
:100BA0006176694374726C21000A0D7777772E4D58
:100BB000696B726F4B6F707465722E646520286369
:100BC0002920486953797374656D7320476D6248B5
:100BD000000A0D74686520757365206F662074685F
:100BE000697320736F667477617265206973206F13
:100BF0006E6C79207065726D6974746564200A0D7D
:100C00006F6E206F726967696E616C204D696B72DF
:100C10006F4B6F707465722D486172647761726595
:100C2000004143542044534C004A65746920736169
:100C300074656C6C6974005370656B7472756D20AB
:100C4000736174656C6C697420284C6F77207265D1
:100C5000736F6C7574696F6E29005370656B747275
:100C6000756D20736174656C6C6974202832303442
:100C70003829005370656B7472756D2073617465EB
:100C80006C6C6974004D756C74697369676E616C26
:100C90002050504D000A0D52656365697665723AC1
:100CA0002000756E6B6E6F776E2E205573696E67C0
:100CB0002050504D2E2E2E006E6F74207375707064
:100CC0006F72746564206279206861726477617202
:100CD0006521000A0D3D3D3D3D3D3D3D3D3D3D3DD8
:100CE0003D3D3D3D3D3D3D3D3D3D3D3D3D3D3D3D34
:100CF0003D3D3D3D3D3D3D3D000A0D466C6967680B
:100D000074436F6E74726F6C0A0D48617264776120
:100D100072653A25642E25640A0D536F66747761F7
:100D200072653A5625642E2564256320000A0D3D20
:100D30003D3D3D3D3D3D3D3D3D3D3D3D3D3D3D3DE3
:100D40003D3D3D3D3D3D3D3D3D3D3D3D3D3D3D3DD3
:100D50003D3D000011241FBECFEFD0E4DEBFCDBF6C
:100D600011E0A0E0B1E0E8E5F7EE00E00BBF02C063
:100D700007900D92A03DB107D9F718E0A0EDB1E0C2
:100D800001C01D92A433B107E1F77AEAE2E0F0E096
:100D900081E280935700D4907E010894E11CF11CFD
:100DA00020EF37EF41E050E087016FE0DA01C90141
:100DB0002F5F3F4F4F4F5F4FABBFFC018791F80153
:100DC00081938F01615067FFF1CFF7016EE0819150
:100DD00078277095615067FFFACF8889781729F0D6
:100DE000F7E9DF1611F40000FECF0E94BB070C9458
:100DF000AB730C9400008091D705E82FFF27EE0F0E
:100E0000FF1FED53F94F808191818D5E9F4F14F04C
:100E100010920301808191818A5B9F4FCCF4809175
:100E200003018823A9F481E08093030180913304B6
:100E30008F5F80933304853038F088EE93E0909391
:100E4000FF018093FE0104C066E970E00E949432C5
:100E50008091330499279093AD058093AC05089554
:100E60001F93CF93DF93182F882389F080E091E0C0
:100E70009F938F938DE391E19F938F93E091FF0375
:100E8000F091000409950F900F900F900F908091B2
:100E9000F905823308F046C084EF91E00E940F15F7
:100EA000EC01112329F0CE010E9418158823D9F3F3
:100EB00080911D0190911E012091F90582389105C4
:100EC00084F433E0239FC001112480930001112397
:100ED00059F168EC70E0832F0E94943288E091E031
:100EE00011C0822F9927880F991F880F991F80930F
:100EF00000011123C9F068EC70E084E00E94943294
:100F000083E191E09F938F938DE391E19F938F9382
:100F1000E091FF03F091000409950F900F900F905E
:100F20000F9002C080930001112309F1809100010C
:100F30006AE00E94FE72892F99279F938F93809178
:100F400000010E94FE7299279F938F938EE191E09A
:100F50009F938F938DE391E19F938F93E091FF0394
:100F6000F091000409958DB79EB708968DBFDF916B
:100F7000CF911F910895CFEFD0E4DEBFCDBF88247D
:100F8000992414B815B8B7EECB2EB3E0DB2E8EEC57
:100F90009FEFC80ED91ED7FEFACF189B06C0199B2B
:100FA00002C08DE007C08BE005C0199B02C084E140
:100FB00001C08AE08093020181E887B93E9A8FEFF1
:100FC00088B98BE184B981E085B98EE38AB987E479
:100FD0008BB9469A84B7877F84BF8091600088610F
:100FE000809360001092600080ED97E09093FF0185
:100FF0008093FE011092E9021092E8021092C80656
:101000001092C7061092EB021092EA021092ED02C3
:101010001092EC0220910201243128F088E894E03B
:10102000A0E0B0E004C08BE095E0A0E0B0E08093E9
:10103000930190939401A0939501B09396012A3067
:1010400011F0243111F4289801C0289A0E947815D3
:101050000E9449150E9445110E9411300E945919A1
:101060000E94A72E0E94B65D0E94F8670E947B6FC7
:10107000809102018C3010F4299A01C0299878944B
:101080000E94BC2D10924802109202020E94BD3EA6
:10109000809102028823E1F31092480288E391E0F4
:1010A0009F938F93ADE3AA2EA1E1BA2EBF92AF9288
:1010B000E091FF03F0910004099580EA9FE00E940F
:1010C0000F156C01C0E0D0E00F900F900F900F90C3
:1010D000F3E9EF2EF6E0FF2E8E01109202020E943D
:1010E000BD3E809102028823E1F3F801EC5BF94FE9
:1010F00085851816ACF408C0909302020E94BD3E8C
:10110000809102028823E1F3C6010E941815982FEE
:10111000882331F4F801EE56F94F8181882364F772
:10112000F701808187FF13C02196DF93CF9321972A
:101130008AE491E09F938F93BF92AF92E091FF0377
:10114000F091000409958DB79EB706968DBF219644
:101150000C5F1F4FE4E0F0E0EE0EFF1ECC30D10537
:1011600008F4BBCFC0E0D0E002E916E0E1E5EE2EE6
:10117000E6E0FE2EF801818187FD1CC0F701808129
:101180001816C4F42196DF93CF9321978EE491E053
:101190009F938F938DE391E19F938F93E091FF0352
:1011A000F0910004099581E08093FC018DB79EB712
:1011B00006968DBFF801818180788183219684E035
:1011C00090E0E80EF91E080F191FCC30D10590F2FF
:1011D0008CE691E09F938F93CDE3D1E1DF93CF93A2
:1011E000E091FF03F091000409950E94BD3E0F902D
:1011F0000F900F900F9082E991E09F938F93DF9370
:10120000CF93E091FF03F0910004099588EE93E0FD
:101210000E940F156C010E945F190F900F900F90A4
:101220000F90C6010E9418158823D9F382EB91E034
:101230009F938F93DF93CF93E091FF03F09100048E
:10124000099580E00E947833809102010F900F9001
:101250000F900F908A3011F0843111F4289801C05A
:10126000289A80ED97E09093FF018093FE0185E539
:10127000809335048EE090E00E94342C9927182F3B
:1012800000278FE090E00E94342C080F111D10936E
:10129000D5010093D4018AE090E00E94342C992774
:1012A000182F00278BE090E00E94342C080F111DAE
:1012B0001093D3010093D2010F5F1F4F39F080913B
:1012C000D4019091D5018F5F9F4F41F41092D501C9
:1012D0001092D4011092D3011092D2018091D201C8
:1012E0009091D3019F938F938091D4019091D501D8
:1012F0009F938F9387EB91E09F938F93DF93CF938F
:10130000E091FF03F091000409958DB79EB7089610
:101310008DBF8AED91E09F938F93DF93CF93E09100
:10132000FF03F091000409958091E3050F900F9061
:101330000F900F90E091FF03F091000482FF07C02F
:1013400086EE91E09F938F93DF93CF9308C082EF57
:1013500091E09F938F938DE391E19F938F930995F4
:101360000F900F900F900F900E94D01E88E893E18D
:101370009093BA018093B90181E0809334040E9474
:1013800030078091FC050E94E16E84E092E09F931B
:101390008F93DF93CF93E091FF03F09100040995C1
:1013A00080ED97E00E940F156C018AEF90E00E949B
:1013B0000F15EC010F900F900F900F90CE010E942F
:1013C0001815882339F084E690E00E940F15EC018F
:1013D0000E94377080910202882309F484C18091B1
:1013E0000F01882309F47FC1109202028091330417
:1013F000882319F00E94FB0602C00E940E410E9441
:10140000BD3E209102012A3011F0243111F42898B8
:1014100001C0289A8091EE02882331F08091EE027B
:1014200081508093EE0209C080916F0080628093AA
:101430006F001092C4061092C3068091B90190917A
:10144000BA0101979093BA018093B9018091B901D3
:101450009091BA01892B21F0809147028823A1F154
:101460008091B9019091BA01892BB1F40E94BD2EEF
:1014700085E090E09093BA018093B9018091BE0518
:101480009091BF0501969093BF058093BE05809112
:10149000BD0280688093BD0280910801909109018E
:1014A0008F5F9F4F19F58091E5028823F9F080E165
:1014B00097E29093FF018093FE0180E890E0909383
:1014C00009018093080112C02A3011F0243111F46F
:1014D000289801C0289A8091FE019091FF01892BE4
:1014E00029F48091BD028F778093BD028091020222
:1014F000882321F08091E502882311F40E9489114C
:101500000E94EF0DC6010E941815882309F4E7C058
:1015100084E190E0C80ED91E80910501882321F056
:1015200081508093050125C080933F041092C90229
:101530001092C8021092C7021092C6021092C50201
:101540001092C40280910801909109018F5F9F4F12
:1015500081F48091EE02882361F488E99AE3909304
:10156000FF018093FE0180E09CE09093090180934D
:1015700008018091D403882339F081508093D403EB
:101580008091BD028F7B11C01092D2031092D103C3
:101590001092D0031092CF038091FE019091FF0131
:1015A000892B29F48091BD0280648093BD028091D3
:1015B0000001282F332780911D0190911E01821771
:1015C0009307CCF48091BD0280628093BD0280912C
:1015D0000801909109018F5F9F4FC1F480E797E167
:1015E0009093FF018093FE0180E093E090930901C6
:1015F000809308010BC08091FE019091FF01892B1F
:1016000029F48091BD028F7D8093BD020E946961A3
:1016100084E08093FD018091E502882329F45AEA51
:10162000852E55E0952E12C08091D6018F5F809354
:10163000D601813359F41092D6018091D001909156
:10164000D10101969093D1018093D0010894811C1F
:10165000911C22E782162BE0920609F040C08824F4
:1016600099242091D4013091D5012F5F3F4F3093C1
:10167000D5012093D4018091D2019091D30101969C
:101680009093D3018093D201832F9927682F8EE006
:1016900090E00E943C2C8091D4019091D5019070F3
:1016A000682F8FE090E00E943C2C8091D2019091B5
:1016B000D301892F9927682F8AE090E00E943C2C63
:1016C0008091D2019091D3019070682F8BE090E0CF
:1016D0000E943C2C84E190E00E940F156C010E9456
:1016E000B9610E940D688091FD01882309F066CEE2
:1016F0000E94D75D63CE1F920F920FB60F921124F6
:101700008F939F93EF93FF93809107018823E1F4D8
:101710008091F0019091F10101969093F1018093F5
:10172000F001FC01EC51FB4FE081ED3019F0803A03
:10173000910539F41092F1011092F00181E080934B
:101740000701E093C60004C01092F1011092F0016D
:10175000FF91EF919F918F910F900FBE0F901F906F
:1017600018951F920F920FB60F9211242F933F934B
:101770004F935F936F937F938F939F93AF93BF9399
:10178000CF93EF93FF9390E08091C6008093E801A0
:101790005091F601503A10F09093F7018091E801D2
:1017A0008D3009F065C08091F701823009F060C08A
:1017B0009093F701852F99278E5B9B4FFC01329701
:1017C00040812091F2013091F301241B3109DC01A9
:1017D00011978C91281B3109C9019F709093F301D7
:1017E0008093F20146E0969587954A95E1F7982F08
:1017F000935C9093F4012F733070235C2093F50178
:101800008081981729F48C91281711F491E006C073
:1018100090E08091E5018F5F8093E501C091E70141
:10182000CC2309F074C0992309F471C081E080933E
:10183000E701580F5093E4015150E52FFF27EE5B6D
:10184000FB4F8DE0808380914404823509F05FC0B6
:101850000E94D01E88E190E02CE00FB6F894A89585
:10186000809360000FBE20936000C093FC014FC0C6
:101870002091F701822F992781309105F9F082306C
:1018800091051CF4892B21F040C0029711F13DC055
:101890008091E801833239F48091E701882319F4BB
:1018A00081E08093F7018091E8018093420481E018
:1018B0008093F6018091E801992722C02F5F209341
:1018C000F701E52FFF27EE5BFB4F8091E801808356
:1018D00009C0E52FFF27EE5BFB4F8091E801808375
:1018E000503A20F45F5F5093F60102C01092F70166
:1018F0002091E8018091F2019091F301820F911DF6
:101900009093F3018093F20102C01092F701FF91CE
:10191000EF91CF91BF91AF919F918F917F916F91F7
:101920005F914F913F912F910F900FBE0F901F909D
:101930001895AC01A0E0B0E09D01A817B90748F4E4
:10194000E4EEF4E08191280F311D1196A417B5073C
:10195000C8F33F70FD01EC51FB4FC90156E096956D
:1019600087955A95E1F7835C80831196FD01EC51D0
:10197000FB4F2F733070822F835C8083AB51BB4F42
:101980008DE08C93109207018091E4048093C6004F
:101990000895A0E0B0E0EFECFCE00C9477732C85A8
:1019A0009D850E85BB2483E28093E4049F59909328
:1019B000E5042093E60433E0E32EF12C002309F440
:1019C0009EC0CF84D888BE016D5E7F4FA989BA8939
:1019D0000150109709F493C01097B9F0F601EB0D80
:1019E000F11DB3949081119791F4002349F1FB010B
:1019F0006E5F7F4FDB01C080D1806E5F7F4F0D90A7
:101A0000BC91A02DBB24015002C090E019C01097DA
:101A1000B9F0F601EB0DF11DB3944081119791F4EB
:101A2000002341F1FB016E5F7F4FDB01C080D1805D
:101A30006E5F7F4F0D90BC91A02DBB24015002C062
:101A400040E018C01097B1F0F601EB0DF11DB39412
:101A50001081119781F4002371F0FB013296DB01B4
:101A6000CD90DC90BF016E5F7F4FA081B181BB2420
:101A7000015001C010E0F701EC51FB4F892F869512
:101A80008695835C80830894E11CF11CF701EC517E
:101A9000FB4F892F99278370907024E0880F991F3E
:101AA0002A95E1F755279A0194E0369527959A955E
:101AB000E1F7822B835C80830894E11CF11CF70121
:101AC000EC51FB4F4F705070440F551F440F551F82
:101AD000812F992726E0969587952A95E1F7842B03
:101AE000835C80830894E11CF11CF701EC51FB4FEF
:101AF0001F73135C10830894E11CF11C6ACFC701AB
:101B00000E94990CE9E00C949373A3E07A2F409122
:101B1000E4014650442309F458C0E72FFF27EE5B49
:101B2000FB4F80818D537F5FE72FFF27EE5BFB4FDD
:101B300020812D537F5FE72FFF27EE5BFB4F308126
:101B40003D537F5FE72FFF27EE5BFB4F60816D53B7
:101B50007F5F9927880F991F880F991F522F5295E1
:101B60005F70582B822F99278F709070F4E0880F48
:101B7000991FFA95E1F7232F26952695282B832F79
:101B8000992783709070E6E0880F991FEA95E1F736
:101B9000682B41504F3FC9F0EA2FFF27EE5BFB4F08
:101BA0005083AF5F41504F3F81F0EA2FFF27EE5B3C
:101BB000FB4F2083AF5F41504F3F39F0EA2FFF27A3
:101BC000EE5BFB4F6083AF5FA5CF85E494E090931D
:101BD000E3018093E201A350A093E1010895A1E005
:101BE000B0E0E5EFFDE00C947D738091E701882380
:101BF00009F43FC30E94850D80914304823609F0A9
:101C000001C28091440499278037910509F4ACC042
:101C100081379105A4F48636910509F458C18736B9
:101C2000910524F48B349105F1F0ECC18D369105CA
:101C300009F46FC08E36910509F453C0E3C18337B0
:101C4000910509F4E1C0843791052CF481379105A1
:101C500009F491C0D7C18437910511F189379105F5
:101C600009F46CC1CFC1E091E201F091E301808100
:101C7000918190930103809300032091FE023091A3
:101C8000FF02821B930B845E9D4F68E671E00E9409
:101C90001E73845B90409093FD028093FC02B2C15E
:101CA0008091E401A091E201B091E301853140F01F
:101CB00080E1EDE1F4E00D9001928A95E1F70DC02D
:101CC0008D919D910D90BC91A02D80931D049093BA
:101CD0001E04A0931F04B093200480EF8093DF01C3
:101CE00046C0809107018823E1F38DE490E09F9343
:101CF0008F9384E496E09F938F9381E08F938F93EB
:101D00008EE48F930E94C90C8DB79EB707968DBF46
:101D100079C1A091E201B091E3011C91113059F415
:101D20008DE4E4E4F6E00D9001928A95E1F70E94DB
:101D30003C2D198301C01982809107018823E1F3AA
:101D400081E090E09F938F93CE0101969F938F93B4
:101D500081E08F938F938DE48F930E94C90CADB770
:101D6000BEB71796ADBF4EC181E08093EA018FEFF9
:101D70008093050147C1E091E201F091E301808188
:101D80008F3F39F40E949F2DE091E201F091E30131
:101D90008083E091E201F091E3018081882311F4D6
:101DA00081E003C0863010F085E08083E091E2019D
:101DB000F091E30180810E94522CE091E201F091C8
:101DC000E30180818983809107018823E1F38DE617
:101DD00090E09F938F9386ED95E09F938F9381E0A2
:101DE00090E09F938F93CE0101969F938F9382E013
:101DF0008F9381E08F9381E58F930E94C90CEDB79B
:101E0000FEB73B96EDBFFEC02091E2013091E301A9
:101E1000D9018C918150853008F040C0F901818151
:101E20008235E1F52F5F3F4F8DE6E6EDF5E0D90114
:101E30000D9001928A95E1F7F90182910E94BB2CE5
:101E4000809114069927AA27BB27BC01CD0124EC59
:101E500039E040E050E00E94DF72DC01CB0180936A
:101E6000B3019093B401A093B501B093B6018091F2
:101E700015069927AA27BB27BC01CD010E94DF7256
:101E8000DC01CB018093AF019093B001A093B1012D
:101E9000B093B2010E949F2D898301C01982809165
:101EA00007018823E1F381E090E09F938F93CE01B7
:101EB00001969F938F9381E08F938F9383E58F9308
:101EC0000E94C90C8DB79EB707968DBF26C0E091C2
:101ED000E201F091E301E0818E2F8150853018F40A
:101EE0008E2F0E94522C0E949F2D89838091070182
:101EF0008823E1F381E090E09F938F93CE010196D8
:101F00009F938F9381E08F938F9386E48F930E94AA
:101F1000C90CADB7BEB71796ADBF8091E502882357
:101F200029F46EE670E089810E94943280E00E947C
:101F300030078091FC050E94E16E64C0E091E201EF
:101F4000F091E3018081992787FD90959093DE06BB
:101F50008093DD068181992787FD90959093E00617
:101F60008093DF068281992787FD90959093E20602
:101F70008093E1068381992787FD90959093E406ED
:101F80008093E3068481992787FD90959093E606D8
:101F90008093E5068581992787FD90959093E806C3
:101FA0008093E7068681992787FD90959093EA06AE
:101FB0008093E9068781992787FD90959093EC0699
:101FC0008093EB068085992787FD90959093EE0688
:101FD0008093ED068185992787FD90959093F00673
:101FE0008093EF068285992787FD90959093F2065E
:101FF0008093F1068385992787FD90959093F40649
:102000008093F3068091440499278436910509F45E
:10201000C5C085369105ACF48136910509F479C0C7
:10202000823691052CF48B34910509F455C019C101
:102030008236910509F47AC08336910509F489C086
:1020400010C18C36910509F4F7C08D3691054CF41A
:102050008736910509F402C18836910509F4BCC0A0
:1020600000C18437910529F08637910509F4F2C043
:10207000F8C08091E401A091E201B091E3018531C3
:1020800040F080E1EDE1F4E00D9001928A95E1F7F6
:102090000DC08D919D910D90BC91A02D80931D043C
:1020A00090931E04A0931F04B09320048091070115
:1020B0008823E1F31F92809104018F9384E58F932D
:1020C0000E94C90C8AEF8093DF018FEF8093050196
:1020D0000F900F900F90C5C0E091E201F091E301E5
:1020E0008081918190930103809300032091FE02EF
:1020F0003091FF02821B930B845E9D4F68E671E076
:102100000E941E73845B90409093FD028093FC02BA
:10211000A8C0E091E201F091E30180818093060183
:10212000803298F08FE1809306010FC0A091E20108
:10213000B091E3018BE0E5E3F4E00D9001928A9524
:10214000E1F780913E048093C6058FEF80930501EF
:1021500088C08091DB019091DC01892B89F4E091AA
:10216000E201F091E301E081EE2351F08AE0E89F83
:10217000C00111240E940F159093100480930F0446
:10218000E091E201F091E30190818AE0989FC00123
:1021900011249093DC018093DB0115C08FEF8093B5
:1021A0000501E091E201F091E30190818AE0989FBE
:1021B000C00111249093DE018093DD01892B19F079
:1021C00081E08093EC0180EA9FE00E940F159093DC
:1021D000D8018093D70145C08FEF80930501E0912E
:1021E000E201F091E301908197FD08C082E08093C5
:1021F000E9011092DA011092D9011AC090958091EC
:102200004202892B8093420291818AE0989FC0010B
:1022100011249093DA018093D90184E08093E9013D
:1022200080EA9FE00E940F159093D8018093D70118
:1022300081E08093ED0115C08FEF80930501E0915F
:10224000E201F091E30180818093430281E0809379
:10225000EE0107C081E08093EB0103C081E0809331
:10226000EF011092E7011092E3011092E201109247
:10227000E101E3E0CF5F0C949973982F8091C00047
:1022800085FFFCCF9093C60008950F931F9388E1BC
:102290008093C1008091C00082608093C0008091D3
:1022A000C10080688093C1008091C10080648093E8
:1022B000C10000E010E00093C5008AE290E0809346
:1022C000C4008091DD019091DE010E940F15909372
:1022D0001204809311048CED90E00E940F159093EE
:1022E000410480934004109213048EE480931404FC
:1022F00088E0809317048BE08093150410921604F5
:102300001093E3010093E2011092E1011F910F91FC
:102310000895A0E1B0E0EFE8F1E10C947A738091C8
:102320000701882309F48CC28091D7019091D801CC
:102330000E941815882361F01092DA011092D901D9
:102340001092DE011092DD011092DC011092DB018F
:102350008091D9019091DA01892B41F08091E204BA
:102360009091E3040E941815882329F48091ED01CF
:10237000882309F460C080910701882309F45BC0B9
:102380008091E90100E211E08430A8F00E94E41E8F
:1023900080E590E09F938F931F930F9381E08F933D
:1023A0008F9388E48F930E94C90C2DB73EB7295FA5
:1023B0003F4F2DBF34C0109244028CE294E09F93B3
:1023C0008F9389ED9EE19F938F93E091FF03F091AE
:1023D0000004099584E190E09F938F931F930F93DE
:1023E00081E090E09F938F9389EE91E09F938F938C
:1023F00082E08F9381E08F9388E48F930E94C90CD1
:102400008091E901982F8F5F8093E9012DB73EB746
:10241000215F3F4F2DBF943010F01092E901809161
:10242000D9019091DA010E940F159093E3048093F3
:10243000E2041092ED018091EE01882351F1809128
:102440000701882331F10E94E41E80E590E09F930C
:102450008F9380E291E09F938F9321E030E03F9350
:102460002F938FE191E09F938F933F932F9383E47A
:1024700092E09F938F9383E08F9381E08F938CE41E
:102480008F930E94C90C1092EE018DB79EB70F96E4
:102490008DBF8091EB018823D1F0809107018823C3
:1024A000B1F08AE090E09F938F9383E194E09F9353
:1024B0008F9381E08F938F9386E58F930E94C90C51
:1024C0001092EB012DB73EB7295F3F4F2DBF809192
:1024D000EF018823D9F0809107018823B9F08BE0C0
:1024E00090E09F938F9385E394E09F938F9381E097
:1024F0008F93809104018F9387E48F930E94C90C7E
:102500001092EF018DB79EB707968DBF8091400462
:10251000909141040E941815882309F461C08091AC
:102520000701882309F45CC08091F2059927880F80
:10253000991F880F991F7C010027F7FC0095102F29
:1025400080913A0390913B03A0913C03B0913D03ED
:10255000BC01CD01A80197010E94537330932E0452
:1025600020932D048091320390913303A091340382
:10257000B0913503BC01CD01A80197010E945373AE
:102580003093300420932F048091D1028093310442
:102590008091D0028093320488E090E09F938F93E3
:1025A0008DE294E09F938F9381E08F9383E08F93EC
:1025B0008BE68F930E94C90C809133042DB73EB7F0
:1025C000295F3F4F2DBF853018F086E0809333049C
:1025D00083E690E00E940F1590934104809340049D
:1025E0008091DD019091DE01892B41F080911104F1
:1025F000909112040E941815882321F48091EC0117
:10260000882329F180910701882309F182E490E071
:102610009F938F9384E895E09F938F9381E08F93AE
:102620008F9384E48F930E94C90C1092EC018DB7B4
:102630009EB707968DBF8091DD019091DE010097D6
:1026400031F00E940F159093120480931104809131
:10265000DB019091DC01892B09F485C080910F0486
:10266000909110040E941815882309F47CC0809171
:102670000701882309F477C08091F2059927880F14
:10268000991F880F991F7C010027F7FC0095102FD8
:1026900080913A0390913B03A0913C03B0913D039C
:1026A000BC01CD01A80197010E945373309302042D
:1026B000209301048091320390913303A09134035D
:1026C000B0913503BC01CD01A80197010E9453735D
:1026D000309304042093030420918B0730918C07DE
:1026E00040918D0750918E07DA01C90103E0880FF0
:1026F000991FAA1FBB1F0A95D1F7820F931FA41F12
:10270000B51F820F931FA41FB51F20919301309115
:1027100094014091950150919601BC01CD010E9418
:10272000537330930604209305048EE090E09F934A
:102730008F9381E094E09F938F9381E08F938F93A9
:1027400083E48F930E94C90C8091DB019091DC019E
:102750000E940F159093100480930F042DB73EB77D
:10276000295F3F4F2DBF809106018F3F71F199275F
:1027700014E0880F991F1A95E1F7845D9D4F40E1A1
:1027800050E0BC01CE0101960E94017180E190E011
:102790009F938F93CE0101969F938F9381E090E05A
:1027A0009F938F9386E091E09F938F9382E08F9326
:1027B00081E08F9381E48F930E94C90C8FEF809307
:1027C00006018DB79EB70B968DBF8091C6058823F5
:1027D000D1F0809107018823B1F081E090E09F93D0
:1027E0008F9386EC95E09F938F9381E08F938F93E7
:1027F00082E48F930E94C90C1092C6052DB73EB794
:10280000295F3F4F2DBF8091EA018823C9F0809155
:1028100007018823A9F084E390E09F938F9383ECD2
:1028200096E09F938F9381E08F938F9380E58F93B2
:102830000E94C90C1092EA018DB79EB707968DBF12
:10284000E6E0C05F0C9496731F920F920FB60F9242
:1028500011242F933F935F936F937F938F939F9355
:10286000AF93BF93EF93FF938091FD01882329F0ED
:102870008091FD0181508093FD018091E2038823C6
:1028800019F081508093E20380910502815080937A
:1028900005028F3FB9F489E08093050280910A0117
:1028A0008F5F817080930A01882319F481E08093FF
:1028B0000202809103029091040201969093040217
:1028C000809303028091FE019091FF01892BC9F052
:1028D0008091FE019091FF0101979093FF018093F9
:1028E000FE018091FE019091FF012091080130913D
:1028F000090182239323892B11F021E009C020E0F4
:1029000007C020E08FEF9FEF9093090180930801AB
:1029100080910201222331F08A3011F45A9A07C0C3
:10292000479A05C08A3011F45A9801C0479880919F
:10293000D403882309F063C08091E30583FF5FC05F
:1029400086B19927FC01E071F07084FF0AC0809184
:10295000000290910102019690930102809300027F
:102960004EC08091000290910102892B09F443C06E
:1029700080910002909101028A569140E0F5809189
:1029800000029091010269E270E00E940A73809156
:10299000000290910102860F971F9093010280938D
:1029A000000280910002909101020B9750F08091FB
:1029B0000002909101020A97909301038093000313
:1029C00004C0F0930103E093000380910003909111
:1029D00001032091FE023091FF02821B930B845E63
:1029E0009D4F68E671E00E941E73845B9040909357
:1029F000FD028093FC021092010210920002FF91EE
:102A0000EF91BF91AF919F918F917F916F915F9166
:102A10003F912F910F900FBE0F901F90189520910E
:102A2000030230910402280F391FC901019608954D
:102A30002091030230910402821B930B892F992766
:102A40008695807490700895CF93DF930E940F1540
:102A5000EC01CE010E9418158823D9F3DF91CF91A4
:102A60000895CF93DF930E940F15EC0109C0809168
:102A70000F01882329F090930F018FEC80937A0047
:102A8000CE010E941815982F882389F3DF91CF91EA
:102A900008959FB7F8945F983E9A469A8091B00047
:102AA0008F708093B0008091B00083608093B000FD
:102AB0008091B1008B738093B1008091B1008B60E5
:102AC0008093B1001092B2008FEF8093B300809199
:102AD000B00080688093B000809170008A7F8093FE
:102AE0007000809170008260809370009FBF089595
:102AF0008AE090E00E940F1590930D0280930C02E3
:102B000082E085BD83EA84BD17BC84EB88BD86E086
:102B100086BD80916E00816080936E0008951F9243
:102B20000F920FB60F9211242F933F934F935F9301
:102B30006F937F938F939F93AF93BF93CF93DF93C5
:102B4000EF93FF938091020190910602843108F087
:102B500011C1992309F066C38091B00086FFECC0D3
:102B60008091B0008F7B8093B00089EA93E09093CE
:102B700008028093070280910B0190910C019C0147
:102B8000220F331F280F391F80919F019927880F2B
:102B9000991F880F991F280F391F37FF02C02D5F1B
:102BA0003F4FC901959587959595879590930C0111
:102BB00080930B019093FB018093FA01809135067D
:102BC0006091030620913A0330913B0340913C030E
:102BD00050913D0380FF2CC0772788279927EA0171
:102BE000D90157FF04C0A158BF4FCF4FDF4FE7E0D7
:102BF000D595C795B795A795EA95D1F79D01AE01F3
:102C00000E94DF729B01AC0197FF04C0215C3F4F23
:102C10004F4F5F4F66E055954795379527956A95D5
:102C2000D1F78091FA019091FB01820F931F2BC085
:102C3000772788279927EA01D90157FF04C0A158AF
:102C4000BF4FCF4FDF4F27E0D595C795B795A795D5
:102C50002A95D1F79D01AE010E94DF729B01AC0164
:102C600097FF04C0215C3F4F4F4F5F4FF6E05595F3
:102C7000479537952795FA95D1F78091FA0190916C
:102C8000FB01821B930B9093FB018093FA018091CF
:102C90000406282F3327220F331F220F331F809162
:102CA000FA019091FB01821793077CF08091050651
:102CB000282F3327220F331F220F331F8091FA0151
:102CC0009091FB012817390724F43093FB012093DE
:102CD000FA0120910702309108028091FA01909147
:102CE000FB01280F391F20503240309308022093F7
:102CF00007028091FA019091FB0197FD039695954B
:102D00008795959587959093FB018093FA0145E00F
:102D10002D3D340718F08CED95E005C02757314064
:102D200030F487E791E09093080280930702809146
:102D300007029091080243C28091B00080648093A2
:102D4000B00080910A06282F33278DED96E0289F4A
:102D5000A001299F500D389F500D1124CA012091C8
:102D6000090230910A02821B930B90930802809310
:102D7000070255C2992309F055C28091B00086FF21
:102D800023C28091B0008F7B8093B000E0910B0252
:102D9000EE23F1F480910A06282F33278DED96E07B
:102DA000289FA001299F500D389F500D1124CA0162
:102DB0002091090230910A02821B930B9093080222
:102DC0008093070210920A0210920902469A27C2C3
:102DD00089EA93E090930802809307028E2F992747
:102DE0008330910509F4A4C1843091053CF481300D
:102DF000910561F0029709F4D2C0AAC1843091050F
:102E000009F499C1059709F4A0C1A2C180910B01F1
:102E100090910C019C01220F331F280F391F8091C4
:102E20009F019927880F991F880F991F280F391F15
:102E300037FF02C02D5F3F4FC90195958795959546
:102E4000879590930C0180930B019093FB018093E5
:102E5000FA01809135066091030620913A03309182
:102E60003B0340913C0350913D0380FF2CC07727EA
:102E700088279927EA01D90157FF04C0A158BF4FFD
:102E8000CF4FDF4F27E0D595C795B795A7952A95E2
:102E9000D1F79D01AE010E94DF729B01AC0197FF4B
:102EA00004C0215C3F4F4F4F5F4FA6E055954795BB
:102EB00037952795AA95D1F78091FA019091FB015A
:102EC000820F931F27C077278827992757FF04C0B1
:102ED00021583F4F4F4F5F4FF7E055954795379536
:102EE0002795FA95D1F70E94DF729B01AC0197FFFD
:102EF00004C0215C3F4F4F4F5F4FE6E0559547952B
:102F000037952795EA95D1F78091FA019091FB01C9
:102F1000821B930B9093FB018093FA01809104062E
:102F2000282F3327220F331F220F331F8091FA01DE
:102F30009091FB01821793077CF080910506282F62
:102F40003327220F331F220F331F8091FA019091F4
:102F5000FB012817390724F43093FB012093FA0171
:102F600080910702909108022091FA013091FB01B3
:102F7000820F931F80509240909308028093070223
:102F80008091FA019091FB0197FD039695958795A5
:102F9000959587959093FB018093FA01ECC0809101
:102FA0000D0190910E019C01220F331F280F391F34
:102FB00080919E019927880F991F880F991F280FCC
:102FC000391F37FF02C02D5F3F4FC9019595879587
:102FD0009595879590930E0180930D019093F9013B
:102FE0008093F8018091350660910706A091320325
:102FF000B0913303C0913403D091350381FF2AC0CF
:103000007727882799279D01AE01D7FF04C0215853
:103010003F4F4F4F5F4FA7E0559547953795279501
:10302000AA95D1F70E94DF729B01AC0197FF04C003
:10303000215C3F4F4F4F5F4FF6E0559547953795D1
:103040002795FA95D1F78091F8019091F901820FB7
:10305000931F29C07727882799279D01AE01D7FFA5
:1030600004C021583F4F4F4F5F4FE7E055954795BC
:1030700037952795EA95D1F70E94DF729B01AC0145
:1030800097FF04C0215C3F4F4F4F5F4F76E055954F
:103090004795379527957A95D1F78091F8019091CA
:1030A000F901821B930B9093F9018093F8018091B1
:1030B0000806282F3327220F331F220F331F80913A
:1030C000F8019091F901821793077CF0809109062D
:1030D000282F3327220F331F220F331F8091F8012F
:1030E0009091F9012817390724F43093F9012093BE
:1030F000F80180910702909108022091F801309127
:10310000F901820F931F80509240909308028093A0
:1031100007028091F8019091F90197FD039695952A
:103120008795959587959093F9018093F80123C031
:103130008091590702C0809131079927880F991F04
:10314000880F991F87559E4F12C080916107F5CF58
:10315000FF27EE0FFF1FED53F94F20813181220F22
:10316000331F8091070290910802820F931F909362
:10317000080280930702809107029091080255E0AF
:103180008D3D950718F08CED95E005C0875791406F
:1031900030F487E791E09093080280930702209132
:1031A0000702309108022C5B3040309308022093D4
:1031B00007028091090290910A02820F931F909357
:1031C0000A02809309022BC08091B0008064809332
:1031D000B0008CEB90E090930802809307028091FE
:1031E000090290910A0284549F4F90930A0280939F
:1031F00009028091FC01882331F08091EE02853B29
:1032000010F0469801C0469A80910B028F5F809320
:103210000B0290910A06981710F410920B0281E0AD
:1032200080930602209107023091080241E02F3777
:10323000340730F08FEF8093B3002F5F30400FC022
:103240002F3F3105C9F0C0F0A9014F5F50404F3703
:10325000510550F480E88093B300205830403093FB
:1032600008022093070212C08FEF8093B30050939F
:103270000802409307020AC0809107028093B300BE
:10328000109208021092070210920602FF91EF912D
:10329000DF91CF91BF91AF919F918F917F916F916E
:1032A0005F914F913F912F910F900FBE0F901F9004
:1032B000189510927C008FEC80937A000895CF933C
:1032C000DF9383E090E00E94342CC82FDD27C531C6
:1032D000D10508F02A97C7BD1092150284E690E048
:1032E0000E943115809113019091140180529340F6
:1032F00010F4C0E0D0E0CA3FD105F8F4C7BD82E3C6
:1033000090E00E94311581E494E09F938F938DE3C8
:1033100091E19F938F93E091FF03F0910004099551
:1033200080911301909114010F900F900F900F90C6
:103330008052934010F02196DECF6C2F83E090E016
:103340000E943C2CC093D3058CE291E00E94311581
:10335000DF91CF910895EF92FF921F93CF93C0E03A
:10336000C0931002C0930F02C0930E0280ED97E04D
:103370000E940F157C011CE8C33019F41B3008F0C3
:1033800019E0C0E080912502909126028C5F934065
:1033900024F48091120181500AC0809125029091FD
:1033A00026028750944034F0809112018F5F809301
:1033B000120101C0C1E080912302909124028C5F30
:1033C000934024F48091110181500AC0809123021E
:1033D000909124028750944034F0809111018F5FC6
:1033E0008093110101C0CF5F809121029091220250
:1033F0008C5F934024F48091100181500AC0809129
:1034000021029091220287509440C4F080911001D3
:103410008F5F8093100113C083E494E09F938F9398
:103420008DE391E19F938F93E091FF03F09100046E
:1034300009950F900F900F900F904DC0CF5F88E0CF
:1034400080934A020E94AD2E809112018A3030F49E
:1034500081E0809310028AE0809312018091120132
:10346000863F30F081E08093100285EF8093120157
:10347000809111018A3030F481E080930F028AE05C
:103480008093110180911101863F30F081E080939B
:103490000F0285EF80931101809110018A3030F482
:1034A00081E080930E028AE08093100180911001E8
:1034B000863F30F081E080930E0285EF809310010B
:1034C00080914A02882339F0C7010E941815882389
:1034D00009F0A2CFF5CF10920F018FEC80937A0004
:1034E00080910F018823E1F31A3020F48AE090E004
:1034F0000E943115115009F03FCF86E490E00E9400
:103500003115CF911F91FF90EF9008951F920F9268
:103510000FB60F921124AF92BF92CF92DF92EF922B
:10352000FF920F931F932F933F934F935F936F934C
:103530007F938F939F93AF93BF93EF93FF9380916C
:103540002E02282F3327442755278F5F80932E0282
:10355000F9012231310508F0FAC3EA5BFF4F0C9400
:10356000A573809178009091790046C08091780091
:10357000909179009AC18091780090917900909310
:10358000300280932F02C5C180914603909147037A
:103590002091780030917900821B930B9093C8059D
:1035A0008093C7058091C7059091C80590933A0212
:1035B00080933902CCC1809178009091790020915C
:1035C000480330914903821B930B9093D20580935B
:1035D000D1058091D1059091D20590933C028093C2
:1035E0003B02B7C38091330290913402209178005E
:1035F00030917900820F931F9093340280933302AD
:1036000081E0A8C38091310290913202209178002C
:1036100030917900820F931F909332028093310290
:1036200084E098C380911D0190911E019C01220F9E
:10363000331F280F391F809178009091790063E043
:1036400070E00E940A73260F371F3695279536952E
:10365000279530931E0120931D0185E07BC3809147
:10366000780090917900AA2797FDA095BA2FBC0108
:10367000CD010E942B727B018C01809140039091BF
:103680004103A0914203B09143039C01AD01C801E5
:10369000B7010E948F71DC01CB01BC01CD010E94FA
:1036A000F871DC01CB0190931C0280931B02809186
:1036B0001B0290911C0202970CF446C080914003BB
:1036C00090914103A0914203B091430320E030E880
:1036D0004BE354E4BC01CD010E94F47188230CF04B
:1036E00088C08091400390914103A0914203B09122
:1036F00043032AE037ED43EA5CE3BC01CD010E94BD
:103700009071DC01CB018093400390934103A0931F
:103710004203B09343038091BE029091BF02845F45
:10372000914008F066C08091400390914103A091C0
:103730004203B09143032DEC3CEC4CEC5DE3BC0147
:10374000CD010E9490714BC080911B0290911C0290
:103750008F5F9F4F0CF04DC08091400390914103CB
:10376000A0914203B091430320E030E849E054E4E3
:10377000BC01CD010E94DB721816DCF5809140037C
:1037800090914103A0914203B09143032AE037EDA9
:1037900043EA5CE3BC01CD010E948F71DC01CB01E7
:1037A0008093400390934103A0934203B09343035B
:1037B0008091BE029091BF02845F9140D0F48091CD
:1037C000400390914103A0914203B09143032DEC3B
:1037D0003CEC4CEC5DE3BC01CD010E948F71DC013F
:1037E000CB018093400390934103A0934203B09395
:1037F000430381E080931A028091780090917900D0
:103800009093CA058093C90580911B0290911C0278
:103810009C01442737FD4095542F809102039091DD
:103820000303A0910403B0910503820F931FA41F0B
:10383000B51F8093020390930303A0930403B093F6
:10384000050320910203309103034091040350913A
:10385000050357FF04C021503C4F4F4F5F4F0AE014
:1038600055954795379527950A95D1F7809102038D
:1038700090910303A0910403B0910503821B930B65
:10388000A40BB50B8093020390930303A09304034E
:10389000B09305032EC180913102909132022091A4
:1038A000780030917900820F931F909332028093B9
:1038B000310210922D0250C2809102018A3071F4BF
:1038C000809178009091790020912F023091300200
:1038D000820F931F01969695879517C040912F02EE
:1038E00050913002843159F4209178003091790060
:1038F000240F351F8FEF97E0821B930B06C080913A
:10390000780090917900840F951F90932202809304
:10391000210286E01FC280914603909147032091C7
:10392000780030917900821B930B9093C8058093A7
:10393000C7058091C7059091C80520913902309143
:103940003A02820F931F9093200280931F0287E018
:1039500001C28091780090917900209148033091C4
:103960004903821B930B9093D2058093D1058091DC
:10397000D1059091D20520913B0230913C02820FFB
:10398000931F90931E0280931D02E3C12091330286
:10399000309134028091780090917900280F391F7E
:1039A0003093340220933302809102018A3019F45B
:1039B000220F331F04C0220F331F220F331F3093F7
:1039C0003402209333022091330230913402C90132
:1039D00037FD0796A3E095958795AA95E1F7909313
:1039E0002602809325028091350290913602820F43
:1039F000931F97FD01969595879590933602809336
:103A000035022091520330915303821B930B909304
:103A10001C0180931B0120912B0230912C0280917C
:103A20001B0190911C01280F391F37FF02C02F5F27
:103A30003F4F3595279530932C0220932B02E0CDF4
:103A4000209131023091320280917800909179007A
:103A5000280F391F309332022093310280910201E6
:103A60008A3019F4220F331F04C0220F331F220F94
:103A7000331F309332022093310220913102309172
:103A80003202C90137FD079663E0959587956A95DF
:103A9000E1F7909324028093230280913702909162
:103AA0003802820F931F97FD019695958795909305
:103AB0003802809337022091500330915103821BCA
:103AC000930B90931A018093190120912902309150
:103AD0002A028091190190911A01280F391F37FF8E
:103AE00002C02F5F3F4F3595279530932A022093D0
:103AF000290283E02FC110922E0281E080930F01F2
:103B0000809111029091120201969093120280937B
:103B10001102809178009091790090931401809324
:103B200013018091130190911401AA27BB27A09043
:103B30003D02B0903E02C0903F02D0904002A80EDD
:103B4000B91ECA1EDB1EA0923D02B0923E02C09278
:103B50003F02D0924002809141028F5F80934102E8
:103B6000823108F4F6C08091150190911601A09160
:103B70001701B09118017C018D0123E0EE0CFF1CB0
:103B8000001F111F2A95D1F7E81AF90A0A0B1B0B1F
:103B9000EA0CFB1C0C1D1D1D80911502992787FD49
:103BA0009095A92FB92FBC01CD0126EC34E240E05D
:103BB00050E00E94DF72DC01CB01E81AF90A0A0B1F
:103BC0001B0BD801C7010496A11DB11DB7FF05C08D
:103BD000D801C7010B96A11DB11D13E0B595A7959E
:103BE000979587951A95D1F78093150190931601B3
:103BF000A0931701B09318018091CB059091CC054B
:103C00007C010027F7FC0095102F80911501909101
:103C10001601A0911701B0911801E81AF90A0A0BD0
:103C20001B0BE092E002F092E1020093E20210939B
:103C3000E302209116023091170240911802509130
:103C4000190257FF04C0215F3F4F4F4F5F4FF4E011
:103C50005595479537952795FA95D1F78091160296
:103C600090911702A0911802B0911902821B930B38
:103C7000A40BB50B8093160290931702A093180221
:103C8000B09319028091160290911702A091180228
:103C9000B09119028E0D9F1DA01FB11F80931602B7
:103CA00090931702A0931802B09319028091130207
:103CB00090911402AC01E4E0440F551FEA95E1F73E
:103CC000481B590B8091160290911702A09118027F
:103CD000B0911902B7FF03C00F96A11DB11D74E08A
:103CE000B595A795979587957A95D1F72091E0029C
:103CF0003091E102281B390B63E0220F331F6A95D4
:103D0000E1F7240F351F37FF02C0215F3F4F44E02A
:103D1000359527954A95E1F73093140220931302C5
:103D2000D601C501D7FE03C00196A11DB11DB595F1
:103D3000A7959795879580933D0290933E02A09317
:103D40003F02B093400289E08093410202C010928A
:103D50002E0282E080932D0280912D0280937C00C0
:103D600080912E02882319F08FEC80937A00FF91C6
:103D7000EF91BF91AF919F918F917F916F915F91E3
:103D80004F913F912F911F910F91FF90EF90DF90F6
:103D9000CF90BF90AF900F900FBE0F901F901895CF
:103DA00090E2E0E2F1E08FE49193815087FFFCCF55
:103DB000089590914402E0E2F1E0E90FF11D808363
:103DC0009F5F909344020895EF92FF920F931F9389
:103DD000CF93DF932091420220FF0AC080914302DB
:103DE000882311F0815002C080911F01809343020B
:103DF00021FF0CC09091430280911F01981719F484
:103E00001092430203C09F5F90934302822F992731
:103E100080FF04C081FF02C0109243020E94D01EA6
:103E200080914302282F3327C9EDEC2ECEE1FC2EE2
:103E3000C091FF03D09100048A3098F481E180930F
:103E400044023F932F938AE794E09F938F93FF92CE
:103E5000EF92FE0109952DB73EB72A5F3F4F2DBF68
:103E600011C080E1809344023F932F938FE794E049
:103E70009F938F93FF92EF92FE0109958DB79EB7A6
:103E800006968DBF20914302822F9927AA27BB2730
:103E9000FC01419710F00C94E728E85AFF4FB9ED68
:103EA000EB2EBEE1FB2EC091FF03D09100040C94D9
:103EB000A5731092440284E894E09F938F93FF923D
:103EC000EF92FE01099584E1809344020F900F90D8
:103ED0000F900F9089E690E09F938F938EE490E08F
:103EE0009F938F931F921F92809102016AE00E941C
:103EF000FE72892F99279F938F93809102010E94D0
:103F0000FE7299279F938F9384E994E09F938F93F8
:103F1000FF92EF92E091FF03F0910004099588E28F
:103F2000809344022DB73EB7225F3F4F2DBF85E4FB
:103F300096E09F938F930E949F2D99279F938F9335
:103F400089EA94E09F938F93FF92EF92E091FF03B1
:103F5000F091000409958091B9019091BA012DB7B3
:103F60003EB7285F3F4F2DBF069730F48CE3809318
:103F7000440287EB94E0CDC090914702992311F45D
:103F80000C94F0288CE380934402892F99279F9307
:103F90008F9384EC94E09F938F9389ED9EE19F93A0
:103FA0008F9377C08091E305A9EDEA2EAEE1FA2E5A
:103FB000C091FF03D091000480FF74C010924402AE
:103FC0008091E0029091E102A091E202B091E302BF
:103FD000BC01CD0125E030E040E050E00E94537389
:103FE0003F932F9389ED94E09F938F93FF92EF92ED
:103FF000FE01099584E1809344022DB73EB72A5F04
:104000003F4F2DBF8091DC029091DD02A091DE0236
:10401000B091DF02BC01CD0125E030E040E050E08E
:104020000E9453733F932F9386EE94E09F938F9358
:10403000FF92EF92E091FF03F0910004099588E26E
:10404000809344028DB79EB706968DBF8091130171
:10405000909114019F938F9383EF94E09F938F939C
:10406000FF92EF92E091FF03F091000409958CE339
:10407000809344022DB73EB72A5F3F4F2DBF87B5CF
:1040800099279F938F9380E095E09F938F93FF9262
:10409000EF92E091FF03F091000409958DB79EB770
:1040A000069639C7109244028DE095E09F938F9356
:1040B000FF92EF92FE01099584E1809344020F90F4
:1040C0000F900F900F908CE195E09F938F93FF924C
:1040D000EF92E091FF03F0910004099588E280934C
:1040E00044020F900F900F900F9085E295E09F9300
:1040F0008F93FF92EF92E091FF03F09100040995F6
:104100008CE3809344020F900F900F900F9084E304
:1041100095E09F938F93FF92EF92EFC71092440226
:104120008DE395E09F938F9309ED1EE1FF92EF924F
:10413000FE01099584E1809344020F900F900F9047
:104140000F9080913A0390913B03A0913C03B09172
:104150003D03B7FF04C081509C4FAF4FBF4FFAE003
:10416000B595A79597958795FA95D1F7BF93AF9396
:104170009F938F938AE495E09F938F931F930F9360
:10418000E091FF03F0910004099588E280934402D6
:104190002DB73EB7285F3F4F2DBF809132039091DE
:1041A0003303A0913403B0913503B7FF04C08150AD
:1041B0009C4FAF4FBF4FEAE0B595A7959795879570
:1041C000EA95D1F7BF93AF939F938F9389E595E0DD
:1041D0009F938F931F930F93E091FF03F09100043F
:1041E00009958CE3809344028DB79EB708968DBFE6
:1041F00080910003909101039F938F9388E695E04F
:104200009F938F931F930F93EEC31092440280915C
:10421000C7069091C8069F938F938091C506909191
:10422000C6069F938F9387E795E09F938F93FF92A6
:10423000EF92FE01099584E1809344028DB79EB709
:1042400008968DBF8091CB069091CC069F938F935B
:104250008091C9069091CA069F938F9387E895E055
:104260009F938F93FF92EF92E091FF03F0910004F0
:10427000099588E2809344022DB73EB7285F3F4FEF
:104280002DBF8091CF069091D0069F938F93809100
:10429000CD069091CE069F938F9387E995E09F93EB
:1042A0008F93FF92EF92E091FF03F0910004099544
:1042B0008CE3809344028DB79EB708968DBF8091A2
:1042C000D3069091D4069F938F938091D1069091BD
:1042D000D2069F938F9387EA95E076C510924402A9
:1042E0008091D805E82FFF27EE0FFF1FED53F94F00
:1042F000808191819F938F938091D705E82FFF272D
:10430000EE0FFF1FED53F94F808191819F938F93A3
:1043100087EB95E09F938F93FF92EF92FE010995B3
:1043200084E1809344028DB79EB708968DBF80913B
:10433000DA05E82FFF27EE0FFF1FED53F94F8081BD
:1043400091819F938F938091D905E82FFF27EE0FDE
:10435000FF1FED53F94F8081918188589F4F9F93A4
:104360008F9387EC95E09F938F93FF92EF92E0916C
:10437000FF03F0910004099588E2809344022DB771
:104380003EB7285F3F4F2DBF8091DC05E82FFF2708
:10439000EE0FFF1FED53F94F8081918182599F4F9E
:1043A0009F938F938091DB05E82FFF27EE0FFF1F70
:1043B000ED53F94F8081918182599F4F9F938F9345
:1043C00087ED95E09F938F93FF92EF92E091FF032B
:1043D000F091000409958CE3809344028DB79EB759
:1043E00008968DBF8091DE05E82FFF27EE0FFF1F97
:1043F000ED53F94F8081918182599F4F9F938F9305
:104400008091DD05E82FFF27EE0FFF1FED53F94FD9
:104410008081918182599F4F9F938F9387EE95E082
:10442000D3C41092440287EF95E09F938F9309EDD8
:104430001EE1FF92EF92FE010995809102010F901B
:104440000F900F900F908A3009F0A1C084E1809303
:10445000440280915203909153039C0197FF02C044
:10446000295F3F4F287F821B930B9F938F938091EF
:1044700052039091530397FD079673E095958795A6
:104480007A95E1F79F938F932091520330915303D4
:1044900037FF02C0295F3F4F63E0359527956A9546
:1044A000E1F78091250290912602821B930B9F9346
:1044B0008F9385E096E09F938F931F930F93E091E6
:1044C000FF03F0910004099588E2809344028DB7C0
:1044D0009EB70A968DBF80915003909151039C0125
:1044E00097FF02C0295F3F4F287F821B930B9F934A
:1044F0008F93809150039091510397FD079653E05D
:10450000959587955A95E1F79F938F932091500346
:104510003091510337FF02C0295F3F4F43E035958B
:1045200027954A95E1F78091230290912402821BFE
:10453000930B9F938F9386E196E09F938F931F93A6
:104540000F93E091FF03F091000409958CE38093B1
:1045500044022DB73EB7265F3F4F2DBF80914E03DB
:1045600090914F039F938F9380914E0390914F03AF
:104570002091210230912202821B930B9F938F93F3
:1045800087E296E09F938F931F930F93B6C38B3070
:1045900019F0843109F0ADC084E180934402809128
:1045A0005203909153039C0197FF02C0215F3F4F3C
:1045B000207F821B930B97FD0196959587959F937E
:1045C0008F93809152039091530397FD0F9624E0AF
:1045D000959587952A95E1F79F938F9320915203A4
:1045E0003091530337FF02C0295F3F4F83E0359579
:1045F00027958A95E1F78091250290912602821BEA
:10460000930B9F938F9385E396E09F938F931F93D4
:104610000F93E091FF03F0910004099588E28093E5
:1046200044022DB73EB7265F3F4F2DBF8091500308
:10463000909151039C0197FF02C0215F3F4F207F63
:10464000821B930B97FD0196959587959F938F936A
:10465000809150039091510397FD0F96B4E095958A
:104660008795BA95E1F79F938F93209150033091EE
:10467000510337FF02C0295F3F4FA3E035952795CF
:10468000AA95E1F78091230290912402821B930B5B
:104690009F938F9387E496E09F938F931F930F933D
:1046A000E091FF03F091000409958CE380934402AC
:1046B0008DB79EB70A968DBF80914E0390914F03A0
:1046C00097FD0196959587959F938F9380914E03C3
:1046D00090914F032091210230912202821B930B73
:1046E0009F938F9389E596E09F938F931F930F93EA
:1046F0006FC38D3009F074C584E1809344028091CA
:10470000120199279F938F938091520390915303A5
:1047100097FD0F96E4E095958795EA95E1F79F93CD
:104720008F93209152033091530337FF02C0295FCA
:104730003F4F73E0359527957A95E1F780912502F3
:1047400090912602821B930B9F938F9388E696E0AD
:104750009F938F931F930F93E091FF03F0910004B9
:10476000099588E2809344028DB79EB70A968DBF63
:104770008091110199279F938F938091500390917D
:10478000510397FD0F9664E0959587956A95E1F73B
:104790009F938F93209150033091510337FF02C0B4
:1047A000295F3F4F53E0359527955A95E1F7809162
:1047B000230290912402821B930B9F938F938CE78B
:1047C00096E09F938F931F930F93E091FF03F091D7
:1047D000000409958CE3809344022DB73EB7265F11
:1047E0003F4F2DBF8091100199279F938F93809108
:1047F0004E0390914F0397FD0196959587959F9352
:104800008F9380914E0390914F032091210230911C
:104810002202821B930B9F938F9380E996E09F93D4
:104820008F931F930F93E091FF03F091000409957C
:104830008DB79EB70A966FC31092440284EA96E041
:104840009F938F93FF92EF92FE01099584E18093ED
:1048500044020F900F900F900F9080914803909119
:1048600049039F938F9380911D0290911E029F9305
:104870008F9381EB96E09F938F93FF92EF92E0915D
:10488000FF03F0910004099588E2809344022DB75C
:104890003EB7285F3F4F2DBF80914603909147035D
:1048A0009F938F9380911F02909120029F938F93EB
:1048B00080EC96E09F938F93FF92EF92E091FF033D
:1048C000F091000409958CE3809344028DB79EB764
:1048D00008968DBF8091400390914103A0914203BF
:1048E000B0914303BC01CD010E94F871DC01CB0102
:1048F0009F938F9380914E0790914F079F938F9333
:104900008FEC96E061C21092440280911D0190915B
:104910001E016AE070E00E941E739F938F93809146
:104920001D0190911E016AE070E00E941E737F934A
:104930006F938EED96E09F938F93FF92EF92FE011F
:10494000099584E1809344028DB79EB708968DBF88
:1049500080910108909102086AE070E00E940A7359
:104960009F938F9380910108909102086AE070E014
:104970000E940A737F936F9382EF96E09F938F93C9
:10498000FF92EF92E091FF03F0910004099588E215
:10499000809344022DB73EB7285F3F4F2DBF8091D3
:1049A0000308909104089F938F9386E097E09F936C
:1049B0008F93FF92EF92E091FF03F091000409952D
:1049C0008CE3809344028DB79EB706968DBF80918D
:1049D0000508909106089F938F9386E197E09F9337
:1049E0008F93FF92EF92E091FF03F09100040995FD
:1049F0002DB73EB72A5F3F4FF4C11092440288E2C0
:104A000097E09F938F93FF92EF92FE01099584E1C7
:104A1000809344020F900F900F900F908091C306E7
:104A20009091C4069F938F9381E397E09F938F9318
:104A3000FF92EF92E091FF03F0910004099588E264
:104A4000809344028DB79EB706968DBF8091EE028B
:104A500099279F938F9381E497E09F938F93FF9281
:104A6000EF92E091FF03F091000409958CE38093AD
:104A700044022DB73EB72A5F3F4F2DBF8091C2063B
:104A8000992701979F938F9381E597E0FECA109233
:104A9000440281E697E09F938F93FF92EF92FE018D
:104AA000099584E1809344020F900F900F900F902E
:104AB0008091FC029091FD029F938F9389E697E08D
:104AC0009F938F93FF92EF92E091FF03F091000488
:104AD000099588E2809344022DB73EB72A5F3F4F85
:104AE0002DBF80910003909101039F938F9387E7DF
:104AF00097E09F938F93FF92EF92E091FF03F091E5
:104B0000000409958CE3809344028DB79EB7069606
:104B10008DBF8091FE029091FF029F938F9385E855
:104B200097E05DCF109244028091EF0299279F9306
:104B30008F9383E997E09F938F93FF92EF92FE010B
:104B4000099584E1809344028DB79EB706968DBF88
:104B50008091F00299279F938F938FE997E09F931D
:104B60008F93FF92EF92E091FF03F091000409957B
:104B700088E2809344022DB73EB72A5F3F4F2DBF96
:104B80008091F10299279F938F938BEA97E09F93EF
:104B90008F93FF92EF92E091FF03F091000409954B
:104BA0008CE3809344028DB79EB706968DBF8091AB
:104BB000F20299279F938F9387EB97E010CF109283
:104BC00044028091F30299279F938F9383EC97E09F
:104BD0009F938F93FF92EF92FE01099584E180935A
:104BE00044028DB79EB706968DBF8091F402992737
:104BF0009F938F938FEC97E09F938F93FF92EF9209
:104C0000E091FF03F0910004099588E2809344024B
:104C10002DB73EB72A5F3F4F2DBF8091F5029927F0
:104C20009F938F938BED97E09F938F93FF92EF92DB
:104C3000E091FF03F091000409958CE38093440216
:104C40008DB79EB706968DBF8091F60299279F93E8
:104C50008F9387EE97E0C3CE1092440283EF97E0E4
:104C60009F938F93FF92EF92FE01099584E18093C9
:104C700044020F900F900F900F9080919F01992701
:104C80009F938F938BEF97E09F938F93FF92EF9279
:104C9000E091FF03F0910004099588E280934402BB
:104CA0008DB79EB706968DBF8091FA019091FB015A
:104CB0009F938F9389E098E09F938F93FF92EF9259
:104CC000E091FF03F091000409958CE38093440286
:104CD0002DB73EB72A5F3F4F2DBF8091050699271C
:104CE0009F938F938091040699279F938F9387E1D9
:104CF00098E09F938F93FF92EF92E091FF03F091E2
:104D0000000409958DB79EB7089605C1109244021C
:104D100085E298E09F938F93FF92EF92FE010995B1
:104D200084E1809344020F900F900F900F90809138
:104D30003904992787FD90959F938F93809138042C
:104D4000992787FD90959F938F9385E398E09F9394
:104D50008F93FF92EF92E091FF03F0910004099589
:104D600088E2809344022DB73EB7285F3F4F2DBFA6
:104D700080913A04992787FD90959F938F93809116
:104D80003B0499279F938F9385E498E09F938F939B
:104D9000FF92EF92E091FF03F091000409958CE3FC
:104DA000809344028DB79EB708968DBF80913F04D3
:104DB00099279F938F9380913C04992787FD909525
:104DC0009F938F9385E598E09F938F93FF92EF9247
:104DD000E091FF03F091000409952DB73EB7285FDD
:104DE0003F4F2DBFFDC11092440285E698E09F938E
:104DF0008F93FF92EF92FE01099584E18093440224
:104E00000F900F900F900F9080919F0699278F77AA
:104E100090709F938F9380919B0699278F779070C6
:104E20009F938F938091970699278F7790709F9388
:104E30008F938091930699278F7790709F938F938C
:104E400085E798E09F938F93FF92EF92E091FF03A5
:104E5000F0910004099588E2809344028DB79EB7D3
:104E60000C968DBF8091AF0699278F7790709F9396
:104E70008F938091AB0699278F7790709F938F9334
:104E80008091A70699278F7790709F938F93809139
:104E9000A30699278F7790709F938F9386E898E069
:104EA0009F938F93FF92EF92E091FF03F0910004A4
:104EB00009958CE3809344022DB73EB7245F3F4FA2
:104EC0002DBF8091BF0699278F7790709F938F9306
:104ED0008091BB0699278F7790709F938F938091D5
:104EE000B70699278F7790709F938F938091B30621
:104EF00099278F7790709F938F9387E998E09F937E
:104F00008F93FF92EF92E091FF03F09100040995D7
:104F10008DB79EB70C968DBF63C11092440288EA8C
:104F200098E09F938F9309ED1EE1FF92EF92FE01AF
:104F3000099584E1809344020F900F900F900F9099
:104F400080919F06881F8827881F97E0899FC0014E
:104F500011248D969F938F9380919B06881F88279D
:104F6000881F96E0899FC00111248D969F938F938F
:104F700080919706881F8827881F95E0899FC00128
:104F800011248D969F938F9380919306881F882775
:104F9000881F9927880F991F880F991F8D969F93B7
:104FA0008F9387EB98E09F938F93FF92EF92E0911E
:104FB000FF03F0910004099588E2809344022DB725
:104FC0003EB7245F3F4F2DBF8091AF06881F8827D3
:104FD000881F9BE0899FC00111248D969F938F931A
:104FE0008091AB06881F8827881F9AE0899FC0019F
:104FF00011248D969F938F938091A706881F8827F1
:10500000881F99E0899FC00111248D969F938F93EB
:105010008091A306881F8827881F992723E0880F7F
:10502000991F2A95E1F78D969F938F938BEC98E0CB
:105030009F938F93FF92EF92E091FF03F091000412
:1050400009958CE3809344028DB79EB70C968DBF73
:105050008091B306881F8827881F9CE0899FC00124
:1050600011248D969F938F938FED98E09F938F934C
:10507000FF92EF92E091FF03F09100040995809177
:10508000B7062DB73EB72A5F3F4F2DBF87FF12C02F
:1050900080E48093440280EF98E09F938F93FF9287
:1050A000EF92E091FF03F091000409950F900F90AB
:1050B0000F900F908091BB0687FF12C084E480930D
:1050C000440283EF98E09F938F931F930F93E09197
:1050D000FF03F091000409950F900F900F900F902F
:1050E0008091BF0687FF7CC088E48093440286EFEE
:1050F00098E09F938F931F930F93E091FF03F0919C
:10510000000409950F900F900F900F9069C01092B6
:10511000440289EF98E09F938F93FF92EF92FE01F4
:10512000099584E1809344020F900F900F900F90A7
:105130008091D2019091D3019F938F9387E099E062
:105140009F938F93FF92EF92E091FF03F091000401
:10515000099588E2809344028DB79EB706968DBF6D
:105160008091D4019091D5019F938F9384E199E030
:105170009F938F93FF92EF92E091FF03F0910004D1
:10518000099589E4809344022DB73EB72A5F3F4FCB
:105190002DBF81E299E09F938F93FF92EF92E09170
:1051A000FF03F09100040995809142020F900F9047
:1051B0000F900F9083FF14C01092D5011092D4016C
:1051C00060E070E08EE090E00E944D2C09C080917C
:1051D0001F01281719F4215020931F011092430238
:1051E00010924202E6E0CDB7DEB70C949673F999BF
:1051F000FECF92BD81BDF89A80B599270895F9999F
:10520000FECF1FBA92BD81BD60BD0FB6F894FA9A69
:10521000F99A0FBE08954AEA20E030E026173707D2
:1052200040F4FC018191480F2F5F3F4F261737074D
:10523000C8F3842F99270895EAEA40E050E0461722
:10524000570778F49C01F999FECF32BD21BDF89A39
:1052500080B5E80F4F5F5F4F2F5F3F4F46175707EF
:1052600090F38E2F9927089581E08093D90582E0ED
:105270008093D80583E08093D70584E08093DA0596
:1052800085E08093DB0586E08093DC0587E08093F2
:10529000DD0588E08093DE0589E08093DF058AE004
:1052A0008093E0058BE08093E1058CE08093E2053C
:1052B00008951F93CF93DF9382E58093D605809165
:1052C0000201843150F085E08093F60510921706B4
:1052D0008BE18093F2058EE40AC083E08093F605AB
:1052E00080E2809317068EE18093F20585E5809336
:1052F0001406809315068AE68093E30561E06093C7
:1053000036065EE15093E4058FEF8093E6058AE070
:105310008093E7055093E5055093E90585E0809378
:10532000EA0580E48093EB051092EC0584E180931C
:10533000E8058EE08093ED05E0E1E093EE051CE0EA
:105340001093EF05F8E0F093F00586EE8093F105F9
:1053500080E88093F30540E54093F40586E9809367
:10536000F5054093F7058093F80581E28093F905F0
:1053700083E28093FA055093FB0580E28093FD055C
:105380001092FE051092FF05109200061092010681
:105390001092190610921A0610921B0610921C0603
:1053A00024E62093020638E2309303066093350624
:1053B0001092040697EF9093050676E070930A0624
:1053C0008DE780930B0680930C0680930D06209347
:1053D000060630930706109208069093090682E3AA
:1053E00080930E069AE590930F0680931006109214
:1053F0003406909311064093120660931306E093CF
:105400001606209318068FE580931D0683EF809380
:105410001F068AEA80932106809322068FE08093FC
:105420001E06809320068EEF809323062093240689
:105430009093250690932606909327068BE48093FD
:1054400028068093290680932A0610922B067093D3
:105450002C06F0932D0690932E0650932F06209342
:1054600030062093310684E0809332066093FC0579
:10547000A7E3B6E0E0E7F1E0ED01019009921A95AB
:10548000E1F76DE670E0CD01815690400E940B2956
:1054900080934306DF91CF911F910895CF93DF93BF
:1054A00082E58093D60580910201843150F085E039
:1054B0008093F605109217068BE18093F2058EE437
:1054C0000AC083E08093F60580E2809317068EE1A0
:1054D0008093F20585E580931406809315068AE68D
:1054E0008093E305E1E0E09336065EE15093E40546
:1054F0008FEF8093E6059AE09093E7055093E505DA
:105500005093E90585E08093EA0580E48093EB05FC
:105510001092EC058FE08093E8059093ED0580E113
:105520008093EE0566E06093EF05F8E0F093F005F8
:1055300086EE8093F10580E88093F3052AE52093B9
:10554000F40588E78093F5052093F7058093F80527
:1055500081E28093F90583E28093FA055093FB057D
:1055600070E27093FD051092FE051092FF051092F7
:105570000006109201061092190610921A06109257
:105580001B0610921C0644E64093020638E2309354
:105590000306E09335061092040697EF90930506F4
:1055A00060930A068DE780930B0680930C06809328
:1055B0000D06409306063093070610920806909356
:1055C000090682E380930E0620930F06809310064F
:1055D000109234062093110680E5809312068CE326
:1055E00080931306709316069BE4909318068FE53C
:1055F00080931D0683EF80931F068AEA809321061D
:105600008093220684E180931E06809320068EEF0D
:105610008093230640932406209325062093260694
:1056200020932706909328069093290690932A06A4
:1056300010922B0660932C06F0932D0620932E06D5
:1056400050932F06409330064093310684E08093B8
:105650003206E093FC05A7E3B6E08CE0E7E7F1E073
:10566000ED01019009928A95E1F76DE670E0CD01B8
:10567000815690400E940B2980934306DF91CF9181
:105680000895CF93DF9382E58093D6058091020140
:10569000843150F085E08093F605109217068BE177
:1056A0008093F2058EE40AC083E08093F60580E2E1
:1056B000809317068EE18093F20585E580931406AA
:1056C000809315068AE68093E30571E070933606B1
:1056D0004EE14093E4058FEF8093E6058AE08093E6
:1056E000E7054093E5054093E90585E08093EA05E9
:1056F00080E48093EB051092EC058FE08093E80541
:1057000068E06093ED0590E19093EE0556E05093CC
:10571000EF056093F00586EE8093F10580E88093B5
:10572000F30534E63093F40588E78093F50530936C
:10573000F7058093F80581E28093F90583E2809371
:10574000FA0584E18093FB059093FD051092FE0518
:105750001092FF0510920006109201061092190691
:1057600010921A0610921B0610921C063093020625
:1057700028E220930306709335061092040697EFF3
:105780009093050650930A068DE780930B0680934D
:105790000C0680930D0630930606209307061092A0
:1057A00008069093090692E390930E062AE520934B
:1057B0000F0690931006109234062093110680E590
:1057C0008093120686E48093130680E28093160687
:1057D000909318068FE580931D0683EF80931F0634
:1057E0008AEA809321068093220640931E06409306
:1057F00020068EEF809323063093240620932506FF
:1058000020932606209327068BE480932806809316
:10581000290680932A0610922B0650932C0660933B
:105820002D0620932E0640932F063093300630939A
:10583000310684E0809332067093FC05A7E3B6E05E
:105840008CE0EFE7F1E0ED01019009928A95E1F734
:105850006DE670E0CD01815690400E940B29809347
:105860004306DF91CF910895F999FECF92BD81BD96
:10587000F89A80B599270895F999FECF1FBA92BD7D
:1058800081BD60BD0FB6F894FA9AF99A0FBE0895DB
:1058900067EF78E20E943C7108954FEF58E20E9452
:1058A00076710895EF92FF920F931F93CF93C82FB5
:1058B0008150853008F0C3E08EE6C89F8001112436
:1058C00086EFE82E8FEFF82EE00EF11E6DE670E009
:1058D000C7010E941C29682F98012D593F4F8FB393
:1058E0009927AC014270507081FDF9CF32BD21BDC6
:1058F000F89A80B5861711F0CA0121C08FB3992795
:105900009C012270307081FDF9CFF2BCE1BCF89AA5
:1059100080B5823511F0C90112C08EE6C89FC00162
:1059200011240A9727EF38E24EE650E0BC0186EDDD
:1059300095E00E9417710E94AA6181E090E0CF91EA
:105940001F910F91FF90EF900895282F863010F04F
:1059500025E003C0882309F421E0F999FECF1FBA9E
:1059600082E090E092BD81BD20BD0FB6F894FA9A16
:10597000F99A0FBE0895CF93C82F8091D60582352E
:1059800009F042C0C63010F0C5E003C0CC2309F4D2
:105990003BC06DE670E086ED95E00E940B29809398
:1059A00043068EE6C89FC00111242FEF38E24EE671
:1059B00050E066ED75E00A970E9454712FEF38E2CF
:1059C0004CE050E067ED75E080E590E00E94547196
:1059D0006CE070E087ED95E00E940B29282FF99983
:1059E000FECF1FBA8CE590E092BD81BD20BD0FB601
:1059F000F894FA9AF99A0FBE8C2F0E94A52C0E9457
:105A0000AA6181E090E002C080E090E0CF9108952B
:105A10006DE470E088EE93E00E941C29482F8FB35C
:105A200099279C012270307081FDF9CF85E394E0C5
:105A300092BD81BDF89A80B5841779F48FB3992708
:105A40009C012270307081FDF9CF88EE93E092BD09
:105A500081BDF89A80B5813011F0C901089527EF12
:105A600038E24EE450E068EE73E084E496E00E9491
:105A7000177181E090E00895809144068130A9F487
:105A80006DE470E084E496E00E940B298093910617
:105A90002FEF38E24EE450E064E476E088EE93E0E5
:105AA0000E94547181E090E0089580E090E00895B4
:105AB000CF93DF9381E080934406E4E4F6E08FE047
:105AC000158616861786108A8150349687FFF8CF80
:105AD00080E480935106809352061092530680937F
:105AE00054068093550690EC9093560610925706F4
:105AF000809358068093590610925A0690935B063D
:105B000090935C0680935D0610925E0680935F061C
:105B100090936006A5E4B6E087E0E9E8F1E0ED01E6
:105B2000019009928A95E1F76DE470E0CD0101974B
:105B30000E940B2980939106DF91CF910895F999E6
:105B4000FECF82E090E092BD81BDF89A80B5282F0B
:105B5000863078F023E0322FF999FECF1FBA82E029
:105B600090E092BD81BD30BD0FB6F894FA9AF99AD3
:105B70000FBE822F99270895DF92EF92FF920F9325
:105B80001F93CF93FF24DF2CEF2C81E090E00E9445
:105B9000342C823539F031E0E32E62E581E090E08B
:105BA0000E943C2C6CE070E080E590E00E941C2993
:105BB000C82FF999FECF8CE590E092BD81BDF89A8F
:105BC00080B58C1711F421E0D22EC1E001E010E085
:105BD000EE2029F48C2F0E94522C8823E9F591E0C5
:105BE000F92E1F930F9389E299E09F938F938DE392
:105BF00091E19F938F93E091FF03F0910004099549
:105C00008DB79EB706968DBF0230110589F003301F
:105C1000110524F40130110529F00AC003301105E3
:105C200021F006C00E94592905C00E94412B02C0E4
:105C30000E944E2ADD2059F027EF38E24CE050E078
:105C400060E570E087ED95E00E94177102C00E9448
:105C500034298C2F0E94BB2CCF5F0F5F1F4FC630A3
:105C600008F4B6CFFF2019F083E00E94A52C0E9413
:105C70009F2DC82F0E94522C8C2F99279F938F9372
:105C80008FE499E09F938F930DE311E11F930F939E
:105C9000E091FF03F091000409958DB79EB7069639
:105CA0008DBFEE2021F40E94082D882399F488E608
:105CB00099E09F938F931F930F93E091FF03F091CF
:105CC000000409950E94582D0E943C2D0F900F90C2
:105CD0000F900F901092E40290E0E1E5F6E0CFE043
:105CE0008081349618160CF49F5FC150C7FFF8CF1F
:105CF0009093E402892F99279F938F9385E496E0F0
:105D00009F938F9389E899E09F938F931F930F93AD
:105D1000E091FF03F091000409958DB79EB70896B6
:105D20008DBF8AEA99E09F938F931F930F93E09121
:105D3000FF03F091000409950F900F900F900F90C2
:105D4000CF911F910F91FF90EF90DF9008951092E7
:105D5000B9008AE28093B800089585EA8093BC0078
:105D6000089584E98093BC0008951092B90080934F
:105D7000BB0085E88093BC0008950E94B12E10926C
:105D80004A028091BB001092490280E88093BC00D7
:105D90001092BD001092BA001092BB001092B90090
:105DA0001092B8000E94A72E0E94AD2E80E00E94A3
:105DB000B52E08958093BB0085E88093BC000895BC
:105DC00085EC8093BC00089585E88093BC0008951D
:105DD0001F920F920FB60F9211242F933F934F9360
:105DE0005F936F937F938F939F93AF93BF93EF9343
:105DF000FF9380914A02282F3327442755278F5F2E
:105E000080934A02F9012731310508F0F2C0E759C1
:105E1000FF4F0C94A57320914902E22FFF27EE0F4C
:105E2000FF1FEE0FFF1FEC5BF94F85851816A4F0DE
:105E30002C3090F4922F9F5FE92FFF27EE0FFF1F6A
:105E4000EE0FFF1FEC5BF94F858518161CF0292F0C
:105E50009C3080F390934902809149028C3051F438
:105E60001092490283E080934A0280914802880F91
:105E70008D5AB4C0880F8E5AB1C080914902E82F64
:105E8000FF27EE0FFF1FEE0FFF1FEE56F94F8F5F3C
:105E9000809349028081A2C08091B9008033E1F4EF
:105EA00080914B02882321F48091490280934B0218
:105EB00080914902E82FFF27EE0FFF1FEE0FFF1F13
:105EC000E157F94F2081822F99278F7790708F3774
:105ED000910514F42F5F20830E94B12E8AE090E098
:105EE0009093BA018093B90110924A026CC08091DC
:105EF000B900909148028034C1F0E92FFF27EE0FDE
:105F0000FF1FEE0FFF1FEE56F94F81818F778183C0
:105F1000892F8F5F809348028C3010F010924802D6
:105F20000E94B12E10924A020DC0E92FFF27EE0FFA
:105F3000FF1FEE0FFF1FEE56F94F818180688183AE
:105F40000E94E02E80914B028093470210924B02F8
:105F500052C080914802E82FFF27EE0FFF1FEE0F7F
:105F6000FF1FEE56F94F8091BB0082830E94E42E02
:105F700042C090914802E92FFF27EE0FFF1FEE0F5E
:105F8000FF1FEE56F94F8091BB008383892F8F5FEF
:105F9000809348028C3010F0109248020E94B12E7B
:105FA00028C080E11BC08091120118C082E116C098
:105FB0008091110113C00E94B12E8AE090E090936D
:105FC000BA018093B9010E94AD2E15C088E906C0C0
:105FD00084E104C08091100101C080E80E94B52EC8
:105FE0000AC00E94B12E8AE090E09093BA0180939B
:105FF000B90110924A028091BC0080688093BC0075
:10600000FF91EF91BF91AF919F918F917F916F9190
:106010005F914F913F912F910F900FBE0F901F9066
:10602000189589E1A7EFB6E0E3ECF6E01182108263
:10603000329611961C921E921296815087FFF6CFCF
:1060400010924F0310924E0310925103109250037E
:10605000109253031092520308951F920F920FB69D
:106060000F9211240F931F932F933F934F935F939E
:106070006F937F938F939F93AF93BF93CF93DF9350
:10608000EF93FF938091360682FDC8C04091860051
:106090005091870080914D0290914E02481B590B00
:1060A000809186009091870090934E0280934D02DC
:1060B000CA018D549440A0914F02B0915002835F69
:1060C0009A4178F480914F028093C206149714F09D
:1060D0001092910181E090E09093500280934F02E2
:1060E000FCC1AD30B1050CF0F8C1CA018B5F904026
:1060F000845B914008F074C0425D5140FD01EA0F9D
:10610000FB1FED53F94F80819181FA01E81BF90BD8
:10611000CF01F7FF03C0909581959F4F06975CF4E0
:106120008091EE02883C20F48091EE02865F01C0EF
:1061300088EC8093EE02FD01EA0FFB1FED53F94F4F
:10614000808191819C01220F331F280F391F240F5A
:10615000351F37FF02C02D5F3F4FE901D595C79529
:10616000D595C795CA0101968C179D0714F4219700
:1061700006C041505040C417D5070CF421968091B9
:10618000EE02833CE0F08D010A0F1B1FF801ED5376
:10619000F94F808191819E01281B390BC90163E071
:1061A00070E00E941E73CB01880F991F860F971F06
:1061B0000950194FD80111969C938E9307C0AA0FCE
:1061C000BB1FA950B94F11961C921E92E0914F022D
:1061D000F0915002EE0FFF1FED53F94FD183C083B2
:1061E00080914F02909150020196909350028093BB
:1061F0004F02059711F45D9A01C05D9880914F029E
:10620000909150028630910511F45C9A01C05C981F
:10621000079711F45B9A61C15B985FC1409186005A
:10622000509187008091510290915202481B590B66
:106230008091860090918700909352028093510242
:10624000CA018D5494406091BB02835F9A4108F06B
:106250007AC060934C0280914C02843008F453C0A1
:106260009091C20680914C02981709F04CC0509151
:10627000BC025B3008F43FC0109291011092BB0247
:1062800040E05F31C0F0E42FFF27EE0FFF1F9F01BA
:1062900029573D4FDF01AD53B94F8D919C91D901E5
:1062A0008D939C93DF01A950B94F8D919C91EF552F
:1062B000FD4F91838083E42FFF27EE0FFF1F9F0187
:1062C0002D53394FDF01AD5ABD4F8D919C91D901AE
:1062D00011969C938E93DF01A359BD4F8D919C9194
:1062E000E950F94F91838083842F8F5F482F8D3041
:1062F00040F28093BB028091BC028F3FB9F08F5F68
:106300008093BC0213C08091BC02853620F08AE0E5
:106310008093BC0202C01092BC02809102018A30BC
:1063200011F0843111F4289A01C0289881E08093FB
:10633000BB028091E502882309F0CFC080914C0216
:106340008093C206CAC06D3008F09FC0CA018B5F3F
:106350009040845B914008F07EC0425D5140E62F42
:10636000FF27EE0FFF1FED5AFD4F80819181FA014B
:10637000E81BF90BCF0105960B97B0F48091BC0296
:106380008A3120F08091EE02865F05C08B3028F0C4
:106390008091EE028E5F8093EE028091EE02893C46
:1063A00018F088EC8093EE02E62FFF27EE0FFF1F18
:1063B000ED5AFD4F808191819C01220F331F280FE0
:1063C000391F240F351F37FF02C02D5F3F4FE901F2
:1063D000D595C795D595C795CA0101968C179D0788
:1063E00014F4219706C041505040C417D5070CF44F
:1063F00021968091EE028E3BD8F0E62FFF27EE0F1C
:10640000FF1FDF01AD5ABD4F8D919C919E01281B4E
:10641000390BC90163E070E00E941E73CB01880F45
:10642000991F860F971FE359FD4F9183808308C002
:10643000E62FFF27EE0FFF1FE359FD4F1182108259
:106440008091BB02E82FFF27EE0FFF1FED5AFD4F93
:10645000D183C08309C0809102018A3011F0843158
:1064600011F4289A01C028988091BB02853011F45C
:106470005D9A05C05D98863011F45C9A05C05C9801
:10648000873011F45B9A01C05B988091BB02843124
:1064900020F48F5F8093BB0220C08431F1F480919F
:1064A00002018A3011F0843111F4289A01C0289831
:1064B0008EE18093BB022CE0C7EFD6E0A7E8B2E004
:1064C000E3ECF6E08D919D91918380833296198261
:1064D00018822296215027FFF5CFFF91EF91DF918F
:1064E000CF91BF91AF919F918F917F916F915F916C
:1064F0004F913F912F911F910F910F900FBE0F90D1
:106500001F9018956817790754F4680F791F77FF63
:1065100002C06F5F7F4FCB01959587950895681BEB
:10652000790B861B970B08951F93CF93DF93182F3A
:10653000EB018091E5028823A1F411501F3F89F0FF
:10654000D093FF01C093FE018091FE019091FF0165
:10655000892BD1F7CE018C0F9D1F0E94241511505D
:1065600078F7DF91CF911F910895CF93DF938091BA
:1065700002018D3011F40E94AB1910927A008091C3
:1065800025029091260290934407809343078091BF
:1065900023029091240290933507809334078091D1
:1065A0002102909122029093850780938407809125
:1065B0001D0290911E029C01442737FD4095542FE7
:1065C000DA01C90172E0880F991FAA1FBB1F7A95D3
:1065D000D1F7820F931FA41FB51F820F931FA41F13
:1065E000B51F9093800780937F0780911F02909141
:1065F00020029C01442737FD4095542FDA01C90140
:1066000062E0880F991FAA1FBB1F6A95D1F7820FFE
:10661000931FA41FB51F820F931FA41FB51F909334
:10662000900780938F0780911B0290911C0290939A
:106630004F0780934E078FEC80937A00AFEEB2E065
:10664000CBEDD5E097E08991E82FFF27EE0FFF1FF4
:10665000ED53F94F0190F081E02DE259FF4F1E16E6
:106660001F061CF0E0E0F0E005C0EF3FF10514F07C
:10667000EFEFF0E08C91282F3327E217F30714F4A3
:10668000815004C02E173F0714F48F5F8C939150F4
:10669000119697FFD8CF809114069927AA27BB2778
:1066A000BC01CD0124EC39E040E050E00E94DF72F3
:1066B000DC01CB018093B3019093B401A093B501A9
:1066C000B093B601809115069927AA27BB27BC0174
:1066D000CD010E94DF72DC01CB018093AF0190936A
:1066E000B001A093B101B093B201DF91CF910895B1
:1066F000A0E0B0E0EEE7F3E30C947273A82EC0E0E4
:10670000D0E07E016E01469AD0934903C0934803BE
:10671000D0934703C093460380E090E0A0E0B0E050
:106720008093400390934103A0934203B0934303AB
:10673000D0935303C0935203D0935103C09350039B
:10674000D0934F03C0934E0310929C0110929B0173
:10675000109215020E94B53284E690E00E94311535
:106760000E94B5328091E30580FF10C08091130133
:1067700090911401875B934038F4809113019091BC
:1067800014018E5E924010F40E945F191FE18AE0AE
:1067900090E00E9431158091210290912202C80F51
:1067A000D91F8091250290912602E80EF91E809152
:1067B000230290912402C80ED91E115017FFE7CF73
:1067C0009701205F3F4F3695279536952795309353
:1067D000530320935203C60140969695879596954C
:1067E000879590935103809350036096A5E0D695CA
:1067F000C795AA95E1F7D0934F03C0934E039093AA
:106800004D0380934C0330934B0320934A03AA20FB
:1068100009F45AC080917F079091800797FF03C0C9
:10682000909581959F4F6CE070E00E941E73EB0184
:10683000709349036093480380918F07909190076C
:1068400097FF03C0909581959F4F6CE070E00E9488
:106850001E7370934703609346038091C90590911E
:10686000CA05AA2797FDA095BA2FBC01CD010E94A9
:106870002B72DC01CB018093400390934103A093E2
:106880004203B0934303BE0184E090E00E944D2C8C
:10689000609146037091470386E090E00E944D2C82
:1068A0008091400390914103A0914203B091430332
:1068B000BC01CD010E94FD71DC01CB01BC0188E06F
:1068C00090E00E944D2C8FC084E090E00E94482C04
:1068D000909349038093480386E090E00E94482CFF
:1068E000909347038093460388E090E00E94482CF1
:1068F000AA2797FDA095BA2FBC01CD010E942B724B
:10690000DC01CB018093400390934103A0934203A9
:10691000B09343038091480390914903815098407C
:10692000C8F480914603909147038150984090F4B9
:106930008091400390914103A0914203B0914303A1
:10694000BC01CD010E94FD71DC01CB01815094405E
:1069500008F449C08BEC99E09F938F938DE391E10C
:106960009F938F93E091FF03F0910004099580912C
:106970007F079091800797FF03C0909581959F4F67
:106980006CE070E00E941E737093490360934803AB
:1069900080918F079091900797FF03C09095819504
:1069A0009F4F6CE070E00E941E73709347036093EA
:1069B00046038091C9059091CA05AA2797FDA09525
:1069C000BA2FBC01CD010E942B72DC01CB01809358
:1069D000400390934103A0934203B09343030F906D
:1069E0000F900F900F90109244071092430710924F
:1069F000350710923407109285071092840784E6B9
:106A000090E00E94311580911D0290911E02AA27EC
:106A100097FDA095BA2F9C01AD01F2E0220F331F24
:106A2000441F551FFA95D1F7280F391F4A1F5B1FC6
:106A3000280F391F4A1F5B1F3093800720937F0761
:106A400080911F0290912002AA2797FDA095BA2F4E
:106A50007C018D01E2E0EE0CFF1C001F111FEA9586
:106A6000D1F7E80EF91E0A1F1B1FE80EF91E0A1FB8
:106A70001B1FF0929007E0928F078091F205682E1D
:106A8000772488249924C9019C01442737FD409527
:106A9000542FC401B3010E94DF725B016C0160934B
:106AA0003A0370933B0380933C0390933D0397011B
:106AB000442737FD4095542FC401B3010E94DF7273
:106AC000DC01CB018093320390933303A093340312
:106AD000B0933503A0921603B0921703C092180327
:106AE000D092190380930E0390930F03A093100389
:106AF000B093110310920A0310920B0310920C032F
:106B000010920D038091150190911601A09117012B
:106B1000B09118019093CC058093CB05109214028C
:106B200010921302109202031092030310920403B6
:106B30001092050380910003909101039093FF024E
:106B40008093FE020E948C5D82E390E09093FF01AF
:106B50008093FE01809114069927AA27BB27BC01C8
:106B6000CD0124EC39E040E050E00E94DF72DC010E
:106B7000CB018856954CAF4FBF4F8093B301909394
:106B8000B401A093B501B093B60180911506992781
:106B9000AA27BB27BC01CD010E94DF72DC01CB011B
:106BA0008856954CAF4FBF4F8093AF019093B00183
:106BB000A093B101B093B201109298011092970185
:106BC0008091000390910103AA2797FDA095BA2F09
:106BD000209193013091940140919501509196013B
:106BE000BC01CD010E94DF72DC01CB0180938B07D9
:106BF00090938C07A0938D07B0938E071092F902A3
:106C00001092F80281E0809301010E94AA618091B4
:106C1000BD0284608093BD028FEF8093FC071092C9
:106C2000FD0780E28093FE07CFEED2E0ABEDB5E04A
:106C300017E08D91E82FFF27EE0FFF1FED53F94F5F
:106C40008081918182598993115017FFF2CF84E698
:106C50008093EE028091FC01882311F0469A579AA6
:106C6000EEE0CDB7DEB70C948E73A3E1B0E0EBE3BA
:106C7000F6E30C946E7380914E0390914F03209134
:106C8000210230912202821B930B909385078093FF
:106C9000840780912B0290912C0297FD07969C010E
:106CA00053E0359527955A95E1F7309344072093A3
:106CB00043078091290290912A0297FD079643E0AD
:106CC000959587954A95E1F790933507809334071A
:106CD00030935107209350079093470780934607BE
:106CE00080917F0790918007AA2797FDA095BA2FE2
:106CF0007C018D01EE0CFF1C001F111FE80EF91E18
:106D00000A1F1B1F80911D0290911E029C014427A7
:106D100037FD4095542FDA01C901F2E0880F991F21
:106D2000AA1FBB1FFA95D1F7820F931FA41FB51F8F
:106D3000820F931FA41FB51FE80EF91E0A1F1B1F09
:106D400017FF08C023E030E040E050E0E20EF31E01
:106D5000041F151FE2E015950795F794E794EA954F
:106D6000D1F7F0928007E0927F0780918F07909192
:106D70009007AA2797FDA095BA2F7C018D01EE0CF4
:106D8000FF1C001F111FE80EF91E0A1F1B1F809118
:106D90001F02909120029C01442737FD4095542FFB
:106DA000DA01C90162E0880F991FAA1FBB1F6A950B
:106DB000D1F7820F931FA41FB51F820F931FA41F2B
:106DC000B51FE80EF91E0A1F1B1F17FF08C083E03E
:106DD00090E0A0E0B0E0E80EF91E0A1F1B1F82E061
:106DE00015950795F794E7948A95D1F7F092900757
:106DF000E0928F0780914E0790914F07AA2797FD49
:106E0000A095BA2F9C01AD01220F331F441F551FBF
:106E1000280F391F4A1F5B1F80911B0290911C0293
:106E2000AA2797FDA095BA2F280F391F4A1F5B1F6D
:106E300057FF04C02D5F3F4F4F4F5F4FF2E0559516
:106E4000479537952795FA95D1F730934F072093BB
:106E50004E0720911D0230911E02C901880F991F13
:106E6000880F991F820F931F820F931F9C01442745
:106E700037FD4095542F80912A0390912B03A091C8
:106E80002C03B0912D03820F931FA41FB51F809375
:106E90002A0390932B03A0932C03B0932D032091EE
:106EA0001F0230912002C901880F991F880F991F76
:106EB000820F931F820F931F9C01442737FD40953B
:106EC000542F8091260390912703A0912803B0911D
:106ED0002903820F931FA41FB51F8093260390934D
:106EE0002703A0932803B093290380915A07909118
:106EF0005B0720911D0230911E02820F931F909319
:106F00005B0780935A0780918707909188072091AB
:106F10001F0230912002820F931F90938807809365
:106F20008707809144039091450301969093450310
:106F3000809344038091220390912303A091240322
:106F4000B0912503BC01CD010E942B725B016C0145
:106F50008091C9059091CA05AA2797FDA095BA2FDF
:106F6000BC01CD010E942B727B018C0180914003FA
:106F700090914103A0914203B09143039C01AD0164
:106F8000C801B7010E948F71DC01CB019C01AD01EA
:106F9000C601B5010E949071DC01CB01BC01CD019D
:106FA0000E94F871DC01CB018093220390932303AC
:106FB000A0932403B09325038FEC80937A00109262
:106FC0000F0120911203309113034091140350914B
:106FD000150329873A874B875C8729543B464140F4
:106FE00050402CF028E43BE641E050E00DC089859C
:106FF0009A85AB85BC85885B9449AE4FBF4F4CF4F6
:1070000028EB34E94EEF5FEF2D833E834F835887A3
:1070100008C089859A85AB85BC858D839E83AF83A7
:10702000B88720911A0330911B0340911C035091A3
:107030001D032D873E874F87588B29543B4641407F
:1070400050402CF028E43BE641E050E00DC08D8537
:107050009E85AF85B889885B9449AE4FBF4F4CF48D
:1070600028EB34E94EEF5FEF29833A834B835C834F
:1070700008C08D859E85AF85B88989839A83AB8347
:10708000BC83A0918407B0918507BA8BA98BFD01C1
:10709000CF01AA2797FDA095BA2FA0900A03B09020
:1070A0000B03C0900C03D0900D03A80EB91ECA1E8E
:1070B000DB1EA0920A03B0920B03C0920C03D09285
:1070C0000D03E0908B07F0908C0700918D071091D5
:1070D0008E07E80EF91E0A1F1B1FE0928B07F09225
:1070E0008C0700938D0710938E07F091D702FB8BCE
:1070F000FF2309F098C18091D602882309F093C13B
:107100008091E30586FF8FC1809134079091350708
:10711000AA2797FDA095BA2FBC01CD0129813A81FC
:107120004B815C810E94DF729B01AC0197FF04C020
:107130002150384F4F4F5F4F6BE05595479537952E
:1071400027956A95D1F780919B01682E7724882432
:107150009924CA01B901A40193010E94DF72DC01E4
:10716000CB0180935E0390935F03A0936003B09381
:107170006103B7FF04C08150904FAF4FBF4F1C0158
:107180002D013CE055944794379427943A95D1F7D4
:1071900020925E0330925F0340926003509261033D
:1071A0008091430790914407AA2797FDA095BA2F95
:1071B000BC01CD012D813E814F8158850E94DF7237
:1071C00097FF04C06150784F8F4F9F4F2BE09595EC
:1071D0008795779567952A95D1F7A40193010E9429
:1071E000DF72DC01CB018093620390936303A09371
:1071F0006403B0936503B7FF04C08150904FAF4F55
:10720000BF4F9C01AD018CE055954795379527956B
:107210008A95D1F72093620330936303409364030C
:107220005093650380915E0390915F0390932C07C8
:1072300080932B07809162039091630390933007B2
:1072400080932F07221933094409550920936203BB
:10725000309363034093640350936503E20EF31E7F
:10726000041F151FE0928B07F0928C0700938D0787
:1072700010938E0780919A018823B1F457FF04C0C0
:107280002F5F3F4F4F4F5F4F559547953795279548
:10729000A21AB30AC40AD50AA0920A03B0920B0339
:1072A000C0920C03D0920D0329893A8979010027F5
:1072B000F7FC0095102F8091620390916303A091D9
:1072C0006403B0916503E80EF91E0A1F1B1FC80175
:1072D000B70129813A814B815C810E94DF729B0159
:1072E000AC0197FF04C02150384F4F4F5F4FBBE0B8
:1072F0005595479537952795BA95D1F780919C017B
:10730000A82EBB24CC24DD24CA01B901A601950115
:107310000E94DF72DC01CB018093560390935703E8
:10732000A0935803B0935903B7FF04C08150904F06
:10733000AF4FBF4F3C014D01ACE0959487947794DB
:107340006794AA95D1F76092560370925703809282
:10735000580390925903C801B7012D813E814F8196
:1073600058850E94DF7297FF04C06150784F8F4F9D
:107370009F4FFBE09595879577956795FA95D1F79F
:10738000A60195010E94DF72DC01CB0180935A03B4
:1073900090935B03A0935C03B0935D03B7FF04C0BD
:1073A0008150904FAF4FBF4FAC01BD01ECE07595E0
:1073B000679557954795EA95D1F740935A035093AF
:1073C0005B0360935C0370935D0329893A8937FFFF
:1073D00003C0309521953F4F21343105E4F1D401AC
:1073E000C30197FE07C0B095A095909581959F4FDA
:1073F000AF4FBF4F81389105A105B10584F4DB0182
:10740000CA0177FF07C0B095A095909581959F4FD1
:10741000AF4FBF4F81389105A105B105E4F081E080
:107420008093FA0218C01092300710922F07109222
:107430002C0710922B0710925A0310925B031092A4
:107440005C0310925D031092560310925703109242
:1074500058031092590380915A0390915B03A091B5
:107460005C03B0915D03BC01CD0124E630E040E057
:1074700050E00E945373E0905603F0905703E21AD5
:10748000F30AF0924207E0924107809156039091EF
:107490005703A0915803B0915903BC01CD0124E6D4
:1074A00030E040E050E00E945373DA01C9012091BE
:1074B0005A0330915B038C01021B130B10933707A7
:1074C000009336078091930190919401A0919501CA
:1074D000B0919601BC01CD0128E631E040E050E0DA
:1074E0000E94DF7220918B0730918C0740918D07AD
:1074F00050918E07261737074807590764F0261B57
:10750000370B480B590B20938B0730938C07409314
:107510008D0750938E0720918B0730918C074091F7
:107520008D0750918E0757FF0CC0260F371F481F3D
:10753000591F20938B0730938C0740938D075093EE
:107540008E0760913407709135076E0D7F1D9B018A
:10755000442737FD4095542F80910E0390910F03DF
:10756000A0911003B0911103820F931FA41FB51FA8
:1075700080930E0390930F03A0931003B093110315
:107580008091DA029091DB02681B790BCB01AA276C
:1075900097FDA095BA2F29853A854B855C85820F8A
:1075A000931FA41FB51F8093120390931303A093FE
:1075B0001403B0931503C090AF01D090B001E090D8
:1075C000B101F090B201C816D906EA06FB06C4F470
:1075D00088EA91E6A0E0B0E08C199D09AE09BF09E8
:1075E0008093120390931303A0931403B093150395
:1075F00080930E0390930F03A0931003B093110395
:1076000022273327A9012C193D094E095F098091D2
:10761000120390911303A0911403B09115038217E4
:107620009307A407B507B4F4D701C601885A914659
:10763000A040B0408093120390931303A0931403CF
:10764000B093150380930E0390930F03A093100340
:10765000B09311036091430770914407600F711F4D
:107660009B01442737FD4095542F8091160390913C
:107670001703A0911803B0911903820F931FA41F41
:10768000B51F8093160390931703A0931803B0932C
:1076900019038091D8029091D902681B790BCB0114
:1076A000AA2797FDA095BA2F2D853E854F8558892D
:1076B000820F931FA41FB51F80931A0390931B037F
:1076C000A0931C03B0931D03E090B301F090B401AC
:1076D0000091B5011091B601E816F9060A071B07DB
:1076E000C4F488EA91E6A0E0B0E08E199F09A00BEF
:1076F000B10B80931A0390931B03A0931C03B093C8
:107700001D038093160390931703A0931803B0935F
:10771000190322273327A9012E193F09400B510BCA
:1077200080911A0390911B03A0911C03B0911D033B
:1077300082179307A407B507B4F4D801C701885A84
:107740009146A040B04080931A0390931B03A093EE
:107750001C03B0931D038093160390931703A0930B
:107760001803B093190380910A0390910B03A09121
:107770000C03B0910D0380931E0390931F03A093FD
:107780002003B093210380911A0390911B03A091D1
:107790001C03B0911D0380933A0390933B03A09385
:1077A0003C03B0933D038091120390911303A09189
:1077B0001403B09115038093320390933303A09385
:1077C0003403B09335038091160390911703A09171
:1077D0001803B09119038093360390933703A09355
:1077E0003803B093390380910E0390910F03A09159
:1077F0001003B091110380932E0390932F03A09355
:107800003003B093310380911B0190911C0197FDCF
:10781000079633E0959587953A95E1F7909344075D
:10782000809343078091190190911A0197FD079663
:1078300023E0959587952A95E1F7909335078093F6
:10784000340780912502909126020F9734F488E145
:107850009CEF909344078093430780912502909179
:107860002602079734F480E398EF909344078093BF
:107870004307209102012A30A9F4809125029091BA
:107880002602835F934034F088EE93E090934407A0
:107890008093430780912502909126028A5F93404E
:1078A000DCF014C08091250290912602815D974002
:1078B00034F088EE93E090934407809343078091DF
:1078C000250290912602805E974034F080ED97E08B
:1078D0009093440780934307809123029091240260
:1078E0000F9734F488E19CEF909335078093340729
:1078F0008091230290912402079734F480E398EF5B
:1079000090933507809334072A30A9F4809123029D
:1079100090912402835F934034F088EE93E090933B
:1079200035078093340780912302909124028A5F67
:107930009340DCF014C08091230290912402815D79
:10794000974034F088EE93E09093350780933407A6
:107950008091230290912402805E974034F080ED64
:1079600097E09093350780933407E091A601EE23CA
:1079700009F4B7C040911B0150911C01809166032E
:1079800090916703481B590B50936D0340936C0310
:1079900020911B0130911C01280F391F37FF02C0B5
:1079A0002F5F3F4F359527953093670320936603EC
:1079B000413851051CF080E890E005C040585F4F09
:1079C00034F480E89FEF90936D0380936C038E2FC7
:1079D0009927A0916C03B0916D03A89FA001A99F66
:1079E000500DB89F500D112457FF02C0415F5F4FEB
:1079F00014E0559547951A95E1F7809143079091CA
:107A00004407840F951F9093440780934307609128
:107A1000190170911A018091680390916903681BA4
:107A2000790B70936B0360936A0340911901509135
:107A30001A01480F591F57FF02C04F5F5F4F5595FE
:107A400047955093690340936803613871051CF0B2
:107A500080E890E005C060587F4F34F480E89FEFE5
:107A600090936B0380936A032E2F332780916A03D0
:107A700090916B03829FB001839F700D929F700D58
:107A80001124AB0177FF02C0415F5F4FE4E05595E1
:107A90004795EA95E1F78091340790913507840F77
:107AA000951F9093350780933407A29FC001A39F31
:107AB000900DB29F900D11249C0180911B0190911B
:107AC0001C01820F931F90931C0180931B018091D6
:107AD000190190911A01860F971F90931A018093B4
:107AE0001901009146071091470780912B0790914B
:107AF0002C07101611065CF59C0197FF04C0222785
:107B00003327281B390BC901AA2797FDA095BA2F47
:107B100020919A01332744275527BC01CD010E94AB
:107B2000DF729B01AC0197FF04C0215C3F4F4F4FB8
:107B30005F4F76E055954795379527957A95D1F71C
:107B40008091410790914207820F931F27C097FFB2
:107B500003C0909581959F4FAA2797FDA095BA2FB6
:107B600020919A01332744275527BC01CD010E945B
:107B7000DF729B01AC0197FF04C0215C3F4F4F4F68
:107B80005F4F66E055954795379527956A95D1F7EC
:107B90008091410790914207821B930B909342077B
:107BA00080934107E0905007F090510780912F0794
:107BB000909130071E141F045CF59C0197FF04C0D0
:107BC00022273327281B390BC901AA2797FDA09527
:107BD000BA2F20919A01332744275527BC01CD01A4
:107BE0000E94DF729B01AC0197FF04C0215C3F4FF4
:107BF0004F4F5F4F96E055954795379527959A9546
:107C0000D1F78091360790913707820F931F27C0D5
:107C100097FF03C0909581959F4FAA2797FDA09548
:107C2000BA2F20919A01332744275527BC01CD0153
:107C30000E94DF729B01AC0197FF04C0215C3F4FA3
:107C40004F4F5F4F86E055954795379527958A9515
:107C5000D1F78091360790913707821B930B909351
:107C60003707809336078091E30587FF44C09B89DF
:107C7000992309F040C08091D6028823E1F5A1E064
:107C8000EA16A1E0FA064CF0809143079091440770
:107C90008E0D9F1D805091400DC0B0E0EB16BFEFE0
:107CA000FB0664F480914307909144078E0D9F1D5D
:107CB00080509F4F9093440780934307E1E0013049
:107CC0001E074CF08091340790913507800F911F6B
:107CD000805091400CC0FFEF00301F0764F480918A
:107CE000340790913507800F911F80509F4F9093DC
:107CF000350780933407AFEEB2E06BED75E057E0E7
:107D0000FB018191BF01E82FFF27EE0FFF1FED530D
:107D1000F94F0190F081E02DE259FF4FEF3FF1055F
:107D200021F01CF0EFEFF0E004C0F7FF02C0E0E04C
:107D3000F0E04C91242F3327E217F307B1F0CF0185
:107D4000821B930B97FD079603E0959587950A95FF
:107D5000E1F7242F280F2C93822F9927E817F90792
:107D600014F4215001C02F5F2C935150119657FFEE
:107D7000C7CFE2E1CD5E0C948A738091E50288233F
:107D8000F9F48091BD028C7F8093BD02A2E9B6E038
:107D9000EDE1F4E09BE08091DF01882309F480832A
:107DA00081918C931496915097FFF5CF8091DF01CC
:107DB000882359F08091DF0181508093DF0105C055
:107DC0008091BD0281608093BD02809192069927C7
:107DD00090939F0580939E05809196069927909396
:107DE000A1058093A00580919A0699279093A305F9
:107DF0008093A20580919E0699279093A505809374
:107E0000A40510924A02109249020E94AD2E0895D4
:107E10008091E505883F38F0EFEFF0E0E81BF109CD
:107E2000E151FD4F80818093AC018091AC018823AA
:107E300029F0843618F084E68093AC018091E70540
:107E4000883F38F0EFEFF0E0E81BF109E151FD4F1A
:107E500080818093AA018091AA01882329F0843629
:107E600018F084E68093AA018091F405883F38F0E9
:107E7000EFEFF0E0E81BF109E151FD4F80818093C5
:107E8000A5018091A5018B3010F48AE002C08F3FDC
:107E900011F48093A50180911E06883F38F0EFEF22
:107EA000F0E0E81BF109E151FD4F808180935C0710
:107EB00080915C07823010F481E002C08F3F11F4A2
:107EC00080935C0780912006883F38F0EFEFF0E068
:107ED000E81BF109E151FD4F808180938207809179
:107EE0008207823010F481E002C08F3F11F480934A
:107EF000820780910B06883F38F0EFEFF0E0E81B37
:107F0000F109E151FD4F80818093590780910C0662
:107F1000883F38F0EFEFF0E0E81BF109E151FD4F49
:107F200080818093310780910D06883F38F0EFEF14
:107F3000F0E0E81BF109E151FD4F8081809361077A
:107F40009091E605983F18F49093AB0109C0EFEFCC
:107F5000F0E0E91BF109E151FD4F80818093AB0115
:107F6000983F18F49093AB0109C0EFEFF0E0E91BE4
:107F7000F109E151FD4F80818093AB018091E905CA
:107F8000883F38F0EFEFF0E0E81BF109E151FD4FD9
:107F900080818093A9018091EB05883F38F0EFEF55
:107FA000F0E0E81BF109E151FD4F80818093A701CA
:107FB0008091F305883F38F0EFEFF0E0E81BF1091E
:107FC000E151FD4F80818093A8018091F505883FA4
:107FD00038F0EFEFF0E0E81BF109E151FD4F80814F
:107FE0008093A4018091F605883F38F0EFEFF0E030
:107FF000E81BF109E151FD4F80818093A60180913A
:10800000F705883F38F0EFEFF0E0E81BF109E151A8
:10801000FD4F80818093A3018091F805883F38F05F
:10802000EFEFF0E0E81BF109E151FD4F8081809313
:10803000A2018091FD05883F38F0EFEFF0E0E81BEA
:10804000F109E151FD4F80818093A0018091FE05EF
:10805000883F38F0EFEFF0E0E81BF109E151FD4F08
:1080600080818093D1028091FF05883F38F0EFEF47
:10807000F0E0E81BF109E151FD4F80818093D002CF
:1080800080910006883F38F0EFEFF0E0E81BF1093F
:10809000E151FD4F80818093CF0280910106883F9E
:1080A00038F0EFEFF0E0E81BF109E151FD4F80817E
:1080B0008093CE0280911906883F38F0EFEFF0E010
:1080C000E81BF109E151FD4F80818093CD02809141
:1080D0001A06883F38F0EFEFF0E0E81BF109E151B4
:1080E000FD4F80818093CC0280911B06883F38F041
:1080F000EFEFF0E0E81BF109E151FD4F8081809343
:10810000CB0280911C06883F38F0EFEFF0E0E81BCF
:10811000F109E151FD4F80818093CA0280910206EE
:10812000883F38F0EFEFF0E0E81BF109E151FD4F37
:10813000808180939F0180910606883F38F0EFEFA1
:10814000F0E0E81BF109E151FD4F808180939E0131
:1081500080910E06883F38F0EFEFF0E0E81BF10960
:10816000E151FD4F808180939D0180911106883FF0
:1081700038F0EFEFF0E0E81BF109E151FD4F8081AD
:1081800080939C0180911206883F38F0EFEFF0E079
:10819000E81BF109E151FD4F808180939B018091A3
:1081A0001306883F38F0EFEFF0E0E81BF109E151EA
:1081B000FD4F808180939A0180911806883F38F0A6
:1081C000EFEFF0E0E81BF109E151FD4F8081809372
:1081D000990180913306883F38F0EFEFF0E0E81B1B
:1081E000F109E151FD4F8081809392078091A001B8
:1081F000282F33272F5F3F4F8CE398E2B9010E946D
:108200001E737093AE016093AD018091F105809370
:1082100083078091F005809348070895A4E1B0E0BA
:10822000E4E1F1E40C946E730E9435363091020162
:108230003C3010F4299A01C02998E090E602F090B1
:10824000E702FA82E9828091480799270A96E816A0
:10825000F90614F49A8389838091EE02843608F03B
:108260005CC080918A0390918B03009731F0019755
:1082700090938B0380938A0307C01092E50280914C
:10828000BD028F7E8093BD023A3011F0343111F47B
:10829000289A01C028988091BE029091BF02895E01
:1082A0009340C0F18091FA05282F33273A83298320
:1082B0008091BD0280618093BD028091D705A82F77
:1082C000BB27AA0FBB1FFD01E950F94F1182108295
:1082D0008091D805282F3327220F331FC9018950D9
:1082E000994FFC0111821082AD53B94F11961C9227
:1082F0001E922D53394FD90111961C921E928091D6
:10830000DA05E82FFF27EE0FFF1FED53F94F11821B
:1083100010828FC21092E5028CC28091EE028D38DD
:1083200008F487C28091BD028F7E8093BD02909138
:10833000FB0582E3989FC001112490938B038093E7
:108340008A03E981FA81B9978CF08091E50288234C
:1083500069F08091BE029091BF02FFEF8F3F9F07AF
:1083600029F001969093BF028093BE028091BE02D5
:108370009091BF028F3F910509F038F510926E037E
:1083800010926F0310927003109271031092720397
:108390001092730310927403109275038A3F910533
:1083A000C9F481E0809391031092760310927703D1
:1083B000109278031092790310920A0310920B0323
:1083C00010920C0310920D0305C08091BD028260D3
:1083D0008093BD028091D905E82FFF27EE0FFF1F84
:1083E000ED53F94F80819181813591050CF441C1A4
:1083F0002091E502222309F03CC18091DA05E82FA3
:10840000FF27EE0FFF1FED53F94F808191818C34D0
:1084100091050CF406C180918C038F5F80938C03CF
:10842000893C08F426C13C3010F4299801C0299AEF
:108430001092E50210928C031092BF021092BE02BD
:108440003091D705E32FFF27EE0FFF1FED53F94FB4
:108450008081918187349105B4F48091D805E82F0B
:10846000FF27EE0FFF1FED53F94F8081918101909F
:10847000F081E02DF7FF03C0F095E195FF4FE73461
:10848000F1050CF478C041E02091D805A22FBB275C
:10849000AA0FBB1FAD53B94F8D919C911197873493
:1084A000910544F0E32FFF27EE0FFF1FED53F94F27
:1084B000808191818D919C918734910574F0809198
:1084C000D705E82FFF27EE0FFF1FED53F94F8081EF
:1084D0009181873491050CF042E0E22FFF27EE0FE7
:1084E000FF1FED53F94F808191818634910574F41B
:1084F0008091D705E82FFF27EE0FFF1FED53F94FAF
:1085000080819181873491050CF043E0E22FFF27B1
:10851000EE0FFF1FED53F94F808191818A5B9F4FD2
:1085200074F48091D705E82FFF27EE0FFF1FED535E
:10853000F94F80819181873491050CF044E0E22F5E
:10854000FF27EE0FFF1FED53F94F808191818A5B6A
:108550009F4F74F48091D705E82FFF27EE0FFF1F80
:10856000ED53F94F80819181863491050CF445E0FB
:10857000842F0E94A52C8091D805E82FFF27EE0FAD
:10858000FF1FED53F94F808191810190F081E02D23
:10859000F7FF03C0F095E195FF4F7E97BCF4809103
:1085A000D705E82FFF27EE0FFF1FED53F94F80810E
:1085B00091818A5B9F4F54F481E08093330488EE6D
:1085C00093E09093FF018093FE0153C00E949F2D82
:1085D0000E94522C80E00E9430078091FC050E948E
:1085E000E16E8091E30580FF10C0809113019091AE
:1085F0001401875B934038F480911301909114012A
:108600008E5E924010F40E945F191092FC0180E08F
:108610000E94783381E080938F038093FC01579A06
:108620001FC080819181855B9F4F0CF580918C03E9
:108630008F5F80938C03893CE0F03C3010F42998E4
:1086400001C0299A1092E50210928C031092BF0289
:108650001092BE0281E00E94783381E080938F0304
:108660000E949F2D68E770E00E94943202C0209320
:108670008C038091D905E82FFF27EE0FFF1FED53E4
:10868000F94F808191818B5A9F4F0CF0D2C020917D
:10869000E502E091DA05222309F0AFC0FF27EE0FD3
:1086A000FF1FED53F94F80819181855B9F4F0CF047
:1086B000A1C080918D038F5F80938D03893C08F466
:1086C000B8C020938D0380918F03882309F48BC059
:1086D00081E090E09093BF028093BE0281E080939E
:1086E000E5021092760310927703109278031092AD
:1086F000790310920A0310920B0310920C0310924C
:108700000D031092060310920703109208031092B3
:1087100009038091F205E82EFF240027112780919C
:108720007F07909180079C01442737FD4095542F87
:10873000C801B7010E94DF72DC01CB0180931A03EC
:1087400090931B03A0931C03B0931D0380918F078C
:10875000909190079C01442737FD4095542FC80104
:10876000B7010E94DF72DC01CB018093120390936A
:108770001303A0931403B093150380913A039091CF
:108780003B03A0913C03B0913D038093160390936B
:108790001703A0931803B0931903809132039091AB
:1087A0003303A0913403B091350380930E0390936B
:1087B0000F03A0931003B093110310926E03109255
:1087C0006F03109270031092710310927203109253
:1087D000730310927403109275038091BD02886038
:1087E0008093BD0226C08CED95E09093FF018093AD
:1087F000FE011FC020938D031CC0FF27EE0FFF1F3B
:10880000ED53F94F808191818C34910584F08091F2
:108810008E038F5F80938E03893C58F01092E5029F
:1088200010928E031092BF021092BE0202C01092EC
:108830008E038091910181508093910180919101EB
:108840008F3F21F08091BD0284FFD5C20E94083F76
:1088500080919A0390919B03AC01440F551F480FE0
:10886000591F0091D705A02FBB27AA0FBB1FFD01E1
:10887000ED53F94FF090ED05CF2CDD2480819181EF
:108880008C9DF0018D9DF00D9C9DF00D11244E0FDF
:108890005F1F57FF02C04D5F5F4F55954795559538
:1088A0004795A950B94F8091EE05682F77278D9194
:1088B0009C91869F9001879F300D969F300D1124CB
:1088C000420F531F50939B0340939A038091D1030F
:1088D0009091D2032091CD033091CE03820F931F4C
:1088E000481B590B5093ED024093EC0280919C037E
:1088F00090919D03AC01440F551F480F591F1091D3
:10890000D805A12FBB27AA0FBB1FFD01ED53F94FBF
:10891000808191818C9DF0018D9DF00D9C9DF00DCD
:1089200011244E0F5F1F57FF02C04D5F5F4F5595DB
:10893000479555954795A950B94F8D919C91869F24
:108940009001879F300D969F300D1124420F531FC9
:1089500050939D0340939C038091CF039091D0034B
:108960002091CB033091CC03820F931F481B590BEE
:108970005093EB024093EA028091DA05E82FFF273B
:10898000EE0FFF1FED53F94F8081918190958195F6
:108990009F4F9093E9028093E8028330910514F091
:1089A000029705C03FEF8E3F930734F402969093F1
:1089B000E9028093E80204C01092E9021092E802F2
:1089C0008091D905E82FFF27EE0FFF1FED53F94FD8
:1089D000C080D18048E750E0C40ED51ED092E70297
:1089E000C092E6028091A5019927AA2797FDA0953C
:1089F000BA2FBC01CD010E942B72DC01CB0120E01B
:108A000030E040E251E4BC01CD010E949071DC01F4
:108A1000CB01BC01CD010E94FD71DC01CB01809333
:108A200089078091A401809362078091A30199270F
:108A3000AA2797FDA095BA2FBC01CD010E942B72E9
:108A4000DC01CB0120E030E040E251E4BC01CD018B
:108A50000E949071DC01CB01BC01CD010E94FD712F
:108A6000DC01CB0180933B078091A20180935207E8
:108A700080913F0480FF61C080919207813808F4A3
:108A80005CC080913804992787FD90954F2D55271C
:108A9000849F9001859F300D949F300D112480910B
:108AA000EC029091ED02820F931F9093ED02809360
:108AB000EC0280913904992787FD9095849F90015D
:108AC000859F300D949F300D11248091EA02909182
:108AD000EB02820F931F9093EB028093EA02809146
:108AE0003A04282F332727FD30958091E802909192
:108AF000E902820F931F9093E9028093E80280912C
:108B00003C04282F332727FD30958091E8059927CD
:108B1000289FB001299F700D389F700D112470930C
:108B200098016093970180913B0499278C159D05CE
:108B300024F49093E7028093E6028091E6029091FC
:108B4000E70297FF04C01092E7021092E6028091BC
:108B5000E30582FF02C0109262074091EC0250913F
:108B6000ED02CA0157FD03969C0135952795359571
:108B7000279537FF03C0309521953F4F8091C20262
:108B80009091C30282179307B4F4CA0157FF03C040
:108B9000909581959F4F97FD03969595879595950F
:108BA00087959093C3028093C2028536910544F065
:108BB00084E690E001C001979093C3028093C202C3
:108BC0004091EA025091EB02CA0157FD03969C01C5
:108BD000359527953595279537FF03C03095219515
:108BE0003F4F8091C0029091C10282179307B4F465
:108BF000CA0157FF03C0909581959F4F97FD03963B
:108C000095958795959587959093C1028093C0021D
:108C10008536910544F084E690E001C00197909379
:108C2000C1028093C0028091BD0284FF08C01092EF
:108C3000C3021092C2021092C1021092C002E12F30
:108C4000FF27EE0FFF1FED53F94F40910F06242F22
:108C50003327808191812817390744F480913406A5
:108C600082FF04C081E08093D50213C0E12FFF276B
:108C7000EE0FFF1FED53F94F842F99272091100617
:108C8000821B9109208131812817390714F4109231
:108C9000D5024091D805E42FFF27EE0FFF1FED53BB
:108CA000F94F50910F06852F992722273327281B2C
:108CB000390B808191818217930744F480913406A7
:108CC00083FF04C081E08093D40216C08091D40257
:108CD000882391F0E42FFF27EE0FFF1FED53F94F8C
:108CE000809110069927851B910920813181821777
:108CF000930714F41092D402E02FFF27EE0FFF1F0A
:108D0000ED53F94F40910F06242F33278081918135
:108D10002817390744F48091340680FF04C081E0AD
:108D20008093D20217C08091D202882399F0E02F5D
:108D3000FF27EE0FFF1FED53F94F842F9927209146
:108D40001006821B9109208131812817390714F4FC
:108D50001092D2024091D705E42FFF27EE0FFF1F9C
:108D6000ED53F94F50910F06852F9927222733276E
:108D7000281B390B808191818217930744F48091DD
:108D8000340681FF04C081E08093D30216C0809135
:108D9000D302882391F0E42FFF27EE0FFF1FED533E
:108DA000F94F809110069927851B91092081318107
:108DB0008217930714F41092D3028091D50288236E
:108DC00019F48091D402811181E08093D6028091C0
:108DD000D202882321F48091D302882351F081E0CC
:108DE0008093D7021092D6021092D5021092D4022C
:108DF00002C08093D7028091D602882321F480910B
:108E0000D702882369F080910E069927A981BA813B
:108E10008A179B0714F49A83898381E08093FA026E
:108E20008091BD0284FF1AC01092E9021092E802FC
:108E30001092ED021092EC021092EB021092EA02F4
:108E40009AE59093890788E78093620790933B07A0
:108E5000809352071092D6021092D7028091550744
:108E600090915607A0915707B091580720913A0367
:108E700030913B0340913C0350913D03820F931F7F
:108E8000A41FB51F8093550790935607A0935707CB
:108E9000B093580780915D0790915E07A0915F079E
:108EA000B091600720903203309033034090340338
:108EB00050903503820D931DA41DB51D80935D0751
:108EC00090935E07A0935F07B093600780914A0775
:108ED00090914B07A0914C07B0914D07E09036035D
:108EE000F09037030091380310913903EB82FC8234
:108EF0000D831E838E0D9F1DA01FB11F80934A07F7
:108F000090934B07A0934C07B0934D0780913C077B
:108F100090913D07A0913E07B0913F07E0902E034E
:108F2000F0902F030091300310913103EF82F88607
:108F300009871A878E0D9F1DA01FB11F80933C07C4
:108F400090933D07A0933E07B0933F07F090D70260
:108F5000FB86FF2029F48091D602882309F460C0A3
:108F600010922A0310922B0310922C0310922D03BF
:108F700010922603109227031092280310922903BF
:108F800010925507109256071092570710925807E3
:108F900010925D0710925E0710925F0710926007B3
:108FA00010924A0710924B0710924C0710924D07EF
:108FB00010923C0710923D0710923E0710923F0717
:108FC00080911A0390911B03A0911C03B0911D0383
:108FD0008093160390931703A0931803B09319037B
:108FE0008091120390911303A0911403B091150383
:108FF00080930E0390930F03A0931003B09311037B
:1090000010921202109211021092D9021092D802FC
:109010001092DB021092DA020B85002309F0F2C1F4
:109020008091D602882309F0EDC18091C905909105
:10903000CA05815092402CF48091E502882309F4FE
:10904000E1C19090FC07A090F20560917F077091BC
:1090500080077C8B6B8B80918F07909190079A8B08
:10906000898B9FEF991609F4D9C0BB24CC24DD2449
:10907000CA01B901A60195010E94537379018A01C1
:10908000EB89FC89CF01AA2797FDA095BA2FE81A92
:10909000F90A0A0B1B0BC201B101A60195010E943E
:1090A000537359016A0129893A89C901AA2797FD91
:1090B000A095BA2FA81AB90ACA0ADB0A292C3324A8
:1090C00027FC3094432C532CC801B701A201910115
:1090D0000E94DF7297FF04C061507E4F8F4F9F4FF9
:1090E0003B014C0129E095948794779467942A95E5
:1090F000D1F7C601B501A20191010E94DF7297FF6D
:1091000004C061507E4F8F4F9F4F5B016C0199E00F
:10911000D594C794B794A7949A95D1F78091C20239
:109120009091C302813491053CF48091C0029091EA
:10913000C10281349105D4F0D401C30197FE03C06C
:109140000196A11DB11D3C014D0195948794779422
:109150006794D601C501D7FE03C00196A11DB11DBC
:109160005C016D01D594C794B794A7948091DA05FA
:10917000E82FFF27EE0FFF1FED53F94F80819181FC
:109180000190F081E02DF7FF03C0F095E195FF4FCE
:109190007A97A4F0C401B30123E030E040E050E04E
:1091A0000E94537339014A01C601B50123E030E042
:1091B00040E050E00E94537359016A018091FE071C
:1091C000282F332727FD3095432F532F261537059A
:1091D0004805590514F439014A01992787FD9095EE
:1091E000909581959F4FAA2797FDA095BA2F681655
:1091F00079068A069B0614F43C014D012A153B05AD
:109200004C055D0514F459016A01A816B906CA0691
:10921000DB060CF0CFC05C016D01CCC0EA2CFF2452
:1092200000271127CA01B901A80197010E945373B1
:1092300039014A014B895C89CA01AA2797FDA0958B
:10924000BA2F681A790A8A0A9B0AC201B101A801D9
:1092500097010E94537359016A0169897A89CB0188
:10926000AA2797FDA095BA2FA81AB90ACA0ADB0A3D
:10927000D401C30197FE03C00F96A11DB11D3C018F
:109280004D0114E095948794779467941A95D1F7DB
:10929000D601C501D7FE03C00F96A11DB11D5C010B
:1092A0006D01B4E0D594C794B794A794BA95D1F75B
:1092B0008091C2029091C302813491053CF4809167
:1092C000C0029091C10281349105A4F0C401B301A0
:1092D00023E030E040E050E00E94537339014A013E
:1092E000C601B50123E030E040E050E00E94537336
:1092F00059016A018091DA05E82FFF27EE0FFF1F61
:10930000ED53F94F808191810190F081E02DF7FFBD
:1093100003C0F095E195FF4F7A97A4F0C401B30123
:1093200023E030E040E050E00E94537339014A01ED
:10933000C601B50123E030E040E050E00E945373E5
:1093400059016A0171E267167104810491042CF0DD
:10935000A0E26A2E712C812C912C80EE68168FEF82
:1093600078068FEF88068FEF980644F4F0EE6F2EA4
:10937000FFEF7F2EFFEF8F2EFFEF9F2E91E2A916BA
:10938000B104C104D1042CF0E0E2AE2EB12CC12C0A
:10939000D12CA0EEAA16AFEFBA06AFEFCA06AFEF18
:1093A000DA0644F470EEA72E7FEFB72E7FEFC72EBC
:1093B0007FEFD72E80911A0390911B03A0911C037D
:1093C000B0911D0386199709A809B90980931A035A
:1093D00090931B03A0931C03B0931D038091120371
:1093E00090911303A0911403B09115038A199B095E
:1093F000AC09BD098093120390931303A093140347
:10940000B093150380911102909112028F3F910544
:1094100009F008F4CCC5BB85BB2309F056C5809183
:10942000D602882309F051C58091FA02882309F0F9
:109430004CC5E0911706EC87EE2309F446C58091F0
:10944000550790915607A0915707B0915807B7FF5D
:1094500004C081509F4FAF4FBF4FE92EFA2E0B2F04
:10946000112707FD1A95E0925507F09256070093D1
:1094700057071093580780915D0790915E07A09160
:109480005F07B0916007B7FF04C081509F4FAF4F97
:10949000BF4F892F9A2FAB2FBB27A7FDBA958D877A
:1094A0009E87AF87B88B80935D0790935E07A093EC
:1094B0005F07B09360078091F205A82EBB24CC24EF
:1094C000DD2420912A0330912B0340912C035091ED
:1094D0002D03C601B5010E94DF7297FF04C06150E1
:1094E0007F4F8F4F9F4F672E782E892E992487FCB0
:1094F0009A9460922A0370922B0380922C0390928C
:109500002D03209126033091270340912803509189
:109510002903C601B5010E94DF7297FF04C06150A4
:109520007F4F8F4F9F4F272E382E492E552447FCB3
:109530005A94209226033092270340922803509297
:1095400029038091220390912303A0912403B091D9
:109550002503B7FF04C081509F4FAF4FBF4F892FE6
:109560009A2FAB2FBB27A7FDBA9580932203909328
:109570002303A0932403B0932503D801C7018619C0
:109580009709A809B9098093820390938303A09354
:109590008403B093850320911606E22EFF24002752
:1095A0001127BC01CD01A80197010E9453735901F5
:1095B0006A01209392033093930340939403509352
:1095C00095038D859E85AF85B88982199309A40975
:1095D000B5098093860390938703A0938803B09383
:1095E0008903BC01CD01A80197010E945373209308
:1095F0009603309397034093980350939903D601B1
:10960000C501D7FE04C081509F4FAF4FBF4F892F78
:109610009A2FAB2FBB27A7FDBA959093D9028093C1
:10962000D80257FF04C021503F4F4F4F5F4FBB2719
:1096300057FDBA95A52F942F832F9093DB0280932B
:10964000DA028091C2029091C30281349105DCF468
:109650008091C0029091C10281349105A4F480915F
:10966000DA05E82FFF27EE0FFF1FED53F94F80813A
:1096700091810190F081E02DF7FF03C0F095E19515
:10968000FF4F7A97E4F08091FC078F3FC1F48091FF
:10969000D8029091D90297FD019695958795909360
:1096A000D9028093D8028091DA029091DB0297FD73
:1096B0000196959587959093DB028093DA028091CD
:1096C0004A0790914B07A0914C07B0914D07B7FF07
:1096D00004C081509F4FAF4FBF4F892F9A2FAB2FA0
:1096E000BB27A7FDBA9580934A0790934B07A09399
:1096F0004C07B0934D0780913C0790913D07A09196
:109700003E07B0913F07B7FF04C081509F4FAF4F56
:10971000BF4F892F9A2FAB2FBB27A7FDBA958093F8
:109720003C0790933D07A0933E07B0933F0780917D
:109730003A0390913B03A0913C03B0913D032B81F0
:109740003C814D815E81281B390B4A0B5B0B2093BA
:109750007A0330937B0340937C0350937D03809185
:10976000320390913303A0913403B0913503EF801D
:10977000F88409851A85E81AF90A0A0B1B0BE0928E
:109780007E03F0927F030093800310938103209364
:109790008203309383034093840350938503E092C4
:1097A0008603F092870300938803109389038091C6
:1097B000160390911703A0911803B0911903821B0F
:1097C000930BA40BB50B8093160390931703A093F0
:1097D0001803B093190380910E0390910F03A09189
:1097E0001003B09111038E199F09A00BB10B809348
:1097F0000E0390930F03A0931003B0931103FC8505
:10980000FF23E1F02091F8023091F902213831056F
:109810004CF080914E0390914F03019690934F032B
:1098200080934E0320583F4F4CF480914E0390910B
:109830004F03019790934F0380934E031092F902C8
:109840001092F80281E090E090939F0380939E0332
:10985000E0908203F09083030091840310918503CC
:10986000D801C70117FF07C088279927DC018E1987
:109870009F09A00BB10B81509240A040B04034F042
:1098800084E090E090939F0380939E038091A403D3
:109890009091A503A091A603B091A703209155072D
:1098A000309156074091570750915807821B930BF0
:1098B000A40BB50B815E914BAF4FBF4F8F539C49AB
:1098C000A040B04028F08091FD0789310CF4FFC022
:1098D00041E0E41640E1F40640E0040740E01407EC
:1098E0000CF473C08091A003882309F46AC0D801E6
:1098F000C70117FF07C088279927DC018E199F0928
:10990000A00BB10B9C01AD01B7FF04C021503E4F2D
:109910004F4F5F4F69E055954795379527956A9565
:10992000D1F780919E0390919F03820F931F909394
:109930009F0380939E03D801C70117FF03C00796BA
:10994000A11DB11D23E0B595A795979587952A95FB
:10995000D1F78093920390939303A0939403B093D1
:10996000950389589341A040B04064F088E893E1A2
:10997000A0E0B0E08093920390939303A0939403AC
:10998000B0939503209192033091930340919403F7
:109990005091950357FF04C021503F4F4F4F5F4FE9
:1099A000232F342F452F552747FD5A958091D802F4
:1099B0009091D902820F931F9093D9028093D8027D
:1099C00006C081E08093A00302C01092A00360E073
:1099D000E61660EFF6066FEF06076FEF16070CF05E
:1099E00073C08091A103882309F46AC0D801C7011C
:1099F00017FF07C088279927DC018E199F09A00B44
:109A0000B10B9C01AD01B7FF04C021503E4F4F4F39
:109A10005F4FF9E05595479537952795FA95D1F71A
:109A200080919E0390919F03820F931F90939F03B9
:109A300080939E03D801C70117FF03C00796A11D9D
:109A4000B11DE3E0B595A79597958795EA95D1F770
:109A50008093920390939303A0939403B093950300
:109A600088579C4EAF4FBF4F64F488E79CEEAFEF32
:109A7000BFEF8093920390939303A0939403B093CA
:109A80009503209192033091930340919403509158
:109A9000950357FF04C021503F4F4F4F5F4F232F77
:109AA000342F452F552747FD5A958091D802909124
:109AB000D902820F931F9093D9028093D80211C0CC
:109AC00081E08093A1030DC01092A1030AC01092FF
:109AD0009F0310929E0388EE93E09093B8018093C9
:109AE000B7018C85282F332780919E0390919F0387
:109AF0002817390724F430939F0320939E03109175
:109B0000FD07112379F0212F332727FD3095809110
:109B10009E0390919F032817390724F430939F03E5
:109B200020939E03409182035091830360918403AC
:109B300070918503413851056105710574F080917C
:109B400052039091530320919E0330919F03820F03
:109B5000931F909353038093520340585F4F6F4F6E
:109B60007F4F74F4809152039091530320919E0390
:109B700030919F03821B930B909353038093520366
:109B800081E090E090939F0380939E03C0908603B2
:109B9000D0908703E0908803F0908903D701C60135
:109BA000F7FE07C088279927DC018C199D09AE09AB
:109BB000BF0981509240A040B04034F084E090E072
:109BC00090939F0380939E031092960310929703A5
:109BD00010929803109299038091A8039091A90381
:109BE000A091AA03B091AB0320915D0730915E076D
:109BF00040915F0750916007821B930BA40BB50B3C
:109C0000815E914BAF4FBF4F8F539C49A040B040F6
:109C100018F019310CF4FFC001E0C01600E1D006C5
:109C200000E0E00600E0F0060CF473C08091A203AF
:109C3000882309F46AC0D701C601F7FE07C0882748
:109C40009927DC018C199D09AE09BF099C01AD0162
:109C5000B7FF04C021503E4F4F4F5F4F69E055950D
:109C60004795379527956A95D1F780919E039091F6
:109C70009F03820F931F90939F0380939E03D701AE
:109C8000C601F7FE03C00796A11DB11D23E0B595DF
:109C9000A795979587952A95D1F7809396039093EA
:109CA0009703A0939803B093990389589341A040D8
:109CB000B04064F088E893E1A0E0B0E080939603C0
:109CC00090939703A0939803B093990320919603E0
:109CD00030919703409198035091990357FF04C026
:109CE00021503F4F4F4F5F4F232F342F452F552784
:109CF00047FD5A958091DA029091DB02820F931F03
:109D00009093DB028093DA0206C081E08093A20385
:109D100002C01092A20320E0C21620EFD2062FEF5D
:109D2000E2062FEFF2060CF073C08091A3038823A4
:109D300009F46AC0D701C601F7FE07C08827992732
:109D4000DC018C199D09AE09BF099C01AD01B7FF6B
:109D500004C021503E4F4F4F5F4F09E05595479546
:109D6000379527950A95D1F780919E0390919F038F
:109D7000820F931F90939F0380939E03D701C60188
:109D8000F7FE03C00796A11DB11D13E0B595A79579
:109D9000979587951A95D1F780939603909397039B
:109DA000A0939803B093990388579C4EAF4FBF4F31
:109DB00064F488E79CEEAFEFBFEF80939603909337
:109DC0009703A0939803B093990320919603309141
:109DD0009703409198035091990357FF04C0215075
:109DE0003F4F4F4F5F4F232F342F452F552747FDB0
:109DF0005A958091DA029091DB02820F931F909323
:109E0000DB028093DA0211C081E08093A3030DC0CE
:109E10001092A3030AC010929F0310929E0388EE33
:109E200093E09093B8018093B7014C85242F33279A
:109E300080919E0390919F032817390724F4309353
:109E40009F0320939E038091FD07882379F0282F9C
:109E5000332727FD309580919E0390919F0328170B
:109E6000390724F430939F0320939E034091860387
:109E7000509187036091880370918903413851059F
:109E80006105710574F08091500390915103209108
:109E90009E0330919F03820F931F909351038093F1
:109EA000500340585F4F6F4F7F4FCCF48091500369
:109EB0009091510320919E0330919F03821B930B3D
:109EC00090935103809350030AC01092DB021092CA
:109ED000DA021092D9021092D8021092FA028091FE
:109EE0006207882341F41092DB021092DA0210928A
:109EF000D9021092D8028091550790915607A091EF
:109F00005707B09158078093A4039093A503A0939B
:109F1000A603B093A70380915D0790915E07A0917F
:109F20005F07B09160078093A8039093A903A09363
:109F3000AA03B093AB0310922A0310922B03109242
:109F40002C0310922D0310922603109227031092D7
:109F500028031092290310922203109223031092D7
:109F60002403109225031092550710925607109261
:109F700057071092580710925D0710925E071092D3
:109F80005F071092600710924A0710924B071092D9
:109F90004C0710924D0710923C0710923D0710920B
:109FA0003E0710923F071092120210921102E090A9
:109FB000E802F090E902C701F7FE04C0882799275C
:109FC0008E199F0940976CF088EE93E09093B8014A
:109FD0008093B7018091E30584FD03C081E0809305
:109FE00091031091EF05A12EBB24CC24DD24B701F1
:109FF000882777FD8095982F9701F7FE04C02227C8
:10A0000033272E193F09442737FD4095542F0E94CE
:10A01000DF729B01AC01C601B5010E94DF7297FFA0
:10A0200004C061507E4F8F4F9F4FE9E09595879513
:10A0300077956795EA95D1F79B01812F99278E9D9A
:10A04000D0018F9DB00D9E9DB00D1124CD01B7FDA7
:10A0500003969595879595958795280F391F4427E1
:10A0600037FD4095542F2093760330937703409328
:10A0700078035093790380910A0390910B03A09188
:10A080000C03B0910D03821B930BA40BB50B8093B3
:10A090000A0390930B03A0930C03B0930D03815517
:10A0A000934CA040B04064F080E593ECA0E0B0E0B9
:10A0B00080930A0390930B03A0930C03B0930D03BA
:10A0C00080910A0390910B03A0910C03B0910D03B2
:10A0D000805B9C43AF4FBF4F64F480EB9CE3AFEFDA
:10A0E000BFEF80930A0390930B03A0930C03B093EC
:10A0F0000D0340900003509001034114510409F4F2
:10A1000088C18091E30583FF84C180913A039091D7
:10A110003B03A0913C03B0913D03B7FF04C08150C5
:10A120009E4FAF4FBF4F69E0B595A795979587951F
:10A130006A95D1F76C0197FF04C0D094C194D108FF
:10A14000D3948091320390913303A0913403B09162
:10A150003503B7FF04C081509E4FAF4FBF4F59E04A
:10A16000B595A795979587955A95D1F7BC0197FF17
:10A1700003C0709561957F4FC616D7060CF46B012E
:10A18000B601D7FE02C0695F7F4F3B0143E0759483
:10A1900067944A95E1F70894611C711C3CE1E32E39
:10A1A00032E0F32E4E0C5F1C72010027F7FC009585
:10A1B000102F24EE3DEF420E531E80918B0790919D
:10A1C0008C07A0918D07B0918E078090930190909D
:10A1D0009401A0909501B0909601BC01CD01A5011C
:10A1E00094010E945373E21AF30A040B150BC80181
:10A1F000B70128E631E040E050E00E945373DC01F3
:10A20000CB018C01045B10408091840790918507FD
:10A2100097FF03C0909581959F4F8138910514F069
:10A2200000E010E0E090B701F090B801E114F10413
:10A2300089F539E1C316D1046CF58091F80290914B
:10A24000F902800F911F9093F9028093F802809198
:10A2500091038823F9F0C201AA2797FDA095BA2F90
:10A26000BC01CD01A50194010E94DF72DC01CB018C
:10A2700080938B0790938C07A0938D07B0938E07E4
:10A28000BC01CD010E9453733093FF022093FE0264
:10A2900010929103C80123E0880F991F2A95E1F7D6
:10A2A000B3010E941E73CB01AA2797FDA095BA2F78
:10A2B00020918B0730918C0740918D0750918E072C
:10A2C000280F391F4A1F5B1F20938B0730938C0781
:10A2D00040938D0750938E071091A801612F772727
:10A2E000C69EC001C79E900DD69E900D112497FD6D
:10A2F0004F966C0185E0D594C7948A95E1F76C1967
:10A300007D096B0177FD7FC0E114F10409F073C092
:10A31000E090C202F090C3028091C0029091C1020D
:10A32000E80EF91EF7FE04C067E070E0E60EF71EC7
:10A3300003E0F594E7940A95E1F780E490E0E80EF5
:10A34000F91ECA01B901A50194010E945373DA01F3
:10A35000C9012091FE023091FF02442737FD40954C
:10A36000542F821B930BA40BB50B845E9D4FAF4FF4
:10A37000BF4FBC01CD0128E631E040E050E00E9433
:10A380005373DC01CB01845B90408C9DD0018D9D8B
:10A39000B00D9C9DB00D1124CD01B7010E941E731C
:10A3A00083E0189F60011124C616D70614F4B60185
:10A3B00008C0882799278C199D09681779070CF41C
:10A3C000BC019B01442737FD4095542F80910A031F
:10A3D00090910B03A0910C03B0910D03820F931F7A
:10A3E000A41FB51F80930A0390930B03A0930C0343
:10A3F000B0930D030EC00894E108F108F092B80183
:10A40000E092B70106C084EF91E09093B801809389
:10A41000B701809190038150809390038F3F09F0A2
:10A42000DCC088E1809390038091F2059927880F22
:10A43000991F880F991F7C010027F7FC0095102FAA
:10A4400080913A0390913B03A0913C03B0913D036E
:10A45000BC01CD01A80197010E9453733093870579
:10A46000209386058091320390913303A0913403A9
:10A47000B0913503BC01CD01A80197010E9453732F
:10A48000309389052093880580917F0790918007FC
:10A4900097FD0396959587959595879590938B0550
:10A4A00080938A0580918F079091900797FD03967E
:10A4B000959587959595879590938D0580938C05B7
:10A4C000809184079091850790938F0580938E05E6
:10A4D0008091E0029091E102A091E202B091E3024A
:10A4E000BC01CD0125E030E040E050E00E94537314
:10A4F00030939105209390058091C9059091CA05EC
:10A5000090939305809392055092970540929605FB
:10A5100080911D0190911E0190939905809398055B
:10A520008091EE02992790939B0580939A058091E4
:10A530008B0790918C07A0918D07B0918E07209189
:10A540009301309194014091950150919601BC0185
:10A55000CD010E94537330939D0520939C058091FB
:10A560001302909114029093AB058093AA058091F9
:10A57000330499279093AD058093AC058091FA013F
:10A580009091FB019093AF058093AE0580910108F7
:10A59000909102089093B3058093B20580910508CD
:10A5A000909106089093B5058093B4058091FF07BC
:10A5B00099279093C1058093C0058091D103909114
:10A5C000D2039093C3058093C2058091CF039091ED
:10A5D000D0039093C5058093C4058091FA02882327
:10A5E00081F0109272031092730310927403109210
:10A5F000750310926E0310926F0310927003109205
:10A600007103F090D702FF20F1F480916207282FA8
:10A6100033274427552780913A0390913B03A0911B
:10A620003C03B0913D03BC01CD010E94DF72DC010F
:10A63000CB01BC01CD0128EF3AE240E050E00E949E
:10A640005373490102C088249924E090D602EE2079
:10A65000F1F480916207282F3327442755278091F2
:10A66000320390913303A0913403B0913503BC01C0
:10A67000CD010E94DF72DC01CB01BC01CD0128EFCE
:10A680003AE240E050E00E945373390102C0662470
:10A6900077248091360790913707893C91051CF00B
:10A6A00088EC90E005C088539F4F34F488E39FEF17
:10A6B0009093370780933607809141079091420726
:10A6C000893C91051CF088EC90E005C088539F4FB1
:10A6D00034F488E39FEF9093420780934107809181
:10A6E000430790914407AA2797FDA095BA2F209180
:10A6F0008907A22EBB24CC24DD24BC01CD01A601F8
:10A7000095010E94DF729B01AC0180913607909108
:10A710003707AA2797FDA095BA2FE7E0880F991F62
:10A72000AA1FBB1FEA95D1F7280F391F4A1F5B1FCD
:10A7300057FF04C0215C3F4F4F4F5F4F76E0559568
:10A740004795379527957A95D1F78401020F131F06
:10A750001093440700934307809134079091350785
:10A76000AA2797FDA095BA2FBC01CD01A60195019E
:10A770000E94DF729B01AC018091410790914207DA
:10A78000AA2797FDA095BA2F67E0880F991FAA1FE7
:10A79000BB1F6A95D1F7280F391F4A1F5B1F57FF50
:10A7A00004C0215C3F4F4F4F5F4F96E05595479552
:10A7B000379527959A95D1F72301420E531E509253
:10A7C0003507409234078091840790918507880F60
:10A7D000991FAA2797FDA095BA2F20913B073327F1
:10A7E00044275527BC01CD010E94DF725B016C013B
:10A7F00097FF08C02FE330E040E050E0A20EB31E08
:10A80000C41ED51E86E0D594C794B794A7948A95A4
:10A81000D1F780915207282F33274427552780915D
:10A820001E0390911F03A0912003B0912103BC014E
:10A83000CD010E94DF72DC01CB01BC01CD0120EF14
:10A8400035E540E050E00E945373B501620F731F7D
:10A8500070938507609384070150104434F080E0C2
:10A8600090E490934407809343078091430790912D
:10A8700044078050904C34F480E090EC909344076F
:10A880008093430751E0451650E4550634F080E0CC
:10A8900090E490933507809334078091340790912A
:10A8A00035078050904C34F480E090EC909335075D
:10A8B000809334076150704434F080E090E49093CA
:10A8C0008507809384078091840790918507805045
:10A8D000904C34F480E090EC90938507809384074B
:10A8E00080910001482F552780911D0190911E01F4
:10A8F0004817590794F420911D0130911E010981D8
:10A900001A81049FC001059F900D149F900D112482
:10A91000B9010E940A737A83698329813A81220FDF
:10A92000331F220F331F3A8329834091E30540FFF1
:10A9300033C6EE2009F030C6FF2009F02DC6AA2448
:10A94000BB248091B0039091B1039093B1058093A3
:10A95000B00580911302909114029093AB058093FF
:10A96000AA0520915403309155032115310509F0B2
:10A970003FC080911301909114018959934058F080
:10A9800087B5853F20F480911502815011C081E088
:10A990008093B9034EC080911301909114018436C5
:10A9A000910508F587B58B30D0F0809115028F5F47
:10A9B000809315029AE08902900111248091D305B9
:10A9C000821B87BD8CE291E09093FF018093FE0192
:10A9D0008EE591E090935503809354032AC081E063
:10A9E0008093B80326C0F092B803F092B90321C057
:10A9F0008091E0029091E102A091E202B091E30225
:10AA000014E0880F991FAA1FBB1F1A95D1F78093D6
:10AA1000160290931702A0931802B0931902B092F5
:10AA20001402A0921302215030403093550320931A
:10AA300054032091AB0141FF24C02233D8F480910C
:10AA4000BF0181508093BF018F3FD9F51092FB0267
:10AA50008091E0029091E102A091E202B091E302C4
:10AA60008093DC029093DD02A093DE02B093DF02BC
:10AA700081E004C081E08093FB0288EC8093BF01F9
:10AA800020C08091970190919801820F911D209193
:10AA9000E8053327829FA001839F500D929F500DA0
:10AAA0001124CA01AA2797FDA095BA2F8093DC0232
:10AAB0009093DD02A093DE02B093DF0281E08093E9
:10AAC000FB0280913A0390913B03A0913C03B0912B
:10AAD0003D03E0909301F090940100919501109155
:10AAE0009601BC01CD01A80197010E945373590141
:10AAF0006A018091320390913303A0913403B091A5
:10AB00003503BC01CD01A80197010E945373B9011F
:10AB1000C5010E94D7708C01CC9714F00CE310E0B3
:10AB2000C8010E9458658C0180E280939201809157
:10AB3000FB02882309F4BCC38091BD0299279C01C4
:10AB40002071307084FDB4C36091360660FD04C08E
:10AB50008091E30581FD07C0C980DA803093AD03A1
:10AB60002093AC0385C18091BD0281FF5DC14091FE
:10AB7000BB015091BC01CA010F962091E6023091B1
:10AB8000E70282179307ACF58091B803882389F513
:10AB90008091BA0381FF13C08D7F8093BA038091A7
:10ABA000E0029091E102A091E202B091E302809371
:10ABB000DC029093DD02A093DE02B093DF0280916D
:10ABC000BA0381608093BA03241B350B2F503040A9
:10ABD00037FF03C0309521953F4F8091AC03909192
:10ABE000AD03820F931F9093AD038093AC038BE270
:10ABF00062C0CA010F9728173907ACF58091B903D5
:10AC0000882389F58091BA0380FF13C08E7F8093DB
:10AC1000BA038091E0029091E102A091E202B0912A
:10AC2000E3028093DC029093DD02A093DE02B093F6
:10AC3000DF028091BA0382608093BA03241B350B34
:10AC4000215F3F4F37FF03C0309521953F4F8091E3
:10AC5000AC039091AD03821B930B9093AD03809353
:10AC6000AC038DE228C02091BA03822F992783700C
:10AC70009070892BF9F02C7F2093BA031092AD03CA
:10AC80001092AC038091E0029091E102A091E20267
:10AC9000B091E3028093DC029093DD02A093DE0288
:10ACA000B093DF0261FF06C084EF91E09093FF0153
:10ACB0008093FE018DE3809392012091AC0330914B
:10ACC000AD03C90137FF04C088279927821B930B66
:10ACD000815092400CF491C08091E8059927289FFB
:10ACE000B001299F700D389F700D1124CB0160E0D9
:10ACF00075E00E941E73CB01AA2797FDA095BA2F7D
:10AD00002091DC023091DD024091DE025091DF02A1
:10AD1000280F391F4A1F5B1F2093DC023093DD028E
:10AD20004093DE025093DF021092AD031092AC0309
:10AD3000C090E002D090E102E090E202F090E302E5
:10AD4000D701C60180509440A040B04082179307BD
:10AD5000A407B5075CF4D701C60180509C4FAF4FE4
:10AD6000BF4F281739074A075B0744F08093DC027E
:10AD70009093DD02A093DE02B093DF02809136064D
:10AD800081FF06C08BE490E09093FF018093FE0169
:10AD90008091EC05882389F54091B0035091B1036F
:10ADA00057FF02C04D5F5F4F5595479555954795A5
:10ADB00080911D0190911E01209100013327489F31
:10ADC000D001499FB00D589FB00D1124CD01B9019C
:10ADD0000E941E737093BC016093BB0166347105C1
:10ADE0001CF486E490E005C06739710534F086E90B
:10ADF00090E09093BC018093BB01809154039091AB
:10AE00005503892B89F18091E0029091E102A09194
:10AE1000E202B091E3028093DC029093DD02A09302
:10AE2000DE02B093DF0220C08091E0029091E10247
:10AE3000A091E202B091E30280599140A040B0405D
:10AE40008093DC029093DD02A093DE02B093DF02D8
:10AE50008091EC05882311F0992702C088E790E0E3
:10AE60009093BC018093BB01C090B003D090B1031C
:10AE70002090E0023090E1024090E2025090E30224
:10AE80002091DC023091DD024091DE025091DF0220
:10AE9000221533054405550524F08091360680FDC2
:10AEA00049C28091540390915503892B39F0C09089
:10AEB000B003D090B103AA24BB24E2C0D201C101E7
:10AEC000821B930BA40BB50B80937A0390937B03A7
:10AED000A0937C03B0937D038230E0E89E07EFEF00
:10AEE000AE07EFEFBE072CF481E090E8AFEFBFEFC5
:10AEF00009C08F5F9F47A040B04064F08FEF9FE78D
:10AF0000A0E0B0E080937A0390937B03A0937C034E
:10AF1000B0937D03A0907A03B0907B038091AA0147
:10AF2000282F33274427552780917A0390917B035C
:10AF3000A0917C03B0917D03BC01CD010E94DF7222
:10AF400097FF04C0615F7F4F8F4F9F4FE4E095955F
:10AF5000879577956795EA95D1F760937A03709313
:10AF60007B0380937C0390937D0365302CEF720705
:10AF70002FEF82072FEF92072CF484E09CEFAFEFC6
:10AF8000BFEF09C06C5F73408040904064F08CEF6D
:10AF900093E0A0E0B0E080937A0390937B03A093CA
:10AFA0007C03B0937D0380917A0390917B03C81A50
:10AFB000D90A209113023091140237FF02C0295F91
:10AFC0003F4F53E0359527955A95E1F74FEF2C34D5
:10AFD00034071CF42BE43FEF05C0253B310514F08A
:10AFE00025EB30E0C9012830310514F088E090E00D
:10AFF000889FA001899F500D989F500D112418160D
:10B00000190654F4CA0157FD0396959587959595B1
:10B010008795280F391F09C0CA0157FD03969595DA
:10B02000879595958795281B390BC901AA2797FD08
:10B03000A095BA2F2091AC01332744275527BC0196
:10B04000CD010E94DF7297FF04C061587F4F8F4F80
:10B050009F4FA7E09595879577956795AA95D1F726
:10B060009B015FEF613875071CF420E83FEF06C0D5
:10B070006F3F710519F014F020E031E0C21AD30AD5
:10B080002090020330900303409004035090050386
:10B0900057FE08C06FE770E080E090E0260E371E94
:10B0A000481E591EF7E05594479437942794FA9513
:10B0B000D1F78091A901282F332744275527C201B2
:10B0C000B1010E94DF7297FF04C0615E7F4F8F4F16
:10B0D0009F4FE5E09595879577956795EA95D1F728
:10B0E00060937A0370937B0380937C0390937D033A
:10B0F0006138AFEF7A07AFEF8A07AFEF9A072CF40A
:10B1000080E89FEFAFEFBFEF0AC06F3F7105810589
:10B11000910569F064F080E091E0A0E0B0E08093F8
:10B120007A0390937B03A0937C03B0937D0380917B
:10B130007A0390917B03C81AD90A8091A701282F1E
:10B14000332780910008992787FD9095289FF0016B
:10B15000299FF00D389FF00D11249F01F7FF02C0C9
:10B1600021583F4F220F232F221F330BFFEF21388F
:10B170003F071CF420E83FEF06C02F3F310519F0D0
:10B1800014F020E031E0C21AD30A65E9E62EF12C72
:10B19000AE0CBF1C2BE2A21621E0B206E0F48091B7
:10B1A000AC039091AD03892BB1F48091B0039091E1
:10B1B000B103181619067CF48091B2039091B30381
:10B1C0008C159D053CF48091BD019091BE01C8167F
:10B1D000D9060CF06C01C601AA2797FDA095BA2FDD
:10B1E0005DE0880F991FAA1FBB1F5A95D1F79801E0
:10B1F000442737FD4095542FBC01CD010E94537365
:10B2000020937E0330937F03409380035093810308
:10B21000C0907E03D0907F038091AE039091AF03E6
:10B220009C01220F331F280F391F2C0D3D1D37FFA6
:10B2300002C02D5F3F4FA9015595479555954795FC
:10B240005093AF034093AE038091E405282F33273A
:10B25000220F331F220F331F241735076CF4809100
:10B260008307282F3327220F331F220F331F205528
:10B2700030404217530724F03093AF032093AE03BE
:10B280008091360680FF0DC08091AE039091AF0390
:10B2900049815A818417950724F05093AF03409356
:10B2A000AE036091AE037091AF037A83698342C0AD
:10B2B0008091EC05882301F56091B0037091B10392
:10B2C00077FF02C06D5F7F4F7595679575956795A0
:10B2D00040911D0150911E0180910001282F3327BC
:10B2E000649FC001659F900D749F900D1124B9015A
:10B2F0000E941E73CB0101C099279093BC018093DB
:10B30000BB018091BB019091BC01873491051CF475
:10B3100086E490E005C08639910534F086E990E036
:10B320009093BC018093BB0189819A819093AF0374
:10B330008093AE038091BD0281FF2EC18091BD023A
:10B3400084FD2AC18091B4039091B503A091B60306
:10B35000B091B7030097A105B105B1F4E981FA8175
:10B36000CF01AA2797FDA095BA2FECE0880F991F6F
:10B37000AA1FBB1FEA95D1F78093B4039093B5033E
:10B38000A093B603B093B703809113029091140277
:10B39000809113029091140297FF03C090958195BC
:10B3A0009F4F843691050CF0F7C0E980FA80C70101
:10B3B000AA2797FDA095BA2F9801442737FD4095FD
:10B3C000542FBC01CD010E94DF72DC01CB018093C0
:10B3D0007E0390937F03A0938003B0938103B7FF14
:10B3E00004C08150904EAF4FBF4F7C018D017DE076
:10B3F00015950795F794E7947A95D1F7E0927E0337
:10B40000F0927F0300938003109381038091BE022A
:10B410009091BF0227E0803D9207F8F48091B40339
:10B420009091B503A091B603B091B7039C01AD0113
:10B4300069E056954795379527956A95D1F7821B10
:10B44000930BA40BB50BA801970113E0220F331F38
:10B45000441F551F1A95D1F722C03FE0803A930749
:10B4600058F58091B4039091B503A091B603B091C3
:10B47000B7039C01AD01FAE056954795379527959E
:10B48000FA95D1F7821B930BA40BB50BA80197017A
:10B49000E2E0220F331F441F551FEA95D1F7820FB8
:10B4A000931FA41FB51F8093B4039093B503A0937B
:10B4B000B603B093B7033CC02091B4033091B503F9
:10B4C0004091B6035091B70380549F41C0F4DA0114
:10B4D000C9017BE0B695A795979587957A95D1F7A1
:10B4E000281B390B4A0B5B0BD801C7018E0D9F1D22
:10B4F000A01FB11F280F391F4A1F5B1F11C0DA019F
:10B50000C9016CE0B695A795979587956A95D1F78F
:10B51000281B390B4A0B5B0B2E0D3F1D401F511F83
:10B520002093B4033093B5034093B6035093B7030D
:10B530008091B4039091B503A091B603B091B70385
:10B540005CE0B695A795979587955A95D1F7909316
:10B55000B1038093B0034091EA05442399F0552745
:10B560009C01BA010E941E73C901861B970B909320
:10B57000B3038093B203260F371F3093BE0120938D
:10B58000BD010AC01092B3031092B2038FEF93E093
:10B590009093BE018093BD0130904807232D33273F
:10B5A000C901880F991F880F991F8896A981BA81B0
:10B5B0008A179B0714F09A83898340908307842D10
:10B5C0009927880F991F880F991F80559040E9810E
:10B5D000FA818E179F0714F49A838983809147021A
:10B5E0008823A1F08091BE029091BF020297C0977C
:10B5F00068F4E980FA801E141F0444F481E090E0AE
:10B600009093BF028093BE023A83298309811A81F5
:10B61000109395050093940580917603909177039C
:10B62000A0917803B091790312E0880F991FAA1FA7
:10B63000BB1F1A95D1F70091840710918507081B4D
:10B64000190B29813A81213A31058CF0C90137FD66
:10B65000019695958795801791070CF48C0190952C
:10B6600081959F4F081719076CF48C010BC00135A9
:10B67000110514F000E510E03FEF003B130714F450
:10B6800000EB1FEF242D3327220F331F220F331F10
:10B69000C90149815A81841B950B801791070CF4CD
:10B6A0008C0169817A81621B730B061717070CF4F2
:10B6B0008B0180914307909144076091EC02709157
:10B6C000ED02861B970B9093540780935307D090FD
:10B6D000620720916E0330916F0340917003509187
:10B6E0007103DD2041F0861A970AC401AA2797FD4D
:10B6F000A095BA2F04C0AA2797FDA095BA2F280FAE
:10B70000391F4A1F5B1F20936E0330936F034093D2
:10B7100070035093710380916E0390916F03A09119
:10B720007003B091710381509A4FA040B04064F013
:10B7300080E09AEFA0E0B0E080936E0390936F03F7
:10B74000A0937003B093710380916E0390916F0387
:10B75000A0917003B091710380509640AF4FBF4FDE
:10B7600064F480E096E0AFEFBFEF80936E039093B8
:10B770006F03A0937003B09371038090AD0190901C
:10B78000AE019401442737FD4095542F80916E03FC
:10B7900090916F03A0917003B0917103BC01CD0132
:10B7A0000E945373E0905307F0905407E20EF31E8B
:10B7B000B09099016B2D772788279927980117FF5B
:10B7C00004C022273327201B310B37FF02C02F5F15
:10B7D0003F4F3595279549815A81240F351F4427BE
:10B7E00037FD4095542F0E94DF7297FF04C0615CC3
:10B7F0007F4F8F4F9F4F56E095958795779567952B
:10B800005A95D1F79B016E157F050CF47B0130959D
:10B8100021953F4FE216F3060CF47901809134072D
:10B82000909135076091EA027091EB02861B970BAD
:10B830009093330780933207209172033091730302
:10B840004091740350917503DD2041F0661A770A28
:10B85000C301AA2797FDA095BA2F04C0AA2797FD78
:10B86000A095BA2F280F391F4A1F5B1F2093720320
:10B870003093730340937403509375038091720364
:10B8800090917303A0917403B091750381509A4F06
:10B89000A040B04064F080E09AEFA0E0B0E0809378
:10B8A000720390937303A0937403B0937503809114
:10B8B000720390917303A0917403B091750380504B
:10B8C0009640AF4FBF4F64F480E096E0AFEFBFEF1C
:10B8D0008093720390937303A0937403B0937503E2
:10B8E0009401442737FD4095542F80917203909125
:10B8F0007303A0917403B0917503BC01CD010E9444
:10B900005373C0903207D0903307C20ED31E6B2DF5
:10B91000772788279927980117FF04C02227332704
:10B92000201B310B37FF02C02F5F3F4F3595279506
:10B93000A981BA812A0F3B1F442737FD4095542F18
:10B940000E94DF7297FF04C0615C7F4F8F4F9F4F53
:10B9500036E095958795779567953A95D1F79B0150
:10B960006C157D050CF46B01309521953F4FC21687
:10B97000D3060CF4690122E9622E26E0722E94E4CB
:10B98000A92E96E0B92E8BE0582EB3E68B2EB7E0A9
:10B990009B2EF501258512160CF0ABC049815A810A
:10B9A000CA01AA2797FDA095BA2F332727FD309506
:10B9B000432F532FBC01CD010E94DF7297FF04C0BB
:10B9C000615C7F4F8F4F9F4FA6E095958795779548
:10B9D0006795AA95D1F77C8B6B8BC701AA2797FD3A
:10B9E000A095BA2FF5012685332727FD3095432FE3
:10B9F000532FBC01CD010E94DF7297FF04C0615C30
:10BA00007F4F8F4F9F4FF6E0959587957795679578
:10BA1000FA95D1F72B893C89260F371F3C8B2B8B4E
:10BA2000C601AA2797FDA095BA2FF50127853327D0
:10BA300027FD3095432F532FBC01CD010E94DF72AB
:10BA400097FF04C0615C7F4F8F4F9F4FE6E0959555
:10BA5000879577956795EA95D1F72B893C89260FCD
:10BA6000371F3C8B2B8BC801AA2797FDA095BA2FB7
:10BA7000F5012089332727FD3095432F532FBC0133
:10BA8000CD010E94DF72DC01CB01B7FF03C0CF966E
:10BA9000A11DB11D76E0B595A795979587957A95E7
:10BAA000D1F7F401608171812B893C89820F931F4A
:10BAB0000E948232D4018D939C9397FD03969595B5
:10BAC0008795959587959C8B8B8B832D9927EB89F3
:10BAD000FC898E179F073CF4842D99272B893C897C
:10BAE0002817390714F09C8B8B8BEB89D301EC93CF
:10BAF00002C0D3011C925A94E2E0F0E08E0E9F1E29
:10BB000024E030E0A20EB31E620E731E57FE41CF3A
:10BB1000E2E1CC5E0C948A738091C7039091C803D4
:10BB2000A091C903B091CA038093BF039093C0034F
:10BB3000A093C103B093C2038091C3039091C40347
:10BB4000A091C503B091C6038093BB039093BC033F
:10BB5000A093BD03B093BE0308951092D203109238
:10BB6000D1031092D0031092CF03089584B1806A5C
:10BB700084B93D9A82E58CBD1DBC459A81E08093D5
:10BB800095078AEA8093A50783E88093A6078AE051
:10BB90008093A7071092A9071092A8071092AB07ED
:10BBA0001092AA071092FF071092C70708953091CC
:10BBB0009507332309F085C00DB407FE82C084E0E9
:10BBC0008093FD01459A2EB58091D5039927813048
:10BBD000910589F0823091051CF4892B21F03EC03B
:10BBE0000297B9F03BC03093C6072093D6032138A3
:10BBF000A9F581E008C0253549F48091D603820F6C
:10BC00008093D60382E08093D50328C03093D50378
:10BC100025C08091C607E82FFF27EE51F84F2083FB
:10BC20008F5F8093C6079091D6038A31A0F02917C1
:10BC300069F48AE1A2EEB7E0E8ECF7E00D9001923A
:10BC40008A95E1F781E08093C70702C03093C70768
:10BC50001092D50303C0920F9093D6032091A407AE
:10BC6000203208F028C045980000000000000000C5
:10BC700000000000000000000000000000000000C4
:10BC800000000000000000000000000000000000B4
:10BC90000000000000000000E0919D07F0919E0769
:10BCA000E20FF11D80818EBD8091C4079081890FC4
:10BCB0008093C40703C081E0809395072F5F209392
:10BCC000A4070895EF92FF920F931F938091F205BE
:10BCD0009927880F991F880F991F7C010027F7FC6F
:10BCE0000095102F80913A0390913B03A0913C0363
:10BCF000B0913D03BC01CD01A80197010E9453738F
:10BD00003093A9072093A8078091320390913303C1
:10BD1000A0913403B0913503BC01CD01A801970176
:10BD20000E9453733093AB072093AA0720918B078F
:10BD300030918C0740918D0750918E07DA01C9012F
:10BD4000E3E0880F991FAA1FBB1FEA95D1F7820F66
:10BD5000931FA41FB51F820F931FA41FB51F20910F
:10BD60009301309194014091950150919601BC014D
:10BD7000CD010E9453733093B1072093B007E09137
:10BD80004403F091450380915A0790915B07BF01EE
:10BD90000E941E73CB019B01220F331F220F331F02
:10BDA000280F391F280F391F37FF02C02D5F3F4F63
:10BDB00035952795359527953093AD072093AC079A
:10BDC0008091870790918807BF010E941E739B0195
:10BDD000220F331F220F331F260F371F260F371F47
:10BDE00037FF02C02D5F3F4F359527953595279535
:10BDF0003093AF072093AE0710924503109244038F
:10BE000010925B0710925A071092880710928707CA
:10BE10008091A70799278D30910509F460C08E3075
:10BE200091055CF48B30910509F488C08C30910544
:10BE30000CF009C10A9761F08AC18F30910509F4AD
:10BE40005EC18F3091050CF44AC1409769F17FC102
:10BE50008091D1028093B8078091D0028093B90776
:10BE60008091CF028093BA078091CE028093BB0766
:10BE70008091CD028093BC078091CC028093BD0756
:10BE80008091CB028093BE078091CA028093BF0746
:10BE90008091BD028093C0078091BD02837F809313
:10BEA000BD020E949F2D51C180910108909102080E
:10BEB0009093B9078093B807809105089091060880
:10BEC0009093BB078093BA0780911D0190911E014A
:10BED0008093BC07809100018093BD0738C1809199
:10BEE00023068093B807809124068093B907809138
:10BEF00025068093BA07809126068093BB07809120
:10BF000027068093BC0780912B068093BD07809104
:10BF10002C068093BE0780912D068093BF078091E9
:10BF200030068093C00780912E068093C1078091D0
:10BF30002F068093C20780913106CEC0F89480917D
:10BF4000D905E82FFF27EE0FFF1FED53F94F0190A2
:10BF5000F081E02DE038F1051CF0EFE7F0E006C0DD
:10BF60002FEFE138F20714F4E1E8FFEFE093B807B0
:10BF70008091DA05E82FFF27EE0FFF1FED53F94FF1
:10BF80000190F081E02DE038F1051CF0EFE7F0E0E2
:10BF900006C06FEFE138F60714F4E1E8FFEFE09335
:10BFA000B9078091D805E82FFF27EE0FFF1FED534B
:10BFB000F94F0190F081E02DE038F1051CF0EFE73A
:10BFC000F0E006C08FEFE138F80714F4E1E8FFEF86
:10BFD000E093BA078091D705E82FFF27EE0FFF1FE8
:10BFE000ED53F94F0190F081E02DE038F1051CF0A0
:10BFF000EFE7F0E006C02FEFE138F20714F4E1E8D4
:10C00000FFEF7894E093BB078091EF028093BC0729
:10C010008091F0028093BD078091F1028093BE076A
:10C020008091F2028093BF078091F3028093C00752
:10C030008091F4028093C1078091F5028093C2073A
:10C040008091F60249C080913304863018F0109236
:10C05000330485E08093B807809132068093B90756
:10C0600080919005909191059093BB078093BA07BA
:10C070008091DC029091DD02A091DE02B091DF029E
:10C08000BC01CD0125E030E040E050E00E94537358
:10C090003093BD072093BC07809128068093BE078C
:10C0A000809129068093BF0780912A068093C0075C
:10C0B0008091EE028093C1078091C3069091C406DF
:10C0C0008093C207809194059091950597FD039602
:10C0D00095958795959587958093C30738C010925D
:10C0E000B8078EE48093B90788E08093BA078CE0A4
:10C0F0008093BB07809102018093BC0728C0809188
:10C100000A068093B807809135068093B90780911D
:10C110009F018093BA07809103068093BB078091AB
:10C1200004068093BC07809105068093BD0780912B
:10C130009E018093BE07809107068093BF07809180
:10C1400008068093C007809109068093C1078091FB
:10C15000C707882309F4B0C08AEF8093D4034091C5
:10C16000C9075091CA07CA0181509E4F8F5F934003
:10C17000B0F42091CB073091CC07C90181509E4F7C
:10C180008F5F934060F48091E30585FF08C0509372
:10C19000D2034093D1033093D0032093CF038091F7
:10C1A000CF079091D00721E08936920724F490932D
:10C1B000010380930003809100039091010320917B
:10C1C000FE023091FF02821B930B845E9D4F68E656
:10C1D00071E00E941E73845B90409093FD028093F7
:10C1E000FC022091D3073091D4078091FE019091F9
:10C1F000FF018217930740F480913304882321F4D0
:10C200003093FF012093FE018091C807992788365B
:10C21000910501F18936910524F48736910529F0BD
:10C2200053C08936910559F14FC08091D50780934D
:10C23000FC078091D6078093FE078091D7078093F3
:10C24000FD078091D8078093FF078091D9078093DD
:10C2500000083AC08091D50780939F078091D60748
:10C260008093A0078091D7078093A1078091D8077A
:10C270008093A2078091D9078093A30725C080915E
:10C28000D507809396078091D60780939707809172
:10C29000D707809398078091D9079091DA079093F8
:10C2A0009A07809399078091DB079091DC07909320
:10C2B0009C0780939B0708C01092D2031092D10371
:10C2C0001092D0031092CF031F910F91FF90EF9027
:10C2D000089580919507882309F43BC0459885EA25
:10C2E00097E090939E0780939D079091D303E92F49
:10C2F000FF27E054FE4F9F5F9093D303808180938C
:10C30000A707993010F01092D303109295070E945E
:10C31000625E81E08093A40700000000000000003E
:10C32000000000000000000000000000000000000D
:10C3300000000000000000000000000000000000FD
:10C3400000000000000000008091A5078093C40752
:10C350008EBD089587B18C6087B94298439810923A
:10C36000D80380E88093CA011092D7038093C90153
:10C3700008958091DD0381508093DD038F3F09F0A4
:10C38000F4C094E09093DD038091BD02807BE1F0E6
:10C3900080912106882349F08091E003882311F4DD
:10C3A0009093D80381E08093E00380912206882354
:10C3B000B9F08091E103882319F484E08093D703D6
:10C3C00081E08093E1030CC08093E0038093E1035C
:10C3D00080911D068093DE0380911F068093DF030A
:10C3E0008091E003882309F040C080913406282F13
:10C3F000332724FF07C08091E502882319F425FD27
:10C400004DC04EC090911E06983F50F080915C0741
:10C410008D3D30F08091DE0388230CF43FC040C096
:10C42000983F48F080915C078A3028F48091DE03C1
:10C430008823B4F133C08091D80381508093D8030E
:10C440008F3F79F580915C0781508093D80380916C
:10C45000CA01813011F480E801C086958093CA0139
:10C460008091CA019091DE0317C08091D80381505A
:10C470008093D8038F3FA9F489E08093D8038091FB
:10C48000CA01813011F480E801C086958093CA0109
:10C490008091CA0190912106892311F0429A01C02E
:10C4A00042988091E103882309F043C080913406CB
:10C4B000282F332724FF07C08091E502882319F431
:10C4C00026FD50C034C090912006983F50F08091D6
:10C4D00082078D3D30F08091DF0388230CF442C049
:10C4E00026C0983F48F0809182078A3028F48091D6
:10C4F000DF038823E4F036C08091D7038150809316
:10C50000D7038F3F91F58091820781508093D703A5
:10C510008091C901813011F480E801C08695809333
:10C52000C9018091C9019091DF038923D9F443980F
:10C5300008958091D70381508093D7038F3FA9F44A
:10C5400089E08093D7038091C901813011F480E89C
:10C5500001C086958093C9018091C90190912206FE
:10C56000892311F0439A0895439808954FB724E121
:10C5700030E0F8948091C9008F778093C900809152
:10C58000C9008F7B8093C9008091C9008F7D809303
:10C59000C9005A9A52985B9A539A832F992780938D
:10C5A000CD002093CC008091C80082608093C800A9
:10C5B00080E18093C9008091CA008F778093CA0080
:10C5C0008091CA008F7B8093CA008091CA008F7DC2
:10C5D0008093CA008091CA008F7E8093CA008091A8
:10C5E000CA00877F8093CA008091C9008B7F8093A7
:10C5F000C9008091CA0084608093CA008091CA00FB
:10C6000082608093CA008091C80087FF03C0809138
:10C61000CE00F9CF8091C90080688093C9004FBFD8
:10C620000895FF920F931F93CF93DF9380E197E2DA
:10C630000E940F15EC01FF248091C9008F77809331
:10C64000C9008091C9008F7E8093C9005A9883EEFB
:10C6500099E09F938F930DE311E11F930F93E09166
:10C66000FF03F091000409950F900F900F900F9029
:10C6700002C04A996CC0CE010E9418158823C9F3E4
:10C68000E091FF03F0910004FF2009F468C089E104
:10C690009AE09F938F931F930F930995529A0F904F
:10C6A0000F900F900F90CE010E9418158823D9F398
:10C6B00083E690E05A9A019797FFFCCF8FE891E0CC
:10C6C0005A98019797FFFCCF89E090E05A9A01971A
:10C6D00097FFFCCF89E090E05A98019797FFFCCF35
:10C6E0008FE891E05A9A019797FFFCCF8FE891E08D
:10C6F0005A98019797FFFCCF89E090E05A9A0197EA
:10C7000097FFFCCF89E090E05A98019797FFFCCF04
:10C710008FE891E05A9A019797FFFCCF8FE891E05C
:10C720005A98019797FFFCCF89E090E05A9A0197B9
:10C7300097FFFCCF89E090E05A98019797FFFCCFD4
:10C740008FE891E05A9A019797FFFCCF13C08AE5D2
:10C7500090E00E940F15EC0191E0F92E91CF8FE14E
:10C760009AE09F938F931F930F9309950F900F90CB
:10C770000F900F9052985A980E94B662E5E0CDB79C
:10C78000DEB70C949773EF92FF920F931F93CF93A2
:10C79000DF93482F00E010E08091CB01813061F4FD
:10C7A0001092CB0184E48093E2031092E403109290
:10C7B000E3031092E5032BC18091E203882319F46F
:10C7C00021E030E001C098019091E303992371F4D6
:10C7D000232B11F081E010C084E48093E203909356
:10C7E000E4039093E3039093E503FAC0913069F476
:10C7F000232B09F0EBC082E08093E3038091E403F4
:10C800008F5F8093E40383E0E9C09230D1F4232B5F
:10C8100009F0DCC083E08093E2034093E50390914C
:10C82000E403923039F41092E60347FF03C081E03D
:10C830008093E60383E08093E3039F5F9093E40398
:10C84000CFC0933009F0C2C0232B09F0BFC0909332
:10C85000E20382E08093E3038091E4038F5F80939F
:10C86000E4032091E503822F9927782F6627842FF0
:10C870009927682B792B8091FC05813049F47370DE
:10C88000CB018050924063E070E00E941E7317C09D
:10C89000823061F47770CB018050944066E070E0A4
:10C8A0000E941E732695269526950BC073706856B8
:10C8B0007140CB0177FD0196BC0175956795269572
:10C8C0002695022F11270F7010700F5F1F4F0D302C
:10C8D000110508F074C07801E00EF11EF701ED5368
:10C8E000F94F808191819B01281B390BC90137FFCA
:10C8F00003C0909581959F4F069794F48091EE0226
:10C90000883C30F48091EE02865F8093EE0208C08E
:10C9100088EC8093EE0280916F008F7D80936F0092
:10C92000F701ED53F94F808191819C01220F331F54
:10C93000280F391F260F371F37FF02C02D5F3F4FCB
:10C94000E901D595C795D595C795CB0101968C176B
:10C950009D0714F4219706C061507040C617D70791
:10C960000CF421968091EE02843BD0F0F701ED5358
:10C97000F94F80819181FE01E81BF90BCF0163E043
:10C9800070E00E941E73CB01880F991F860F971FBE
:10C9900027EF36E0E20EF31EF7019183808307C094
:10C9A00027EF36E0E20EF31EF70111821082000F2E
:10C9B000111F0D53194FF801D183C08311C00231EB
:10C9C000110570F081E08093CB010AC081E0809373
:10C9D000CB011092E4031092E60384E48093E20317
:10C9E0008091E403803198F08091E603882331F44C
:10C9F0008091CB01882311F4809391011092E4037C
:10CA00001092E6031092E30384E48093E203E6E0ED
:10CA1000CDB7DEB70C949673CF93FC0197FF05C09A
:10CA2000CFEFF095E195FF4F01C0C1E028E631E07E
:10CA3000CF01B9010E941E73FC018B35910554F0A2
:10CA40008B5590408A35910538F484EB90E08E1B2D
:10CA50009F0BFC0141E00DC0CF01855B90408A3502
:10CA6000910518F4E45BF04003C02E1B3F0BF90165
:10CA70004FEFEE0FFF1FE65DF54F259134918C2FA0
:10CA8000992787FD9095289FB001299F700D389FA9
:10CA9000700D1124842F992787FD9095689FA00120
:10CAA000699F500D789F500D1124CA01CF910895B0
:10CAB0002AE530E0281B390BC9010E940C65089556
:10CAC000CF93DF9380E00E947D6A80911D01909159
:10CAD0001E016AE070E00E941E739F938F93809105
:10CAE0001D0190911E016AE070E00E941E737F9309
:10CAF0006F9388EF9AE09F938F93C0E7DAE6DF9316
:10CB0000CF93E091FF03F091000409952DB73EB754
:10CB1000285F3F4F2DBF8091D403882339F186E0F1
:10CB20000E947D6A8FED90E09F938F9380919B0789
:10CB300090919C079F938F938091990790919A076A
:10CB40006AE070E00E940A737F936F9381E09BE03C
:10CB50009F938F93DF93CF93E091FF03F0910004B5
:10CB600009958DB79EB70A968DBF12C086E00E94C8
:10CB70007D6A8EE09BE09F938F93DF93CF93E0914C
:10CB8000FF03F091000409950F900F900F900F9004
:10CB900080E10E947D6A8091D0019091D1016CE387
:10CBA00070E00E940A739F938F938091D0019091BF
:10CBB000D1016CE370E00E940A737F936F938091C0
:10CBC0000508909106089F938F9385E19BE09F93C2
:10CBD0008F93DF93CF93E091FF03F09100040995C9
:10CBE0008091E3052DB73EB7265F3F4F2DBF80FFF5
:10CBF00029C08AE10E947D6A8091920199279F93C2
:10CC00008F938091E0029091E102A091E202B091B5
:10CC1000E302BC01CD0124E630E040E050E00E9498
:10CC200053733F932F9382E29BE09F938F93DF9305
:10CC3000CF93E091FF03F091000409958DB79EB763
:10CC400008968DBFDF91CF910895CF93DF9380E059
:10CC50000E947D6A89E29BE09F938F93C0E7DAE6AA
:10CC6000DF93CF93E091FF03F0910004099580E1F9
:10CC70000E947D6A0F900F900F900F9080918B070C
:10CC800090918C07A0918D07B0918E072091930110
:10CC9000309194014091950150919601BC01CD01D4
:10CCA0000E9453733F932F938091320390913303EB
:10CCB000A0913403B0913503B7FF04C081509C4F5D
:10CCC000AF4FBF4F3AE0B595A795979587953A95A1
:10CCD000D1F79F938F9380913A0390913B03A0915A
:10CCE0003C03B0913D03B7FF04C081509C4FAF4F50
:10CCF000BF4F2AE0B595A795979587952A95D1F7C7
:10CD00009F938F9388E39BE09F938F93DF93CF93C1
:10CD1000E091FF03F091000409958DB79EB70A9644
:10CD20008DBFDF91CF9108950F931F9380E00E94F4
:10CD30007D6A2AE030E08091010890910208B901F3
:10CD40000E940A739F938F9380910108909102082B
:10CD5000B9010E940A737F936F9380911D01909196
:10CD60001E01B9010E941E739F938F9380911D0134
:10CD700090911E01B9010E941E737F936F9384E40A
:10CD80009BE09F938F9300E71AE61F930F93E09128
:10CD9000FF03F0910004099580E10E947D6A8DB740
:10CDA0009EB70C968DBF80910508909106089F93C1
:10CDB0008F9380910308909104089F938F9387E548
:10CDC0009BE09F938F931F930F93E091FF03F0914C
:10CDD000000409958DB79EB708968DBF1F910F91DE
:10CDE00008950F931F93CF93DF938091D403C0E7EF
:10CDF000DAE6882309F490C080E00E947D6A809181
:10CE0000970799279F938F9383E69BE09F938F9338
:10CE10008E01DF93CF93E091FF03F0910004099519
:10CE20008DB79EB706968DBF80919807992782305F
:10CE3000910579F0833091051CF4892B21F019C0FC
:10CE4000039789F016C087E00E947D6A8CE69BE01C
:10CE500005C087E00E947D6A82E79BE09F938F93E5
:10CE6000DF93CF930FC087E00E947D6A88E79BE045
:10CE7000F5CF87E00E947D6A8EE79BE09F938F93BA
:10CE80001F930F93E091FF03F091000409950F9019
:10CE90000F900F900F908091960781FF14C089E04A
:10CEA0000E947D6A84E89BE09F938F9380E79AE6D7
:10CEB0009F938F93E091FF03F091000409950F90E9
:10CEC0000F900F900F9080E10E947D6A8FED90E0AF
:10CED0009F938F9380919B0790919C079F938F9333
:10CEE0008091990790919A076AE070E00E940A7316
:10CEF0007F936F938AE89BE09F938F9380E79AE6F6
:10CF00009F938F93E091FF03F091000409958DB7F3
:10CF10009EB70A968DBF12C082E00E947D6A8CE99E
:10CF20009BE09F938F93DF93CF93E091FF03F0916A
:10CF3000000409950F900F900F900F90DF91CF9103
:10CF40001F910F910895CF93C82F2091E70320934D
:10CF5000E80399278F32910509F1803391051CF47C
:10CF60004F97A1F02CC08F34910501F18F389105B6
:10CF700031F5222319F481E090E038C086E0289F43
:10CF8000F0011124E052F54F849117C086E0289FEC
:10CF9000F0011124EF51F54F84910FC086E0289FD6
:10CFA000F0011124EE51F54F849107C086E0289FCF
:10CFB000F0011124ED51F54F84918093E703909196
:10CFC000E7038091E8039813C0E00E94836A909180
:10CFD000E70386E0989FF0011124EC51F54F25916D
:10CFE00034918C2FF901099580E090E0CF9108955C
:10CFF000109202081092010810920608109205087B
:10D0000010920408109203088AE090E00E940F1525
:10D010009093EA038093E9030895CF93DF9380917F
:10D02000E9039091EA030E941815882309F4A8C027
:10D030008091E9039091EA030A969093EA03809322
:10D04000E903E0E0F0E09F0190E0A2E9B6E04BE008
:10D05000ED01898187FF07C09F5F8A81E80FF11D7D
:10D060008C91280F311D4150149647FFF1CF232B8F
:10D0700041F52091EF033091F0034091F10350917D
:10D08000F203BB27A52F942F832F9093EE03809359
:10D09000ED03AA27BB27281B390B4A0B5B0BCF01DB
:10D0A000AA27BB27280F391F4A1F5B1F2093EF03B6
:10D0B0003093F0034093F1035093F203E5E0F0E086
:10D0C00013C02091ED033091EE032E173F0718F4A3
:10D0D000E21BF30B02C0E0E0F0E0892F9927880FF4
:10D0E000991FE80FF91F3596F0930208E0930108A5
:10D0F000EF3FF10578F480911D0190911E018E9F04
:10D1000090018F9F300D9E9F300D1124C90164E660
:10D1100070E013C0CF0196958795969587952091DD
:10D120001D0130911E01289FA001299F500D389F9D
:10D13000500D1124CA0169E170E00E940A737093D6
:10D140000408609303082091EB033091EC032E0F49
:10D150003F1F3093EC032093EB035EE02131350752
:10D1600078F0809105089091060801969093060842
:10D170008093050820513E403093EC032093EB034D
:10D18000DF91CF9108954FB720E430E0F89480917B
:10D19000C9008F778093C9008091C9008F7B8093ED
:10D1A000C9008091C9008F7D8093C9005A9A529816
:10D1B0005B9A539A832F99278093CD002093CC00BC
:10D1C0008091C80082608093C80088E18093C90084
:10D1D0008091CA008F778093CA008091CA008F7BAC
:10D1E0008093CA008091CA008F7D8093CA0080918D
:10D1F000CA008F7E8093CA008091CA00877F809387
:10D20000CA008091C9008B7F8093C9008091CA00B9
:10D2100084608093CA008091CA0082608093CA00B3
:10D220008091C80087FF03C08091CE00F9CF809124
:10D23000C90080688093C9004FBF08950F931F9362
:10D24000CF93DF93482F4F5F893108F089C08091D9
:10D25000C206841710F44093C206CB0183539B424D
:10D2600068E170E00E941E73A42FBB27FD01EA0F46
:10D27000FB1FED53F94F808191819B01281B390BD6
:10D28000C90137FF03C0909581959F4F069794F48D
:10D290008091EE02883C30F48091EE02865F8093AC
:10D2A000EE0208C088EC8093EE0280916F008F7DC3
:10D2B00080936F00FD01EA0FFB1FED53F94F808152
:10D2C00091819C01220F331F280F391F260F371F12
:10D2D00037FF02C02D5F3F4FE901D595C795D59522
:10D2E000C795CB0101968C179D0714F4219706C0B2
:10D2F00061507040C617D7070CF421968091EE025A
:10D30000843BD8F08D010A0F1B1FF801ED53F94F34
:10D3100080819181FE01E81BF90BCF0163E070E091
:10D320000E941E73CB01880F991F860F971F09500B
:10D33000194FF8019183808307C0AA0FBB1FA95022
:10D34000B94F11961C921E92E42FFF27EE0FFF1F7C
:10D35000ED53F94FD183C083443011F41092910101
:10D36000DF91CF911F910F910895CF93DF9320917B
:10D370000708822F9927807F9070409709F06CC032
:10D380002F3109F046C0809108088093F70320915F
:10D390000A082093F90380910B088093F803822FE9
:10D3A00099279093C4068093C306222309F054C0A2
:10D3B0008091D705282F3327220F331FF901E95019
:10D3C000F94F118210828091D805A82FBB27AA0F90
:10D3D000BB1FFD01E950F94F118210828091DA05DF
:10D3E000E82FFF27EE0FFF1FCF018950994FEC0167
:10D3F000198218822D53394FE90119821882AD53D1
:10D40000B94F11961C921E92ED53F94F1182108262
:10D4100023C0C22FCF70CA30F8F4809108088093DF
:10D420003108809109088093300880910A08809320
:10D43000330880910B088093320860913008709116
:10D4400031088C2F0E941E69609132087091330858
:10D450008C2F8F5F0E941E69DF91CF910895CF932B
:10D46000C82F8F3F49F48091FA038F3F29F410921F
:10D47000FC031092FB0332C02091FC03222339F4F9
:10D48000CF3111F485E001C084E08093FD038091E9
:10D49000FD039091FB038217A0F4892F8095809360
:10D4A000FB038F3F19F48EEF8093FB038091FB0306
:10D4B000C81711F40E94B5691092FC031092FB0387
:10D4C0000BC0E22FFF27E95FF74FC0832F5F209348
:10D4D000FC039C0F9093FB03C093FA03CF91089534
:10D4E0009091F603933240F4E92FFF27E35FF74F63
:10D4F00080839F5F9093F6030895833218F48D5FC5
:10D500008093F603089590E2E0E1F8E08FE19193D3
:10D51000815087FFFCCF0895CF93CFB723E031E050
:10D52000F8948091C9008F778093C9008091C900D9
:10D530008F7B8093C9008091C9008F7D8093C90043
:10D540005A9A52985B9A539A832F99278093CD00C9
:10D550002093CC008091C80082608093C80088E14D
:10D560008093C9008091CA008F778093CA00809110
:10D57000CA008F7B8093CA008091CA00806280932A
:10D58000CA008091CA0080618093CA008091CA005D
:10D5900088608093CA008091C90084608093C9002C
:10D5A0008091CA0084608093CA008091CA00826022
:10D5B0008093CA008091C80087FF03C08091CE008D
:10D5C000F9CF8091C90080688093C9008091C9001B
:10D5D00080648093C9000E94836ACFBFCF91089571
:10D5E000282F99278F709070892B31F42095809186
:10D5F000F503822B8093F50308958091CE01882353
:10D6000009F441C08091BD0285FF0AC082E9809380
:10D610000D0883E280930E0885E580930F0802C011
:10D6200010920D088091CF018F3071F48091F50335
:10D630000E94A367882341F081E980930D088093BD
:10D640000E0881E380930F081092CE018091C800EC
:10D6500085FFFCCF8091C9008F7E8093C9008091A7
:10D66000C9008E7F8093C90080910D08882311F432
:10D670008EEF01C08EE78093CE008091F5038093FA
:10D68000CF011092F50308951F920F920FB60F92DB
:10D6900011248F939F93EF93FF939091CE01992341
:10D6A00009F040C08091FE03882361F480910D0849
:10D6B000882311F483E003C0813999F481E08093D9
:10D6C000FE030FC0833099F480910D08882349F040
:10D6D00090930D088091C9008E7F8093C9008EEFD2
:10D6E0001EC08091C90081608093C9000EC0833242
:10D6F00061F48091C9008E7F8093C9008FEF809381
:10D70000CE0081E08093CE0114C08091FE03E82F0B
:10D71000FF27E35FF74F8F5F8093FE038081809345
:10D72000CE0007C01092FE038091C90080618093F3
:10D73000C900FF91EF919F918F910F900FBE0F90B5
:10D740001F901895EF92FF920F931F93CF93DF9343
:10D750007C018B01EA01452B39F0F80181918F01A1
:10D76000F70109952197C9F7E6E0CDB7DEB70C942C
:10D770009673EF92FF920F931F93CF93DF937C01E9
:10D780008B01EA01452B41F0F8010F5F1F4F849197
:10D79000F70109952197C1F7E6E0CDB7DEB70C9404
:10D7A00096730F931F93CF938C01C62F161634F4E4
:10D7B00080E2F8010995C1501C16D4F3CF911F9156
:10D7C0000F9108950F931F93CF938C01C62F1616B8
:10D7D00034F480E3F8010995C1501C16D4F3CF91BD
:10D7E0001F910F910895A5E3B0E0E9EFFBE60C94DB
:10D7F0006E732E96EEADFFAD2E97882499245401BA
:10D800008091F403882321F42C961FAE1EAE2C9732
:10D810005EE4452E512C4C0E5D1E6F01B60105C015
:10D82000153239F00894C11CD11CF6011491112352
:10D83000B9F7A601461B570B31F02C968EAD9FAD64
:10D840002C970E94B96B112309F46AC20894C11C79
:10D85000D11CFF24FDA6FCA64FEFE42EF9A6F6018D
:10D860000894C11CD11C1491153721F0812F8062BE
:10D870008837B1F4F0FE0AC0F20124E030E0420E35
:10D88000531E80809180A280B3800AC0F20142E0E2
:10D8900050E0440E551E808191814C01AA24BB2486
:10D8A000103221F489A58823D1F61DC0133219F452
:10D8B00058E0F52AD4CF1A3211F01D3291F41A3201
:10D8C00059F4F20182E090E0480E591EE081ECA785
:10D8D000EE232CF6E195ECA790E1F92AAFEDFA22C0
:10D8E000BECF1B3211F419A7BACF1E32C1F5F60113
:10D8F0000894C11CD11C14911A3279F4F20122E06F
:10D9000030E0420E531E408151813FEF4F3F53079D
:10D9100014F44FEF5FEFE42EA2CF40E050E0812FF0
:10D9200080538A30A0F4CA0133E0880F991F3A95DA
:10D93000E1F7840F951F480F591F410F511D4053A8
:10D940005040F6010894C11CD11C1491E8CF8FEF10
:10D950004F3F580714F44FEF5FEFE42E85CF10339D
:10D9600029F4F4FC7CCF90E2F92A79CF812F8153FE
:10D970008930D8F440E050E0CA0123E0880F991FB5
:10D980002A95E1F7840F951F480F591F410F511D2C
:10D9900040535040F6010894C11CD11C1491812FB2
:10D9A00080538A3048F34CA75FCF183619F4A4E0AF
:10D9B000FA2A55CF1C3619F4B1E0FB2A50CF1336A2
:10D9C00061F43E010894611C711CF20122E030E018
:10D9D000420E531E808189833CC1143421F01436D9
:10D9E00011F0193651F5143411F431E0F32AF0FE38
:10D9F0000AC0F20144E050E0440E551E8080918040
:10DA0000A280B3800CC0F20182E090E0480E591E63
:10DA1000808191814C01AA2497FCA094BA2CB7FE76
:10DA20000AC0B094A09490948094811C911CA11C75
:10DA3000B11C8DE289A70AE06FC01F3411F01F36B8
:10DA400031F41F3411F491E0F92A08E064C0103772
:10DA500079F4F201A2E0B0E04A0E5B1E8081918170
:10DA60004C01AA24BB2400E1B0E4FB2A18E753C010
:10DA70001337C1F5F20122E030E0420E531E608000
:10DA800071806114710489F43E010894611C711C59
:10DA900088E289838EE6F301818385E78B838CE6B8
:10DAA0008C838D8389E28E831F82E7FC13C08E2DC9
:10DAB000992787FD9095AC0160E070E0C3010E945A
:10DAC0000A71009729F0382E3618E3140CF0C3C001
:10DAD0003E2CC1C0F30101900020E9F731973E2EA2
:10DAE0003618B9C0153511F0153731F4153511F464
:10DAF000F1E0FF2A0AE00FC0183519F0183709F0D5
:10DB0000A0C000E1F3FE07C081149104A104B10498
:10DB100011F020E4F22A19A6EDA6E7FC02C03FEDC1
:10DB2000F32289E2682E712C6C0E7D1E8114910403
:10DB3000A104B10421F44DA5442309F47BC0802F36
:10DB40009927AA27BB278EA79FA7A8ABB9AB202EE2
:10DB5000332490E0891690E0990691E0A90690E0C0
:10DB6000B90648F0C501B4012EA53FA548A959A999
:10DB70000E94317317C0AFEF8A169104A104B1045B
:10DB800049F040F0C401B1010E940A739B0144278F
:10DB9000552708C0882D602F0E94FE72282F33273A
:10DBA000442755272AAB3BAB4CAB5DAB0A3059F44D
:10DBB0008AA9880F880F880F9AA9990F890F382D85
:10DBC000381B832F10C0003139F48AA98295807FD9
:10DBD000482D481B842F07C08AA9880F880F880FFB
:10DBE000582D581B852F90E02EA53FA548A959A96F
:10DBF00082169306A406B50608F091E08AA89BA8B1
:10DC0000ACA8BDA88A3010F4805D04C0895A1835CC
:10DC100009F48F7DD3018E933D01992309F099CFAB
:10DC2000083041F4F3FE06C0803321F080E3FD01AB
:10DC300082933F01CE010196382E3618F8E23F0E4E
:10DC40000BC0112309F46CC03E010894611C711CC7
:10DC50001983B1E03B2E19A6032D2DA4231827FC10
:10DC6000222489A5882311F00F5F02C0F6FC0E5F05
:10DC7000020DEF2CFF24C70180739070892B49F4AB
:10DC80008CA5801B682F2C968EAD9FAD2C970E9483
:10DC9000D16B89A5882331F041E050E0BE01675D7A
:10DCA0007F4F0AC0E6FE0EC080E38AA71BA742E0B2
:10DCB00050E0BE01665D7F4F2C968EAD9FAD2C97D8
:10DCC0000E94A26BC70180739070809749F48CA565
:10DCD000801B682F2C968EAD9FAD2C970E94E26B17
:10DCE000622D2C968EAD9FAD2C970E94E26B832DFA
:10DCF000992787FD9095AC01B3012C968EAD9FAD11
:10DD00002C970E94A26BE4FE89CD2CA5201B2CA78A
:10DD1000622F2C968EAD9FAD2C970E94D16B7ECD3D
:10DD2000E2E1CB5C0C948A732FB740E0F894E0E01A
:10DD3000F0E081E2809357009491E2E0F0E080937C
:10DD400057003491E4E0F0E08093570084912FBFB6
:10DD50009E3199F4363941F4893011F441E00DC017
:10DD60008A3059F442E009C0373939F4863011F469
:10DD700043E003C0853009F444E0842F99270895D7
:10DD80009FB7F8948091C900877F8093C9008091E4
:10DD9000C9008F7E8093C9008091C9008F778093DE
:10DDA000C9008091C9008F7B8093C9008091C90010
:10DDB0008F7D8093C90052985A9A53985B9A9FBF5F
:10DDC00008951F93CF93DF93182F8091F403882336
:10DDD00009F48DC08091CD01181709F488C0809195
:10DDE000F303882321F40E94946E8093F30385E962
:10DDF0009CE09F938F93CDE3D1E1DF93CF93E091AC
:10DE0000FF03F091000409950F900F900F900F9071
:10DE1000812F99278230910501F1833091052CF4EF
:10DE2000009761F0019769F024C084309105D9F022
:10DE300084309105ACF00597C9F01BC085E89CE0E3
:10DE400002C083E79CE09F938F93DF93CF93E09191
:10DE5000FF03F0910004099518C08AE59CE0F3CF18
:10DE600087E39CE0F0CF89E29CE0EDCF81E29CE08B
:10DE7000EACF82EA9CE09F938F93DF93CF93E09168
:10DE8000FF03F0910004099510E00F900F900F90A0
:10DE90000F908091F303843011F0823099F40E9446
:10DEA000C06E812F8150833018F40E94B6621DC06D
:10DEB000143019F40E948C6A18C01530B1F40E9415
:10DEC000C36813C0112389F088EB9CE09F938F9364
:10DED0008DE391E19F938F93E091FF03F091000414
:10DEE00009950F900F900F900F901093CD01DF9137
:10DEF000CF911F9108950F931F9381E08093F403B6
:10DF00004091CC01E1EDFBE020E030E05FE4849162
:10DF100099272F5F3F4F829FB001839F700D929F83
:10DF2000700D112446275150319657FFF0CF409382
:10DF3000CC01E9EAFBE020E030E057E28491992748
:10DF40002F5F3F4F829FB001839F700D929F700D96
:10DF5000112446275150319657FFF0CF4093CC0102
:10DF60008091F303882321F40E94946E8093F3033D
:10DF70008091CC01833459F088E190E029E20FB61A
:10DF8000F894A895809360000FBE2093600083EF03
:10DF90009BE6909300048093FF0383ED9CE09F93A6
:10DFA0008F930DE311E11F930F93E091FF03F09125
:10DFB000000409950F900F900F900F9089E690E064
:10DFC0009F938F938EE490E09F938F931F921F9265
:10DFD000809102016AE00E94FE72892F99279F9327
:10DFE0008F93809102010E94FE7299279F938F93D5
:10DFF00089EF9CE09F938F931F930F93E091FF0312
:10E00000F0910004099581ED9BE09F938F931F93FE
:10E010000F93E091FF03F0910004099589EA9BE0DA
:10E020009F938F931F930F93E091FF03F091000450
:10E0300009958DB79EB746968DBF8DE29DE09F9363
:10E040008F931F930F93E091FF03F09100040995C4
:10E0500083EC8093810080916F00806280936F00D9
:10E060000F900F900F900F901F910F910895809136
:10E07000F403882361F08091CD01843011F40E9473
:10E08000FD6A8091CC01833411F01092F40308955D
:10E090001F920F920FB60F9211242F933F934F931D
:10E0A0005F936F937F938F939F93AF93BF93EF9300
:10E0B000FF932091CE009091CD01892F8150833024
:10E0C00020F4822F0E94C3630BC0943021F4822F6E
:10E0D0000E94F06A05C0953019F4822F0E942F6AC1
:10E0E000FF91EF91BF91AF919F918F917F916F9130
:10E0F0005F914F913F912F910F900FBE0F901F9006
:10E100001895002422273327442751E0BB27EE2708
:10E11000FF27A0E1660F771F881F991F001C221F91
:10E12000331F441F660F771F881F991F001C221F73
:10E13000331F441F2AF4050E2B1F3E1F4F1F04C020
:10E14000051A2B0B3E0B4F0B550FBB1FEE1F587FB5
:10E15000556047FD5250AA95E9F6E695B795579553
:10E16000E695B7955795852F9B2F0895222733273E
:10E1700041E0552768E0880F991F221F331F880F41
:10E18000991F221F331F1AF4240F351F02C0241BAE
:10E19000350B440F551F487F456037FD42506A9547
:10E1A00051F75695479556954795842F0895AA2778
:10E1B00097FF04C0809590958A1F9A1F77FF04C02F
:10E1C000609570956A1F7A1F669F9001779FA001E6
:10E1D000679F300D411D5A1F300D411D5A1F889FEA
:10E1E000F001999F2E0F3F1F401D511D899F300D3B
:10E1F000411D5A1F300D411D5A1FCA01B90111247A
:10E2000080CFFB01DC0102C005900D9241505040CF
:10E21000D8F70895FC014150504030F001900616A7
:10E22000D1F73197CF010895882799270895A0E065
:10E23000B0E0EDE1F1E70C9476736C017B01EA014B
:10E24000590121978FEFCF3FD80789F086010894B5
:10E25000C11CD11CC7010894E11CF11CF5010995F2
:10E26000F80180832197FFEFCF3FDF0779F7EAE0DE
:10E27000CDB7DEB70C949273CF92DF92EF92FF92FC
:10E280000F931F937C016B01FB010995082FC701B8
:10E290000196F6010995182FC8011F910F91FF9063
:10E2A000EF90DF90CF900895A0E0B0E0EAE5F1E7CD
:10E2B0000C9478738C017B01EA01690121978FEF3F
:10E2C000CF3FD80771F0F70121917F01C8010F5F9F
:10E2D0001F4F622FF60109952197FFEFCF3FDF0710
:10E2E00091F7E8E0CDB7DEB70C949473CF92DF924C
:10E2F000EF92FF920F931F936C018B017A01FA0149
:10E300000995812F9927682FC6010196F701099574
:10E310001F910F91FF90EF90DF90CF90089550588C
:10E32000BB27AA270ED00DC1FED030F003D120F0BC
:10E3300031F49F3F11F41EF4F3C00EF4E095E7FBB7
:10E34000E9C0E92F0FD180F3BA176207730784077A
:10E35000950718F071F49EF527C10EF4E0950B2E89
:10E36000BA2FA02D0B01B90190010C01CA01A00127
:10E370001124FF27591B99F0593F50F4503E68F182
:10E380001A16F040A22F232F342F4427585FF3CFC3
:10E39000469537952795A795F0405395C9F77EF494
:10E3A0001F16BA0B620B730B840BBAF09150A1F0DD
:10E3B000FF0FBB1F661F771F881FC2F70EC0BA0F63
:10E3C000621F731F841F48F4879577956795B795EB
:10E3D000F7959E3F08F0B3CF9395880F08F09927E3
:10E3E000EE0F97958795089571D008F481E0089510
:10E3F00004D06894B111D9C00895BCD088F09F575B
:10E4000090F0B92F9927B751A0F0D1F0660F771F80
:10E41000881F991F1AF0BA95C9F712C0B13081F060
:10E42000C3D0B1E00895C0C0672F782F8827B85FA8
:10E4300039F0B93FCCF3869577956795B395D9F7C1
:10E440003EF490958095709561957F4F8F4F9F4FCB
:10E450000895E89409C097FB3EF4909580957095D7
:10E4600061957F4F8F4F9F4F9923A9F0F92F96E920
:10E47000BB279395F695879577956795B795F11195
:10E48000F8CFFAF4BB0F11F460FF1BC06F5F7F4F32
:10E490008F4F9F4F16C0882311F096E911C0772344
:10E4A00021F09EE8872F762F05C0662371F096E84D
:10E4B000862F70E060E02AF09A95660F771F881F1C
:10E4C000DAF7880F9695879597F90895990F0008C0
:10E4D000550FAA0BE0E8FEEF16161706E807F90736
:10E4E000C0F012161306E407F50798F0621B730BD1
:10E4F000840B950B39F40A2661F0232B242B252B52
:10E5000021F408950A2609F4A140A6958FEF811DF4
:10E51000811D089597F99F6780E870E060E0089595
:10E520009FEF80EC089500240A941616170618062B
:10E530000906089500240A94121613061406050607
:10E540000895092E0394000C11F4882352F0BB0F98
:10E5500040F4BF2B11F460FF04C06F5F7F4F8F4FFB
:10E560009F4F089557FD9058440F551F59F05F3F36
:10E5700071F04795880F97FB991F61F09F3F79F0E5
:10E5800087950895121613061406551FF2CF469567
:10E59000F1DF08C0161617061806991FF1CF8695E9
:10E5A0007105610508940895E894BB2766277727CD
:10E5B000CB0197F908958ADF08F48FEF0895629FE1
:10E5C000D001739FF001829FE00DF11D649FE00D6B
:10E5D000F11D929FF00D839FF00D749FF00D659FCC
:10E5E000F00D9927729FB00DE11DF91F639FB00DCB
:10E5F000E11DF91FBD01CF0111240895991B79E098
:10E6000004C0991F961708F0961B881F7A95C9F7C2
:10E6100080950895AA1BBB1B51E107C0AA1FBB1F11
:10E62000A617B70710F0A61BB70B881F991F5A959E
:10E63000A9F780959095BC01CD01089597FB092E0F
:10E6400007260AD077FD04D0E5DF06D000201AF4B3
:10E65000709561957F4F0895F6F7909581959F4F3E
:10E660000895A1E21A2EAA1BBB1BFD010DC0AA1F13
:10E67000BB1FEE1FFF1FA217B307E407F50720F02B
:10E68000A21BB30BE40BF50B661F771F881F991FA6
:10E690001A9469F760957095809590959B01AC01EF
:10E6A000BD01CF01089597FB092E05260ED057FD19
:10E6B00004D0D7DF0AD0001C38F45095409530952F
:10E6C00021953F4F4F4F5F4F0895F6F790958095F6
:10E6D000709561957F4F8F4F9F4F08952F923F9276
:10E6E0004F925F926F927F928F929F92AF92BF9262
:10E6F000CF92DF92EF92FF920F931F93CF93DF930E
:10E70000CDB7DEB7CA1BDB0B0FB6F894DEBF0FBE6A
:10E71000CDBF09942A88398848885F846E847D84B7
:10E720008C849B84AA84B984C884DF80EE80FD80B9
:10E730000C811B81AA81B981CE0FD11D0FB6F8942F
:10E74000DEBF0FBECDBFED010895EE0FFF1F059098
:08E75000F491E02D0994FFCFC4
:10E758005E010A010164FF01FFFF01FC01FC0101E8
:10E76800737373FF03007D0000C409C409640010BB
:10E7780048656C6C6F20576F726C64000000000075
:10E788000000000000000000000000000000000081
:10E798000000000000000000000000000000000071
:10E7A8000000000000000000000000000000000061
:10E7B8000000000000000000000000000000000051
:10E7C80053706F727400004E6F726D616C0000427E
:10E7D8006567696E6E6572000051756164726F00DD
:10E7E8000001200B050000ECFF6440415A466464B8
:10E7F8000A02969696960840403A10FB30380190E7
:10E80800D0030090D00300F40164007800FF036493
:10E818000B0A0D0B0C0E0B0F1001010170FF010FFD
:00000001FF
